:020000040803EF
:10C00000E0E7002051C30308397604083B760408B2
:10C010004D7604084F7604085176040800000000AD
:10C02000000000000000000000000000B9C203088A
:10C030005376040800000000FDC20308A949040863
:10C040006BC30308A35204086BC3030867420408C8
:10C050006BC303086BC30308194004083940040884
:10C060005B4004087B4004089D400408133A040820
:10C07000553A0408973A0408E33A0408F93B0408DF
:10C08000493C0408993C04086BC303086BC30308CC
:10C090006BC303086BC303086BC30308BD400408EC
:10C0A0006BC303086BC303086BC303086BC30308AC
:10C0B000094C04082B4C04084D4C04086BC30308BE
:10C0C0006BC303086BC303086BC303086BC303088C
:10C0D0006BC30308D134040841350408B1350408A2
:10C0E000FF4004089F4204086BC303086BC30308A6
:10C0F0006BC303086BC303086BC303086BC303085C
:10C100006BC303086BC303086F4C04086BC30308BD
:10C110002136040895360408914C0408B34C0408F1
:10C12000E93C0408373D0408873D0408D33D040872
:10C1300000F002F800F0B0F80AA090E8000C824489
:10C140008344AAF10107DA4501D100F0A5F8AFF266
:10C15000090EBAE80F0013F0010F18BFFB1A43F0E5
:10C1600001031847D83C0100F83C01000A444FF095
:10C17000000C10F8013B13F0070408BF10F8014B46
:10C180001D1108BF10F8015B641E05D010F8016B8B
:10C19000641E01F8016BF9D113F0080F1EBF10F8EF
:10C1A000014BAD1C0C1B09D16D1E58BF01F801CB12
:10C1B000FAD505E014F8016B01F8016B6D1EF9D595
:10C1C0009142D6D3704700000023002400250026AA
:10C1D000103A28BF78C1FBD8520728BF30C148BFEA
:10C1E0000B6070476E290EF0CF8370290EF0B58476
:10C1F000662912F09A80652912F09780672912F05B
:10C200009480612912F0938003681B0A28BF41F0D3
:10C21000800169290EF07C8364290EF079837529E9
:10C220000EF076836F290EF0428478290EF0818417
:10C23000E9290FF03782E4290FF03482F5290FF055
:10C240003182EF290EF03F84F8290EF080840368D4
:10C25000DB0928BF41F0800163290FF0EE817329CB
:10C260000FF0F381E3290FF01182F3290FF016820A
:10C27000002070471FB50FF0AFFA04000020002126
:10C2800011F07EF9401C60600020002111F08EF951
:10C29000E0601FBD10B510BD0FF06CFD1146FFF73B
:10C2A000E9FF00F099FE0FF098FD03B4FFF7F2FFED
:10C2B00003BC06F0DEFE0000224B19680868B0E8F7
:10C2C000F00F80F30988BFF36F8F4FF0000080F309
:10C2D00011884EF00D0E70470000000006480068FF
:10C2E000006880F3088862B661B6BFF34F8FBFF372
:10C2F0006F8F00DF00BF00BF08ED00E0EFF30980A3
:10C30000BFF36F8F0F4B1A6820E9F00F106008B56C
:10C310004FF0500080F31188BFF34F8FBFF36F8F42
:10C320000DF0F4F84FF0000080F31188BDE80840EC
:10C3300019680868B0E8F00F80F30988BFF36F8FC1
:10C34000704700BF8C060020EFF3058070470000A7
:10C350000948804709480047FEE7FEE7FEE7FEE799
:10C36000FEE7FEE7FEE7FEE7FEE7FEE704480549D5
:10C37000054A064B704700005F77040831C1030887
:10C38000E0B70020E0E70020E0C70020E0C7002081
:10C39000F94C20460CF0E6FFFBE708B500254FF40A
:10C3A00000761CE020460EF02BFD217828290CD1C8
:10C3B00094F82510262908D1221812F8051C2429E2
:10C3C00003D112F8031C292916D02146EBA006F050
:10C3D00087FA204606F080FA32200CF0C3FF304680
:10C3E00006F040FA044600956A462146EB4806F0FE
:10C3F000A3FB0028EDD1D5E76278412A15D0632A46
:10C4000008D02146E6A006F06BFAEDA1522002F01A
:10C4100081FCDEE782B22146F04806F03EFB0028B0
:10C42000D7D0EFA006F0B6FAD3E72146F1A006F088
:10C4300057FACEE71CB50027DFF8D8834FF48069A0
:10C4400057E0F5A1304606F0B5FC0546002D46DB69
:10C450004FF4007006F006FA04464FF48070009026
:10C46000711900230A22204606F0D5FB20460EF063
:10C47000C7FC217828290CD194F82510262908D149
:10C48000211811F8052C242A03D111F8031C29299D
:10C4900007D02146E4A006F023FA204606F01CFA55
:10C4A00021E06178412915D0432908D02146E6A032
:10C4B00006F016FAECA1522002F02CFCEDE782B255
:10C4C0002146C64806F0E9FA0028E6D0C4A006F0E6
:10C4D00061FAE2E72146EBA006F002FADDE7314619
:10C4E000F0A006F057FA304606F0F6F903200CF0FB
:10C4F00039FF0221D8F800000BF001FD484606F094
:10C50000B1F90646019701AA3146ED4806F014FB41
:10C510000028E8D195E708B5EA4C0025BD4E4FF458
:10C52000807717E0BDF80010404605F026FE10B3F6
:10C53000022836D003283BD0042827D0E2A006F0FA
:10C5400029FAE1A004F02BFE404606F0C5F932209E
:10C550000CF008FF042130680BF0D1FC384606F0DF
:10C5600081F9804600956A464146DC4806F0E4FAC7
:10C570000028E9D1D6E7042120680BF0E7FDD8A018
:10C5800006F008FAD6A004F00AFEDDE70F212068C5
:10C590000BF0DCFDD7A006F0FDF9D6A004F0FFFDFE
:10C5A000D2E7D8A006F0F6F9D6A004F0F8FDCBE764
:10C5B000D9A006F0EFF9D8A004F0F1FDC4E708B562
:10C5C0000025944C4FF400760AE0BDF80010384680
:10C5D00001F047FD384606F07FF932200CF0C2FE2C
:10C5E000202120680BF08BFC304606F03BF9074613
:10C5F00000956A463946794806F09EFA0028E9D146
:10C60000E3E71CB5AF4C834D4BE04FF4806006F080
:10C6100029F906460020019001AA3146C24806F0D9
:10C620008BFA002837D14FF4CC72C0A141F2707060
:10C6300000F0FEFDBDF804203146BE4805F021FDA6
:10C64000032811D0BDF804203146BA4805F019FD81
:10C65000032809D0042120680BF078FDB6A006F06D
:10C6600099F9B5A004F09BFDB84800231A46194675
:10C6700000680BF05BFF1921B5480EF0B6FC4FF4D3
:10C68000D2700090A9A3B3A21921B1480EF0C2F84C
:10C69000AF4806F025F9304606F01EF932200CF0BE
:10C6A00061FE082128680BF02AFC002120680BF0AD
:10C6B0004DFDC0434007F1D4A7E708B54FF47A66B3
:10C6C000544C804D4CE040F2B31298A141F270708E
:10C6D00000F0AEFDA348074605F033FAA148401F1D
:10C6E000804604F015FF43463A469FA1482002F0D9
:10C6F00011FB964800231A46194600680BF016FFF6
:10C70000192193480EF071FC40F2B710009087A3F6
:10C7100090A219218E480EF07DF88D4806F0E0F8C1
:10C72000102006F09FF88146434696A21021484605
:10C730000EF070F8484602F0F2F9102148460EF06B
:10C7400054FC3B4691A2102148460EF063F848463F
:10C7500002F0C8F9484606F0BFF830460CF002FE79
:10C76000102120680BF0CBFB002128680BF0EEFCB9
:10C77000C0434007F1D4A6E7A0860100555342CA42
:10C78000D5B5BDCFC2D0D027B7C727B7A8CAFDBE81
:10C79000DDD6A1A3BA2573202E0000006C10002066
:10C7A000555342CAD5B5BDCFC2D0D0CEB4D6AAC09B
:10C7B000E0D0CDCAFDBEDDD6A1A3BA2573202E00E0
:10C7C000555342CAD5B5BDCFC2D0D0CEB4D6AAC07B
:10C7D000E0D0CDCAFDBEDDD6A10000006807002074
:10C7E0007355736572636D645175657565D2E7B392
:10C7F000F6A3A100555342C9CFCEBBBBFAC8B7C8F8
:10C80000CFCAD5B5BDCAFDBEDDD6A1A3BA2573205A
:10C810002E000000400000202B51495552433A2081
:10C820002272656376220000544350CAD5B5BDCF4D
:10C83000C2D0D027B7C727B7A8CAFDBEDDD6A1A3EF
:10C84000BA25732000000000544350CAD5B5BDCFAF
:10C85000C2D0D0CEB4D6AAC0E0D0CDCAFDBEDDD6FF
:10C86000A13A257320000000544350CAD5B5BDCF6E
:10C87000C2D0D0CEB4D6AAC0E0D0CDCAFDBEDDD6DF
:10C88000A100000054637020736572766572C8B7AA
:10C89000C8CFCAD5B5BDCAFDBEDDD6A13A25732025
:10C8A0000000000054435020CFC2D0D0CAFDBEDDEE
:10C8B000BDE2CEF6CAA7B0DCA3BA25732000000003
:10C8C0004C1F00203C00002054637020756E6B6E7E
:10C8D0006F776E20757263202E00000052230020B7
:10C8E0005463702073657276657220636C6F736534
:10C8F00064202E00546370205044502064656163AE
:10C9000074202E0054637020696E636F6D696E67CA
:10C910002066756C6C202E0054637020696E636F06
:10C920006D696E67202E0000660C00206D61696ED7
:10C930002E630000AA0100205463702053656E64CA
:10C94000446174612045727221000000440000209F
:10C95000FA060020257320256420CACDB7C54543BB
:10C9600032302100AE1C00204353513A25732C2055
:10C970004543323020566F6C746167653A25736D9C
:10C980005600000025736D560000000043535125EA
:10C990007300000001F052FC14200CF0E3FCF9E7F6
:10C9A00008F0D6F903F082FE64200CF0DBFCF7E718
:10C9B00008B500244FF4806509E03146FEA005F07B
:10C9C0008FFF304605F088FF64200CF0CBFC284632
:10C9D00005F048FF064600946A463146FB4806F0DB
:10C9E000ABF80028EDD1E8E708B500244FF48065E6
:10C9F00009E03146F6A005F073FF304605F06CFF04
:10CA000064200CF0AFFC284605F02CFF064600948D
:10CA10006A463146F34806F08FF80028EDD1E8E782
:10CA200008B50026F04DF14C4FF4FA78F04F03E1D1
:10CA30002E70FEE02878401CC1B22970022904D96A
:10CA4000ECA004F0ACFB0AF02BFEAF22AFF22411F5
:10CA500041F2707000F0ECFB002120680BF076FBD7
:10CA6000C043C0070CD0E9A002F018F804F0EFFDB5
:10CA700003280DD0E7A004F092FBEAA005F030FFF8
:10CA8000002120680BF062FBC043C00708D02AE0F9
:10CA9000012120680BF033FAE5A005F021FFEFE754
:10CAA000002120680BF052FBC04380071BD5E3A098
:10CAB00001F0F4FF1E2005F0D5FE81461E214846F8
:10CAC00005F057F8032816D0484604F068FB0F21FC
:10CAD00020680BF03BFB04F0DBFD484605F000FF4F
:10CAE000484605F0F9FE002120680BF02FFBC043FB
:10CAF000C00705D023E0022120680BF000FAECE724
:10CB0000002120680BF022FBC043800717D40021CE
:10CB100020680BF01BFBC043400710D5C9A001F0F3
:10CB2000BDFF02F0DAF8032811D0042120680BF0D1
:10CB30000DFBC8A005F0D4FEC9A004F030FB002115
:10CB400020680BF003FBC043C0070CD027E0042192
:10CB500020680BF0D4F9C6A14C2002F0DBF8CAA083
:10CB600005F0BEFEEBE7002120680BF0EFFAC043B2
:10CB7000800714D4002120680BF0E8FAC0430007B6
:10CB80000DD505F0D2FC032811D0082120680BF048
:10CB9000DDFAC0A005F0A4FEC2A004F000FB002155
:10CBA00020680BF0D3FAC04300071CD025E0082111
:10CBB00020680BF0A4F9BFA001F070FF02F06CF93F
:10CBC0008146BEA14C2002F0A5F8B9F1030F04D0B4
:10CBD000BFA004F0E4FA0AF063FDC7A005F080FEF0
:10CBE00000F094FBDBE7C84804F0ABFFC648401FE9
:10CBF00004F08EFC01F0B1FF2E70C44800231A46E9
:10CC0000194600680BF092FC1921C1480EF0EDF9AD
:10CC10004FF48470AFF2EC23AFF2C82200901921D8
:10CC2000BB480DF0F7FDBA4805F05AFEB9A005F073
:10CC300057FE40460CF096FB012138680BF05FF977
:10CC4000002120680BF082FAC04300077FF4F2AEA7
:10CC5000EEE67CB508F07CF80BF0B7F800F0C0FA0F
:10CC600001F06FFB0BF03EF9614908600BF03AF9F7
:10CC70005E49086001200BF02CFDA4490860A9481A
:10CC8000012300901A466421A7A00DF094FC564C95
:10CC9000A0630CF0C7FD024600200346009001216E
:10CCA000A06B0DF0D7FA08F053F8022104F1080048
:10CCB0000023CDE90010CE0132469FA1AFF29F20A4
:10CCC0000CF061F9092104F10C00CDE900100023FA
:10CCD00032469BA1AFF2EF200CF055F9052104F18B
:10CCE0001000CDE900100023324698A1AFF23F308A
:10CCF0000CF049F91F2104F11400CDE900100023C4
:10CD0000802295A1AFF267300CF03DF9032504F1C4
:10CD10002000CDE900500023324691A1AFF28B30C4
:10CD20000CF031F9062104F12C00CDE900100023AC
:10CD300080228EA1AFF27D600CF025F9072104F16D
:10CD40002800CDE90010002332468CA1AFF24D70CF
:10CD50000CF019F91D2104F13000CDE90010002379
:10CD6000324689A1AFF2A9700CF00DF904F1180058
:10CD7000CDE900500023324686A1AFF665000CF0E5
:10CD800002F9012504F11C00CDE9005000236A02DC
:10CD900083A1AFF65F100CF0F6F804F13400CDE992
:10CDA00000500023324681A1AFF611200CF0EBF8C1
:10CDB00004F124002021FFE05273343835207265DD
:10CDC00063646174613A2573202E00007818002096
:10CDD000527332333220726563646174613A257331
:10CDE000202E000072140020000000203C000020D3
:10CDF00040000020CFB5CDB3CDF8C2E7B1C0C0A38D
:10CE0000A3ACD6D8C6F4CFB5CDB32100CED5CAD603
:10CE1000D6D03A00C4A3BFE9B0B2D7B0D2ECB3A326
:10CE200021000000CED5CAD6CAA7B0DC00000000A1
:10CE3000CED5CAD6B3C9B9A600000000C8EBCDF85C
:10CE4000D6D03A00C1ACBDD3544350B7FECEF1C6E4
:10CE5000F73A0000544350C1ACBDD3CAA7B0DC00C0
:10CE6000544350C1ACBDD3CAA7B0DC2100000000C0
:10CE70004465766963652074637020636F6E6E65C8
:10CE80007463656421000000544350C1ACBDD3B34A
:10CE9000C9B9A60048545450B3F5CABCBBAFCAA721
:10CEA000B0DC000048545450B3F5CABCBBAFCAA7AD
:10CEB000B0DC2100D7A2B2E1D6D03A004465766951
:10CEC0006365205265676973746572210000000014
:10CED00048747470B3F5CABCBBAF4F4BA3ACD7A2B8
:10CEE000B2E1C7EBC7F3CAA7B0DCA3ACD6D8C6F48F
:10CEF000CFB5CDB321000000D3B2BCFED7A2B2E1C2
:10CF0000B3C9B9A6A3A10000AE1C002044000020B4
:10CF1000FA060020CACDB7C545433230D7CAD4B4CB
:10CF2000210000000DD30308526566726573682006
:10CF300054696D65000000004E65745461736B00A8
:10CF400052733233325461736B00000052733438C1
:10CF5000355461736B0000004C65645461736B0061
:10CF60004D656E755461736B00000000546370482A
:10CF7000656172745461736B0000000054637055F6
:10CF8000705461736B00000055636D645461736B82
:10CF9000000000005463705572635461736B0000AD
:10CFA000546370446F776E5461736B0044656275AF
:10CFB000675F7461736B0000CDE900100023324697
:10CFC0001AA1AFF633400BF0DEFF60680CF024F8D6
:10CFD000BDE87C400AF013BF1CB54FF470314FF030
:10CFE000006008F09AF907F0B3FE4FF4407008F0C3
:10CFF0005FF9114800F064FA104800F0EEFA1048AA
:10D0000000F09FF90F4803F0D3FB07F0A1FE0E4894
:10D010002021CDE900100023CA000CA1AFF2CD30D1
:10D020000BF0B1FF0CF0C0FB00201CBD4C69737409
:10D030005461736B000000006E0B0020580000204C
:10D040002B07002024650300040000207374617224
:10D05000745F7461736B000000B585B01322BF4923
:10D0600068460DF043FF9DF80900401C8DF809004B
:10D07000BBA00088ADF80B00684607F0E7FBB74897
:10D0800004F08DF8B7A004F08AF80AF009FB05B0A7
:10D0900000BD70B505460C467B2008F0E3FA012878
:10D0A00004D12246B4A128460DF0E8FF7C2008F008
:10D0B000D9FA012804D12246B2A128460DF0DEFF9C
:10D0C0007D2008F0CFFA012804D12246B0A12846DD
:10D0D0000DF0D4FF7E2008F0C5FA012804D12246C5
:10D0E000AFA128460DF0CAFF7C2008F0BBFA88B932
:10D0F0007D2008F0B7FA68B97E2008F0B3FA48B985
:10D100007A2008F0AFFA012804D12246A8A12846C7
:10D110000DF0B4FFBDE8704008F0CBBB10B504467D
:10D120000B2204F119000DF0A9FF002084F825005E
:10D1300010BD10B504460B2204F125000DF09EFF32
:10D14000002084F8310010BD30B5A1B09B480DF02F
:10D150003FFB9B480DF03CFB9A4C9B48211DFFF781
:10D16000E8FF994B0B222533002198A00DF030FBEE
:10D1700095481930054607F00DF829469248FFF703
:10D18000CDFF294696A00DF023FBA17898A0303959
:10D190000DF01EFB01218C4807F005F88A4A182182
:10D1A00098A00DF015FB88480B2131300446FFF79D
:10D1B00070FF22460B2198A00DF00AFB7F480DF06E
:10D1C00007FB802101A80DF032FF234697A28021A2
:10D1D00001A80DF01FFB01A803F0E1FF21B030BD55
:10D1E00010B507F0F7FB03F0B7FF002005F042FE93
:10D1F0000F2007F099F9FFF7A7FFAFF2A311022064
:10D2000006F0F8FF00F0F2FF03F04BFA03F0AFFA7C
:10D2100007F044FF03F0CAFB4FF4E134204603F06B
:10D22000F7FA204603F026FBBDE8104008F011B8DD
:10D23000FEB50D4614460246804800231946006894
:10D240000BF093FA01281CD0C02005F00BFB06461A
:10D250005D48CDE901543138A0F11E03009078A259
:10D26000C02130460DF0D6FA304603F098FF304624
:10D2700005F036FB304605F02FFBBDE8FE400AF016
:10D280000FBA51481E214F380DF0AFFE4E482B46C5
:10D2900079A21E214F3800940DF0BCFABDE8FE4083
:10D2A00049484F3805F01CBB2DE9F041764D4FF44D
:10D2B0008078404605F0D6FA0746744E7068C0F391
:10D2C0000F240BE042463946284607F043FD3A4614
:10D2D0006FA14C2001F01EFD05F58075641EA4B2FF
:10D2E000F0D2414638460DF080FE32793946284664
:10D2F00007F030FD3A4666A14C2001F00BFD3846A0
:10D3000005F0EAFABDE8F04103F0DEBE10B563486F
:10D310000078002814D12C481022104913380DF041
:10D3200014FD48B100F0E6FF27481422BDE8104084
:10D330000A4913380DF0A2BEBDE8104001F0B7BB9A
:10D3400010BD002140F8191F41608160C16001617A
:10D350004161193819210DF048BE0000045C00201D
:10D36000303100005274635F416C725F43616C6CDA
:10D370006261636B21000000D6D8C9CFB5E7C6F45F
:10D38000B6AF0000C8EDB8B4CEBBC6F4B6AF00006F
:10D39000B6C0C1A2BFB4C3C5B9B7C6F4B6AF00002A
:10D3A000B4B0BFDABFB4C3C5B9B7C6F4B6AF0000F6
:10D3B000D3B2B8B4CEBBC6F4B6AF00003CF9040893
:10D3C00080F904086E0B00202B0700200D0A426F25
:10D3D0006F74B0E6B1BE203A20252A2E2A730000D1
:10D3E0000D0A41505020B0E6B1BE203A202573000E
:10D3F0000D0A52756E4170704E756D3A2041505055
:10D40000256400000D0AC9E8B1B8B1E0BAC5203AF8
:10D4100020252E2A730000000D0AD6D8C6F4D4ADFC
:10D42000D2F2203A20252E2A73000000D6D8C6F466
:10D43000D4ADD2F23A25732E000000004400002043
:10D44000C9CFB4CE3A25732C20C9CFB4CE3A2573B8
:10D450002C20B5B1C7B0257320256420C7C0D5BC2A
:10D4600045433230CAA7B0DCA3ACCFB5CDB3C8EDCD
:10D47000D6D8C6F4A3A10000257320256420C7C018
:10D48000D5BC45433230210000F80708801C00203D
:10D49000B1BEB5D86C6F673A257300005C00002000
:10D4A000F8220146F74807F0F8BC10B5F8210DF056
:10D4B0009CFDBDE81040F822F349F24807F04ABC51
:10D4C0007CB50446F14805F0DFFA2046FFF7EDFF92
:10D4D0005B202070302060703220A0703120E0701E
:10D4E000207CFF2809D104F11000402105460DF0F1
:10D4F0007CFDE7A128460DF054FC94F85000FF286D
:10D5000009D104F15000402105460DF06EFDE2A165
:10D5100028460DF046FC94F89000FF2809D104F14C
:10D520009000402105460DF060FDDCA128460DF07D
:10D5300038FC94F8D000FF2809D104F1D000102164
:10D5400005460DF052FDD9A128460DF02AFC94F8AD
:10D55000E000FF2816D0A8B1CB49D848E03101F04F
:10D560009FFB94F8F000FF2817D0B0B1C649D3480C
:10D57000F03101F0A2FB5D2084F8F7002046BDE801
:10D580007C408DE704F1E000102105460DF02DFDF3
:10D59000C6A128460DF005FCE3E70020C4F8F00022
:10D5A000A4F8F400009001900A22694641F6583030
:10D5B00005F089FB694604F1F0000DF0F2FBDAE7B3
:10D5C00001460322BE4807F068BC00220280827038
:10D5D00001460322BA4807F0BDBB10B504462046F9
:10D5E000FFF7F3FF2046BDE81040E9E72DE9F041E1
:10D5F00005460F46032640F2492005F033F904465C
:10D600003B464FF40077AFA2394604F126000DF0F7
:10D6100001F9002801DDB8420BDD40F2A722AAA1E2
:10D62000AEA005F0B7F9204605F056F90220BDE896
:10D63000F08128222270642190FBF1F23032A27036
:10D6400090FBF1F201FB12020A2192FBF1F230325F
:10D65000E27090FBF1F201FB120030302071A6491C
:10D6600008786071401CC0B20870392801D9302098
:10D6700008700422A1A1A01D0DF000FD012104F1FC
:10D680000A0006F090FD3B2184F82210B5F8231023
:10D69000A4F82310262184F82510687843280ED09A
:10D6A00072216170032297A120460DF03CFB2046B9
:10D6B00005F016F9204605F00FF93046B7E752217C
:10D6C000617003228FA120460DF02DFB20460DF046
:10D6D00097FB82B221468C4805F0DFF90028E9D09B
:10D6E00040F2C12278A189A005F054F9E2E7532065
:10D6F00070472DE9F04707463C46A078217930383D
:10D7000000EBC00202EB001001EB8001E0786FF04B
:10D710002F02303800EB800002EB40000D18DFF8DC
:10D7200064A1F8225849504607F014FB4FF4807664
:10D73000304605F097F88046534B7CA2F03399466B
:10D74000314640460DF066F8064694F8230031282D
:10D7500004D1611991F82610242902D030281DD057
:10D7600021E0102148460DF040FC2A4604F1260134
:10D7700048460DF083FCF8224349504607F08DFBE4
:10D78000C6F5807108EB06004B466DA20DF042F81D
:10D79000532441463846FFF729FF05E0601990F809
:10D7A0002600242806D04924404605F095F8204656
:10D7B000BDE8F087532441463846FFF717FFF3E7EB
:10D7C0002DE9F04707463C46A0782179303800EB38
:10D7D000C00202EB001001EB8001E0786FF02F0235
:10D7E000303800EB800002EB40000D18DFF894A009
:10D7F000F8222549504607F0ADFA4FF480763046BE
:10D8000005F030F88046204B52A2E033994631466D
:10D8100040460CF0FFFF064694F82300312804D15F
:10D82000611991F82610242902D030281DD021E05A
:10D83000102148460DF0D9FB2A4604F1260148463E
:10D840000DF01CFCF8221049504607F026FBC6F5E7
:10D85000807108EB06004B4643A20CF0DBFF53241B
:10D8600041463846FFF7C2FE05E0601990F82600F1
:10D87000242805D04924404605F02EF8204697E795
:10D880007CE00000008801086E0B00206807002083
:10D890002F41424D0000000041424D0053686F701F
:10D8A0003334343739343734390000003132312ED3
:10D8B00034312E37392E383700000000AA010020FD
:10D8C000009001082573000055534552434D445CB8
:10D8D00075736572636D642E6300000025732C25DB
:10D8E000643A757044617461427566207370696C46
:10D8F0006C6F766572A3A100480000204D41433A49
:10D900000000000024582900660C002025732C25F7
:10D91000643A73546370305175657565207370692E
:10D920006C6C6F766572A3A1000000002A47455415
:10D930002A20546370506F72743A5B25735D210026
:10D940002A5345542A20546370506F72743A5B25F1
:10D95000735D21002A4745542A2054637049503A88
:10D960005B25735D210000002A5345542A2054632F
:10D970007049503A5B25735D2100000053244146F5
:10D980003846FFF733FE76E72DE9F04707463C4679
:10D99000A0782179303800EBC00202EB001001EBD7
:10D9A0008001E0786FF02F02303800EB800002EB4E
:10D9B00040000D18DFF8F4A3F822FB49504607F0A9
:10D9C000C9F94FF48076304604F04CFF8046F64BA0
:10D9D000F7A2D0339946314640460CF01BFF06466D
:10D9E00094F82300312804D1611991F826102429D4
:10D9F00002D030281DD021E0102148460DF0F5FA64
:10DA00002A4604F1260148460DF038FBF822E64983
:10DA1000504607F042FAC6F5807108EB06004B4607
:10DA2000E8A20CF0F7FE532441463846FFF7DEFD2E
:10DA300005E0601990F82600242805D049244046C6
:10DA400004F04AFF2046B3E6532441463846FFF728
:10DA5000CDFDF4E72DE9F04707463C46A078217953
:10DA6000303800EBC00202EB001001EB8001E078DF
:10DA70006FF02F02303800EB800002EB40000D18F1
:10DA8000DFF828A3F822C849504607F063F94FF49D
:10DA90008076304604F0E6FE8046C34BCEA290333B
:10DAA0009946314640460CF0B5FE064694F82300F0
:10DAB000312804D1611991F82610242902D0302888
:10DAC0001DD021E0402148460DF08FFA2A4604F18E
:10DAD000260148460DF0D2FAF822B349504607F025
:10DAE000DCF9C6F5807108EB06004B46C0A20CF0CD
:10DAF00091FE532441463846FFF778FD05E0601952
:10DB000090F82600242805D04924404604F0E4FE7D
:10DB100020464DE6532441463846FFF767FDF4E7BB
:10DB20002DE9F04707463C46A0782179303800EBD4
:10DB3000C00202EB001001EB8001E0786FF02F02D1
:10DB4000303800EB800002EB40000D18DFF85CA2DB
:10DB5000F8229549504607F0FDF84FF4807630469C
:10DB600004F080FE8046904BA7A250339946314680
:10DB700040460CF04FFE064694F82300312804D1AD
:10DB8000611991F82610242902D030281DD021E0F7
:10DB9000402148460DF029FA2A4604F1260148465C
:10DBA0000DF06CFAF8228049504607F076F9C6F578
:10DBB000807108EB06004B4699A20CF02BFE532413
:10DBC00041463846FFF712FD05E0601990F826003F
:10DBD000242805D04924404604F07EFE2046E7E58F
:10DBE000532441463846FFF701FDF4E72DE9F0479D
:10DBF00007463C46A0782179303800EBC00202EBA2
:10DC0000001001EB8001E0786FF02F02303800EB5C
:10DC1000800002EB40000D18DFF890A1F822624965
:10DC2000504607F097F84FF48076304604F01AFE1D
:10DC300080465D4B80A210339946314640460CF039
:10DC4000E9FD064694F82300312804D1611991F8C2
:10DC50002610242902D030281DD021E0402148463A
:10DC60000DF0C3F92A4604F1260148460DF006FAE4
:10DC7000F8224D49504607F010F9C6F5807108EBBF
:10DC800006004B4672A20CF0C5FD532441463846AF
:10DC9000FFF7ACFC05E0601990F82600242805D0B9
:10DCA0004924404604F018FE204681E553244146AD
:10DCB0003846FFF79BFCF4E72DE9F84307463C465E
:10DCC000DFF8E890F8223849484607F043F84FF467
:10DCD0008075284604F0C6FD06466348804606F077
:10DCE00059FACDF80080DFF8C08060A2294698F884
:10DCF000023030460CF08EFD054694F823003128A2
:10DD000004D167A1A01C05F055F820B194F82300B8
:10DD1000302821D025E094F82600302807D031287B
:10DD200005D0322803D0332801D050241AE088F8D7
:10DD30000200F8221C49484607F0AFF898F8023074
:10DD4000C5F58071701957A20CF064FD532431465B
:10DD50003846FFF74BFC05E051A1A01C05F02AF85E
:10DD600030B14924304604F0B7FD2046BDE8F883C1
:10DD7000532431463846FFF739FCF3E72DE9F047E5
:10DD800007463C46DFF82490F8220749484606F04B
:10DD9000E1FF4FF48075284604F064FD0646DFF885
:10DDA000088098F801308FE06E0B00200088010891
:10DDB0002A4745542A2046747049503A5B25735DC2
:10DDC000210000002A5345542A2046747049503AD5
:10DDD0005B25735D210000002A4745542A204674C4
:10DDE0007050617373776F72643A5B25735D2100C5
:10DDF0002A5345542A2046747050617373776F72AA
:10DE0000643A5B25735D21002A4745542A204674F5
:10DE100070557365726E616D653A5B25735D2100A7
:10DE20002A5345542A20467470557365726E616D8D
:10DE3000653A5B25735D21002A4745542A204674C4
:10DE400070466F6C6465723A5B25735D210000005B
:10DE50002A5345542A20467470466F6C6465723AA2
:10DE60005B25735D21000000440700202A474554CC
:10DE70002A2052756E4170704E756D3A5B4150505C
:10DE800025635D20212020202A4745542A20417007
:10DE90007056657273696F6E3A5B25735D20210061
:10DEA000303031002A5345542A2052756E4170702B
:10DEB0004E756D3A5B41505025635DD6D8C6F4BAB5
:10DEC000F3C9FAD0A721000092A2294630460CF0EF
:10DED000A1FC054694F82300312805D1AFF240019A
:10DEE000A01C04F067FF20B194F8230030281DD057
:10DEF00022E094F82600302803D0312801D05024A5
:10DF00001BE088F80100F8228849484606F0C5FF62
:10DF100098F80130C5F58071701985A20CF07AFC73
:10DF2000532431463846FFF761FB06E0AFF290011B
:10DF3000A01C04F03FFF28B14924304604F0CCFC7B
:10DF4000204635E4532431463846FFF74FFBF4E7CB
:10DF5000F0B58DB00446F82274497A4806F0FAFE0E
:10DF600079A104F1260004F025FF18B149240DB071
:10DF70002046F0BD4FF40076304604F073FC0746AF
:10DF80007348054606F006F96848F030A0F1200213
:10DF9000A0F1E003CDE90932A0F11001CDE90B10A9
:10DFA0006C4A6038A2F10903CDE905329039CDE918
:10DFB0000710111FA0F18C029038C378CDE902251B
:10DFC00001930491817800914378634A3146384641
:10DFD0000CF020FC39462046FFF708FB5324384656
:10DFE00004F07AFCC3E738B504465CA104F12600CE
:10DFF00004F0E0FE10B15025284638BD532559A144
:10E000002046FFF7F3FAC8200BF0ACF95E4C002372
:10E0100041F28832194620680AF0A7FB012803D193
:10E0200000F052FE03F034FB00231A461946206824
:10E030000AF07CFA192155480CF0D7FF4FF487708D
:10E04000AFF27C73009052A2192150480CF0E2FB11
:10E050004E4804F045FC52A003F0A1F809F020FB63
:10E06000CAE710B5044694F824003038112835D298
:10E07000DFE800F0090D1115191D2125292D343473
:10E080003434343431002046FFF7ADFF27E020461A
:10E09000FFF75EFF23E02046FFF770FE1FE02046FB
:10E0A000FFF70AFE1BE02046FFF7A0FD17E0204621
:10E0B000FFF736FD13E02046FFF7CCFC0FE02046CB
:10E0C000FFF762FC0BE02046FFF77AFB07E02046F3
:10E0D000FFF70FFB03E0FFF70AFB00E04E20344997
:10E0E000502809D049280DD04E2811D14968204622
:10E0F000BDE81040FFF77ABA89682046BDE81040B5
:10E10000FFF774BAC9682046BDE81040FFF76EBA41
:10E1100010BD00002A4745542A20496170466C61B1
:10E12000673A5B25635D2120000000006E0B002034
:10E130002A5345542A20496170466C61673A5B2531
:10E14000635D2100008801084745545F4941500044
:10E1500044070020B21C0020D0F90408434D445F5E
:10E16000525354002A5345542A2055736572206334
:10E170006F6E74726F6C206465766963652072657A
:10E18000737461727421000044000020FA060020BC
:10E19000257320256420CACDB7C545433230210000
:10E1A000D6D8C6F4C3FCC1EEC8EDD6D8C6F421005B
:10E1B0004800002049490620487070474749072019
:10E1C0004870704745490520487070474349092009
:10E1D0004870704741490320487070473F490C2000
:10E1E000487070473D490B204870704710B502F0E9
:10E1F0006BFAAFF20F010C2005F0DDFEAFF2230148
:10E200000B2005F0D8FEAFF23301092005F0D3FE54
:10E21000AFF247010D2005F0CEFEAFF25701072007
:10E2200005F0C9FEAFF26B010F2005F0C4FEAFF29E
:10E230007B01BDE81040062005F0BDBE27484278AE
:10E24000011D0D2A48D2DFE802F04747471747274C
:10E25000372F471F47070F00027802EB420201EBFE
:10E260008202527802702EE0027802EB420201EB49
:10E2700082029278027026E0027802EB420201EB01
:10E280008202D27802701EE0027802EB420201EBB9
:10E2900082021279027016E0027802EB420201EB70
:10E2A0008202527902700EE0027802EB420201EB28
:10E2B00082029279027006E0027802EB420201EBE0
:10E2C0008202D279027000224270007800EB400096
:10E2D00001EB800080680047704700005C00002070
:10E2E00008B5FEA00023009003220C21184602F07E
:10E2F00094FC08BD38B51E2004F0B4FA044605228B
:10E30000FC4920460CF0BAFE0122002310211046E1
:10E31000009402F082FC1E2120460CF066FEF549B6
:10E320000A220B3920460CF0A9FE002302220C2100
:10E330000120009402F071FC2046BDE8384004F052
:10E34000CBBA10B5FFF7D6FFBDE81040C8E708B557
:10E35000E9A0012300901A461021002002F05DFC84
:10E36000E8A00023009002221021184602F055FC7C
:10E37000E7A00023009003221021184602F04DFC74
:10E3800008BD08B5DCA0002300900122102118462A
:10E3900002F043FCDBA000900123022210210020A8
:10E3A00002F03BFCDAA00023009003221021184663
:10E3B00002F033FC08BD08B5CFA000230090012275
:10E3C0001021184602F029FCCEA000230090022262
:10E3D0001021184602F021FCCDA000900123032259
:10E3E0001021002002F019FC08BD08B5C5A00023CB
:10E3F000009001221021184602F00FFCC4A0002357
:10E40000009002221021184602F007FCC3A00090E1
:10E41000012303221021002002F0FFFB08BD08B5F4
:10E42000C1A0012300901A461021002002F0F5FB44
:10E43000C0A00023009002221021184602F0EDFB3C
:10E44000BFA00023009003221021184602F0E5FB34
:10E4500008BD08B5B4A00023009001221021184681
:10E4600002F0DBFBB3A00090012302221021002068
:10E4700002F0D3FBB2A00023009003221021184623
:10E4800002F0CBFB08BD08B5A7A000230090012235
:10E490001021184602F0C1FBA6A000230090022222
:10E4A0001021184602F0B9FBA5A000900123032219
:10E4B0001021002002F0B1FB08BD08B59DA000238B
:10E4C000009001221021184602F0A7FB9CA0002317
:10E4D000009002221021184602F09FFB9BA00090A2
:10E4E000012303221021002002F097FB08BD08B58C
:10E4F00099A0012300901A461021002002F08DFB04
:10E5000098A00023009002221021184602F085FBFB
:10E5100097A00023009003221021184602F07DFBF3
:10E5200008BD08B58CA000230090012210211846D8
:10E5300002F073FB8BA00090012302221021002027
:10E5400002F06BFB8AA000230090032210211846E2
:10E5500002F063FB08BD08B586A0012300901A46AF
:10E560001021002002F059FB85A000230090022218
:10E570001021184602F051FB7DA0002300900322D9
:10E580001021184602F049FB08BD08B579A0002308
:10E59000009001221021184602F03FFB78A0009065
:10E5A000012302221021002002F037FB70A000237B
:10E5B000009003221021184602F02FFB08BD08B579
:10E5C00072A0012300901A461021002002F025FBC2
:10E5D00071A00023009002221021184602F01DFBBA
:10E5E00071A00023009003221021184602F015FBB1
:10E5F00008BD08B565A0002300900122102118462F
:10E6000002F00BFB64A000900123022210210020E5
:10E6100002F003FB64A0002300900322102118469F
:10E6200002F0FBFA08BD08B558A0002300900122B3
:10E630001021184602F0F1FA57A0002300900222A0
:10E640001021184602F0E9FA57A000900123032296
:10E650001021002002F0E1FA08BD08B556A0012300
:10E6600000901A461021002002F0D7FA55480023E6
:10E67000009002221021184602F0CFFA514840388B
:10E680000CF0BEFB102809D94E480023303800900A
:10E6900003221021184602F0C0FA08BD34A000235E
:10E6A000009003221021184602F0B7FA08BD08B501
:10E6B00045A0012300901A461021002002F0ADFA77
:10E6C000404800234030009002221021184602F0FA
:10E6D000A4FA3C4840380CF093FB7BE04D454E5586
:10E6E00020202020202020202020202020424143C4
:10E6F0004B0000000F5C002046545020D0C5CFA234
:10E700000000000054435020D0C5CFA200000000FC
:10E71000C9E8B1B8C9FDBCB600000000C9E8B1B88D
:10E72000D0C5CFA200000000B2E9D1AF465450D509
:10E73000CBBAC500B2E9D1AF465450C3DCC2EB003E
:10E74000B2E9D1AF4654502020495000B2E9D1AFD0
:10E75000465450C2B7BEB600B2E9D1AF54435020C0
:10E7600020495000B2E9D1AF544350B6CBBFDA00D4
:10E7700020000000B2E9D1AFB5B1C7B041505000A0
:10E78000C1A2BCB4C9FDBCB641505000B2E9D1AF82
:10E790004D41434944000000B2E9D1AF41505020FF
:10E7A000B0E6B1BE00000000B2E9D1AF424F4F5415
:10E7B000B0E6B1BE00000000465450D5CBBAC53A11
:10E7C00000000000BE0B0020465450C3DCC2EB3AF0
:10E7D00000000000102808D9F74800230090032209
:10E7E0001021184602F019FA08BDAFF27C00002390
:10E7F000009003221021184602F00FFA08BD08B558
:10E80000EEA0012300901A461021002002F005FA24
:10E81000E9480023B030009002221021184602F08F
:10E82000FCF9E54810380CF0EBFA102808D9E2485A
:10E830000023009003221021184602F0EEF908BDD3
:10E84000AFF2D4000023009003221021184602F0FA
:10E85000E4F908BD38B5DBA0012300901A46102169
:10E86000002002F0DAF9D44C0023103C02221021DF
:10E870001846009402F0D1F920460CF0C1FA102895
:10E8800008D9CD480023009003221021184602F039
:10E89000C4F938BDAFF228100023009003221021E4
:10E8A000184602F0BAF938BD08B5C9A00123009096
:10E8B0001A461021002002F0B0F9BF480023C030F2
:10E8C000009002221021184602F0A7F9BA48103829
:10E8D0000CF096FA102808D9B748002300900322BC
:10E8E0001021184602F099F908BDAFF27C10002300
:10E8F000009003221021184602F08FF908BD08B5D8
:10E90000B5A0012300901A461021002002F085F9DD
:10E91000A9480023D030009002221021184602F0AE
:10E920007CF9A54810380CF06BFA102808D9A248D9
:10E930000023009003221021184602F06EF908BD52
:10E94000AFF2D4100023009003221021184602F0E9
:10E9500064F908BD38B5A3A0012300901A46102120
:10E96000002002F05AF9102003F07CFF0446924880
:10E97000A0A220381021837820460BF04BFF002303
:10E98000022210211846009402F047F9AFF220202D
:10E990000023009003221021184602F03EF9204681
:10E9A000BDE8384003F098BF10B5834931202039C5
:10E9B0004870F822944806F070FA94A003F090FF93
:10E9C000022006F04BF8BDE8104008F069BE38B5EB
:10E9D00093A0012300901A461021002002F01DF997
:10E9E000192003F03FFF04460121204605F0DBFB20
:10E9F000002302220C211846009402F00EF904F1C3
:10EA000015000023009003220C21184602F005F99E
:10EA10002046BDE8384003F05FBF38B582A001232F
:10EA200000901A461021002002F0F7F80C2003F0A5
:10EA300019FF0446204605F0ADFB002302221021F9
:10EA40001846009402F0E9F8AFF2DC2000230090B1
:10EA500003221021184602F0E0F82046BDE83840B5
:10EA600003F03ABF08B573A0012300901A461021A5
:10EA7000002002F0D2F8504800231C3800900222F7
:10EA80001021184602F0C9F8AFF21C3000230090A4
:10EA900003221021184602F0C0F808BD08B5002373
:10EAA00000901A461021184602F0B7F808BD38B594
:10EAB000634C2078C1074FF010000AD0009061A38A
:10EAC00000220221382002F07DF82068401C2060DE
:10EAD00038BDAFF26433009000220221382002F0EA
:10EAE00071F8F2E71CB5044610210022009156A3EC
:10EAF0001146104602F066F856490022CDE9002181
:10EB0000002110232022084602F053FA0C21002293
:10EB10000091234611461A2002F054F81CBD1CB582
:10EB2000044610210022009147A31146402002F024
:10EB300049F8484900224031CDE900211023202224
:10EB40000021402002F035FA0C21002200912346DA
:10EB500011465A2002F036F81CBD10B5102003F003
:10EB600081FE04463C4B3DA2102120460BF052FE94
:10EB70002046FFF7D4FF102120460CF036FA364B22
:10EB800038A25B1D102120460BF044FE2046FFF703
:10EB9000A9FF2046BDE8104003F09EBE08B5002343
:10EBA000009001221021184602F037F8BDE8084015
:10EBB000022002F027B800008E0B0020465450209F
:10EBC00049503A00465450C2B7BEB63A0000000061
:10EBD0005443502049503A00544350B6CBBFDA3A20
:10EBE00000000000B5B1C7B0D4CBD0D0415050BA6E
:10EBF000C53A000052756E4170704E756D3A5B25D6
:10EC0000635DA1A30000000000880108C9FDBCB637
:10EC1000C9E8B1B8A3ACBCB4BDABD6D8C6F400004B
:10EC20004D414349443A000041505020B0E6B1BE46
:10EC3000BAC53A00424F4F54B0E6B1BEBAC53A0029
:10EC4000A40100203A0000002020202020202020C5
:10EC50000000000022E40408A91C002025736D5662
:10EC600000000000435351257300000008B5002345
:10EC7000009002221021012001F0CFFF08BD38B51D
:10EC80000C460023009001221021184601F0C5FF18
:10EC90000023022210211846009401F0BEFF38BD67
:10ECA00070B504460D461021601C0CF09EF92946F3
:10ECB000601CBDE870400CF074B810B504460846FE
:10ECC0000CF01AF8608210BD10B5002003F0C0F9F6
:10ECD000BDE81040012002F05ABE10B503F0E2F882
:10ECE00003280FD1454803F0B7F904464349032CE4
:10ECF00009D04A8A491C42A003F04CFEC8200AF001
:10ED000031FB204610BD4A8A491C44A003F0E8FDAF
:10ED1000204610BD0FB4F8B50646032540F2492041
:10ED200003F0A0FD044608AB00934FF4007739468A
:10ED300004F12600079A0BF031FD002801DDB842EE
:10ED40000BDD83223CA141A003F024FE204603F00A
:10ED5000C3FD0220F8BC5DF814FB28222270667007
:10ED6000642290FBF2F13031A17090FBF2F102FBD2
:10ED700011010A2291FBF2F13031E17090FBF2F1C6
:10ED800002FB1100303020711C49891E0878607127
:10ED9000401CC0B20870392801D930200870042204
:10EDA00031A1A01D0CF06AF9012104F10A0005F05F
:10EDB000FAF93B2184F822103022022104F12300C9
:10EDC0000CF00BF9262184F82510032228A12046F7
:10EDD0000BF0A9FF20460CF013F882B2214625481B
:10EDE00003F05BFE20B1A22213A123A003F0D2FD09
:10EDF000204603F071FD2846ACE70000AA01002080
:10EE000054435020536572766572C1ACBDD3CAA716
:10EE1000B0DC3A25733A256420A3A1005443502066
:10EE2000536572766572C1ACBDD3B3C9B9A63A2534
:10EE3000733A256420A3A100555345525F544350B3
:10EE40005C757365725F7463702E630025732C2587
:10EE5000643A757044617461427566207370696CC0
:10EE60006C6F766572A3A1004D41433A000000002B
:10EE700024582900660C002025732C25643A73540D
:10EE80006370305175657565207370696C6C6F7651
:10EE90006572A3A100000000F0B585B001213748DC
:10EEA00005F081F901F0E0FA0746344801F0C6FAAE
:10EEB000024633A1384601F0ADF9384601F04AF96F
:10EEC000044621462FA003F039FD2146324803F0C5
:10EED00037FB0446032C0DD030480821006809F0A8
:10EEE00035F92FA002F05BF9384600F0D7F805B0ED
:10EEF0002046F0BD03F071FB0446032CF4D17B21C6
:10EF00002B480BF072FF00F0E2FD064630000FD0F8
:10EF100028A101F04AF9054615B1E86804280FD088
:10EF2000022427A003F036FD304600F0B7F8DBE7F7
:10EF300000F068F8014627A003F0D2FC0224F3E7B2
:10EF40001322284829690CF099F8264805F0DEFBC1
:10EF50001322244968460BF0C9FF9DF80900401CA4
:10EF60008DF8090020A00088ADF80B00684605F078
:10EF70006DFC1EA0296903F0E1FCD5E72B070020FA
:10EF80006D616300D3B2BCFED7A2B2E14A534F4ECB
:10EF9000A3BA257300000000C00100203C0000203F
:10EFA0004874747020706F7374206572722E000044
:10EFB0000C1E002073797354696D653200000000E7
:10EFC0004E6F20226A736F6E5F74696D6522202E0A
:10EFD00000000000636A736F6E206572723A2573D9
:10EFE00000000000045C0020303100002573CEAA30
:10EFF000BBF1C8A1B5BDB5C4B7FECEF1C6F7CAB165
:10F00000BCE42E00FE480068704770B504460D460B
:10F01000002C01D02DB10AE00DB1012070BD0020FF
:10F0200070BD012070BD207898B1641C6D1C2078E3
:10F030000BF0A7FB064628780BF0A3FB8642F2D024
:10F0400020780BF09EFB044628780BF09AFB201AE0
:10F0500070BD002070BD70B5064630460BF0D0FE86
:10F06000451C284603F0FEFB041E06D02A46314606
:10F0700020460BF03BFF204670BD204603F02CFCE1
:10F08000002070BD10B5282003F0ECFB04461CB135
:10F09000282120460BF0CBFF204610BD70B504465A
:10F0A00019E02568A089C00503D4A06808B1FFF75E
:10F0B000F5FFA089C00503D4206908B103F00CFC5A
:10F0C000A089800503D4206A08B103F005FC20461E
:10F0D00003F002FC2C46002CE3D170BD2DE9F34F68
:10F0E00085B08A4600242546C6490020CDE90201A4
:10F0F000002637468346012001909AF800002D280B
:10F1000005D1C1490020CDE902010AF1010A9AF8AE
:10F110000000302801D10AF1010A9AF800003138C4
:10F12000082817D89AF8000030380EF002FD804603
:10F1300089460022B54B204629460EF061FD424625
:10F140004B460EF049FA04460D461AF8010F3038C6
:10F150000928E7D99AF800002E2827D19AF801004B
:10F16000302823D3392821D80AF1010A9AF800005F
:10F1700030380EF0DEFC804689460022A34B204644
:10F1800029460EF03DFD42464B460EF025FA044658
:10F190000D4600229B4B304639460EF057FF06467F
:10F1A0000F461AF8010F30380928DFD99AF8000005
:10F1B000652801D045281DD11AF8010F2B2802D04F
:10F1C0002D2803D010E00AF1010A0DE04FF0FF30C6
:10F1D00001900AF1010A07E00BEB8B0100EB410BF8
:10F1E0000AF1010AABF1300B9AF80000A0F13001EE
:10F1F0000929F1D901980BFB00F00EF09AFC324678
:10F200003B460EF0E9F902460B4600207F490DF01F
:10F21000A5FC06460F46DDE9020122462B460EF00C
:10F22000EFFC32463B460EF0EBFC04460D460598DB
:10F23000C0E90645204629460EF01EFC05994861A6
:10F2400005980321C16007B05046BDE8F08F401E0D
:10F2500040EA600040EAA00040EA201040EA202096
:10F2600040EA2040401C704770B50446002C08D08E
:10F27000236833B1A26850186168814203DB981893
:10F2800070BD002070BDFFF7E2FF0646304603F078
:10F29000E9FA054665B1D4E9001228460BF026FECE
:10F2A000206803F019FB66602560A068284470BDE3
:10F2B000206803F011FB00206060206070BD10B575
:10F2C0000446002C08D0206830B1A16808440BF037
:10F2D00097FDA168084410BD002010BD2DE9F0473E
:10F2E00007460E46DFF82881D7E906450022134677
:10F2F000204629460EF084FB12D12EB10221304661
:10F30000FFF7B2FF814603E0022003F0ABFA81462B
:10F31000B9F1000F03D03FA00088A9F800009CE0DD
:10F3200078690EF006FC22462B460EF08FFE21F087
:10F330000041002243460EF027FC21D8364A374BC5
:10F34000204629460EF020FC1AD80022344B2046D5
:10F3500029460EF053FD13D82EB115213046FFF784
:10F3600083FF814603E0152003F07CFA8146B9F162
:10F37000000F72D02BA148467A690BF035FA6CE089
:10F380002EB140213046FFF76FFF814603E0402059
:10F3900003F068FA8146B9F1000F5ED02046294695
:10F3A0000DF0C0F922462B460EF050FE21F0004130
:10F3B000002243460EF0E8FB0ED825F0004120461F
:10F3C000194A1A4B0EF0E0FB06D222462B4618A132
:10F3D00048460BF009FA40E0204625F00041064679
:10F3E0000F46154A154B0EF0CFFB06D33046394673
:10F3F0000022134B0EF002FD29D222462B4621E0BB
:10F40000D00100200000F03F0000F0BF00002440C9
:10F410000000B03C300000000000C0FFFFFFDF41F3
:10F420000000E0C12564000044F3C2E4E4E9634C59
:10F43000252E3066000000008DEDB5A0F7C6B03E69
:10F4400065CDCD41F6A148460BF0CEF905E0224648
:10F450002B46F4A148460BF0C7F94846BDE8F087B3
:10F460000178A1F13002092A01D811460AE0A1F180
:10F470004102052A01D8373904E0A1F16102052AC9
:10F480000AD857390A01401C0178A1F13003092B31
:10F4900004D8303A11440EE000207047A1F1410336
:10F4A000052B02D8373A114405E0A1F16103052B81
:10F4B0000BD8573A11440A01401C0178A1F13003DE
:10F4C000092B04D8303A11440EE000207047A1F116
:10F4D0004103052B02D8373A114405E0A1F161033D
:10F4E000052B0AD8573A114409014078A0F130029F
:10F4F000092A04D830390844704700207047A0F129
:10F500004102052A02D8373908447047A0F1610248
:10F51000052A02D8573908447047002070472DE962
:10F52000F04780460D466C1C00202978222907D020
:10F53000BD480560002091E7641C5C2A00D1641C72
:10F540002278222A02D00AB1401CF5D1401C03F0D7
:10F5500089F90746380004D0681C3C464FF480699E
:10F560001AE000207AE75C2903D004F8011B401C54
:10F5700012E0461C3078722825D006DC622816D0AE
:10F58000662818D06E2804D119E074281FD0752879
:10F5900021D004F8010B701C0178222901D0002928
:10F5A000E1D100212170017822296AD06AE0082087
:10F5B00004F8010BEFE70C2004F8010BEBE70A203D
:10F5C00004F8010BE7E70D2004F8010BE3E709203D
:10F5D00004F8010BDFE7701CFFF742FF0546361DFC
:10F5E000A5F55C404845D6D3002DD4D0A5F55840AC
:10F5F000484513D270785C28CDD1B0787528CAD12F
:10F60000F01CFFF72DFFB61DA0F55C414945C2D2A5
:10F61000C5F3090161F39F2000F580350421802D99
:10F6200001D2012108E0B5F5006F01D2022103E00B
:10F63000B5F5803F00D20321601801291AD00229B4
:10F6400011D0032908D0042919D105F0BF0242F0D6
:10F65000800200F8012DAD0905F0BF0242F08002E2
:10F6600000F8012DAD0905F0BF0242F0800200F85C
:10F67000012DAD096D4A525C2A4300F8012D441852
:10F6800089E7401CC8F810700421C8F80C10E5E6A2
:10F690002DE9F04705468A4600240021A9460AE0E4
:10F6A000421E1F2A11D322280FD05C280DD0002023
:10F6B000014309F1010999F800000028F0D18046C2
:10F6C000222721B125B32E4644E00120F0E7A9EB23
:10F6D0000506BAF1000F05D0F11C5046FFF7C4FD36
:10F6E000044603E0F01C03F0BDF8044674B1277033
:10F6F00004F10109294648460BF053FB09F806704E
:10F7000009EB060080F801802046A7E60020A5E668
:10F71000BAF1000F05D003215046FFF7A5FD0446BE
:10F7200003E0032003F09EF804462CB140A12046DC
:10F730000BF037FB204691E600208FE649463DA0BE
:10F740000BF0E7FA08B1641C03E0B9F1200F00D216
:10F75000641D761C96F80090B9F1000F01D0641C6E
:10F76000ECD1BAF1000F05D0E11C5046FFF77CFD4B
:10F77000064603E0E01C03F075F806462EB130465D
:10F7800000F8017B4FF05C0925E0002066E61F29A8
:10F7900007D9222905D05C2903D000F8011B6D1C74
:10F7A00019E000F8019B044615F8012B0C2A25D01E
:10F7B00006DC082A1ED0092A2CD00A2A06D121E00C
:10F7C0000D2A23D0222A12D05C2A0CD01BA120465D
:10F7D0000BF00AF8601D29780029D8D1077080F84D
:10F7E000018030463AE684F80090601CF3E7277009
:10F7F000601CF0E762202070601CECE7662020703F
:10F80000601CE8E76E202070601CE4E77220207026
:10F81000601CE0E774202070601CDCE7006937E7BB
:10F820002565000025660000D0010020A2E4040840
:10F8300022220000225C080C0A0D090075253034D4
:10F840007800000000E0401C002804D00178002966
:10F8500001D02029F7D970472DE9F04107460878F3
:10F86000FE4E7B2803D031600020BDE8F0810620E9
:10F87000F860481CFFF7E6FF054628787D2818D079
:10F88000FFF700FC0446B860A8B12846FFF7DAFF8E
:10F8900001462046FFF743FEFFF7D4FF68B1216918
:10F8A00021620027276101783A2908D030600020C2
:10F8B000DBE7681CD9E70020D7E70020D5E7401C2C
:10F8C000FFF7C0FF0146204600F086F8FFF7BAFFB9
:10F8D0000546280028D1C8E7FFF7D4FBA8B120606F
:10F8E00044600446681CFFF7ADFF01462046FFF761
:10F8F00016FEFFF7A7FF50B1216921622761017849
:10F900003A2906D030600020AFE70020ADE70020A4
:10F91000ABE7401CFFF796FF0146204600F05CF87D
:10F92000FFF790FF054645B128782C28D4D02878D9
:10F930007D2804D03560002097E7002095E7681CFB
:10F9400093E72DE9F04107460878C44E5B2802D0C2
:10F950003160002089E70520F860481CFFF772FF3E
:10F96000044620785D2811D0FFF78CFB0546B8606F
:10F9700070B12046FFF766FF0146284600F02CF8DC
:10F98000FFF760FF0446200004D016E0601C6CE71F
:10F9900000206AE7002068E7FFF774FBB0B1286039
:10F9A00045600546601CFFF74DFF0146284600F004
:10F9B00013F8FFF747FF044654B120782C28EBD00A
:10F9C00020785D2806D0346000204EE700204CE708
:10F9D00000204AE7601C48E770B505460C46002C3D
:10F9E00020D004229EA120460BF029FAE0B1052286
:10F9F0009DA120460BF023FAD0B104229CA1204601
:10FA00000BF01DFAC0B1207822281AD02D2803D07F
:10FA1000A0F13001092919D821462846BDE87040D7
:10FA2000FFF75CBB002070BD0220E860201D70BDA8
:10FA30000020E860601D70BD0120E8606861201D45
:10FA400070BD21462846BDE8704068E55B2805D0BA
:10FA50007B2808D081480460002070BD21462846DC
:10FA6000BDE870406DE721462846BDE87040F3E6EA
:10FA70002DE9F04104460D469046FFF703FB06468C
:10FA8000764F00203860BEB12046FFF7DBFE01460E
:10FA90003046FFF7A1FF044684B1B8F1000F12D041
:10FAA0002046FFF7CFFE0446207860B13046FFF7CE
:10FAB000F5FA3C600020D8E60020D6E63046FFF795
:10FAC000EDFA0020D1E605B12C603046CDE60022EB
:10FAD0001146CDE72DE9F04F85B00646894615461B
:10FAE0001C4600200490072002904FF0000BB068E5
:10FAF00000270021019101E07F1C00680028FBD154
:10FB000037B1002C70D0A76895B34FF0020A32E0ED
:10FB10004CB115B109F1040100E003212046FFF7C3
:10FB2000A3FB024607E015B109F1040000E0032041
:10FB300002F098FE024662B110467B2100F8011BDC
:10FB400085B10A2100F8011B00210923A9F101094F
:10FB500006E0002005B0BDE8F08F00F8013B491C2D
:10FB60004945FADB7D210170002141701046F1E723
:10FB7000FFE74FF0010A0AF101012046FFF774FB8D
:10FB800088B17B2100F8011B15B10A2100F8011B87
:10FB90004FF0000880F80080A0685044A060B6686C
:10FBA00009F101096CE00020D4E78DB149462046F7
:10FBB000FFF75AFB10B10021092204E00020C9E739
:10FBC00000F8012B491C4945FADBA0684844A060B5
:10FBD0002146306AFFF75CFD2046FFF770FBA0600E
:10FBE0001DB14FF0020A02E06CE04FF0010A5146ED
:10FBF0002046FFF739FBA8B13A2100F8011B0DB1EF
:10FC000009210170A0685044A06023462A46494655
:10FC1000304600F026FA2046FFF751FBA0601DB1E8
:10FC2000012002E0002095E70020316809B10121A0
:10FC300000E0002100EB010A0AF101012046FFF774
:10FC400013FB18B3316811B12C2100F8011B15B159
:10FC50000A2100F8011B80F800800DE0D00100208F
:10FC60006E756C6C0000000066616C7365000000CE
:10FC70007472756500000000A0685044A06036688A
:10FC8000002E92D125B109F1010102E0002061E7C7
:10FC900002212046FFF7E8FA28B15DB100270921CB
:10FCA000A9F1010904E0002054E700F8011B7F1CC2
:10FCB0004F45FADB7D21017080F8018020683844CF
:10FCC0000490D7E0BC00204602F0CCFD80465FEAFD
:10FCD000080016D0204602F0C5FD82465FEA0A0001
:10FCE00011D0214640460BF0A2F9214650460BF0B8
:10FCF0009EF9B46809F101098DB302984844029055
:10FD000031E0002026E7404602F0E6FD002021E732
:10FD10000021206AFFF7BCFC03904AF82B00002367
:10FD20002A464946204600F09CF959460BF1010B42
:10FD300048F82100039999B190B10BF061F806469B
:10FD400003980BF05DF8311815B109F1020000E0DD
:10FD50000020014402980844801C029002E002E066
:10FD6000012001902468002CD2D1019818B9029882
:10FD700002F078FD0490049808B9012001900198E0
:10FD8000B0B100240AE05AF8240008B102F0A4FD42
:10FD900058F8240008B102F09FFD641CBC42F2DB5D
:10FDA000504602F099FD404602F096FD0020D1E653
:10FDB00004997B200870049C641C15B10A2004F887
:10FDC000010B4FF0000B84F800B000263BE03DB182
:10FDD0000020092102E004F8011B401C4845FADB21
:10FDE0005AF826000BF00CF800905AF8261020461E
:10FDF000009A0BF07BF8009804443A2004F8010BB9
:10FE000015B1092004F8010B58F8261020460AF015
:10FE1000C8FF58F826000AF0F3FF0444781E864213
:10FE200002D02C2004F8010B15B10A2004F8010BB4
:10FE300084F800B05AF8260002F04EFD58F826006B
:10FE400002F04AFD761CBE42C1DB504602F044FD82
:10FE5000404602F041FD4DB100200921A9F1010900
:10FE600002E004F8011B401C4845FADB7D202070AD
:10FE700084F801B004986DE62DE9FF4F81B0834608
:10FE800090461F464FF000094FF0050ADBF80800C6
:10FE900000260025002401E0761C00680028FBD124
:10FEA0007EB1002F5FD0BE6801213846FFF7DCF934
:10FEB000C8B15B210170B868401CB860DBF808501D
:10FEC0003DE02FB103213846FFF7CEF9044603E0A9
:10FED000032002F0C7FC04461CB1FCA120460AF036
:10FEE00060FF204636E6002034E602993B46424653
:10FEF000491C284600F0B5F83846FFF7E0F9B8602D
:10FF00002868D8B1B8F1000F02D04FF0020901E023
:10FF10004FF0010909F101013846FFF7A5F9F0B1E9
:10FF20002C2100F8011BB8F1000F02D0202100F8AD
:10FF3000011B00210170B8684844B8602D680DB1FC
:10FF4000002CD2D002213846FFF78EF948B15D214E
:10FF5000017000214170386800EB06097FE0002045
:10FF6000F8E50020F6E5B000009002F07BFC0746C3
:10FF7000380005D000990BF05AF8DBF808B01EE005
:10FF80000020E7E5029900234246491C584600F04C
:10FF900068F829466D1C47F8210068B10AF030FF67
:10FFA0000146B8F1000F01D0012000E00020084414
:10FFB00082440AF1020A00E00124DBF800B0BBF140
:10FFC000000F01D0002CDDD01CB9504602F04AFCD5
:10FFD0008146B9F1000F00D1012474B1002405E07D
:10FFE00057F8240008B102F077FC641CB442F7DB38
:10FFF000384602F071FC0020ACE55B2089F8000077
:020000040804EE
:100000004C464FF0000A04F801AF00251EE057F8F7
:1000100025000AF0F5FE834657F825105A4620467B
:100020000AF064FF5C44701E85420AD02C2004F85C
:10003000010BB8F1000F02D0202004F8010B84F866
:1000400000A057F8250002F047FC6D1CB542DEDB2E
:10005000384602F041FC5D20207084F801A048463B
:1000600078E570B50024002809D083B3057B072DFF
:100070006ED2DFE805F01320062D32373B0000205A
:1000800070BD05211846FFF7EFF80446002C5FD03D
:10009000AFF2344120460AF084FE59E006211846AA
:1000A000FFF7E2F80446002C52D0AFF2444120465C
:1000B0000AF077FE4CE005211846FFF7D5F8044614
:1000C00034B3AFF2544120460AF06BFE40E011E039
:1000D0001946FFF703F904463AE01946FFF79EFB7D
:1000E000044635E0FFF7C8FE044631E0FFF7F2FCB6
:1000F00004462DE0037B072B2AD2DFE803F00A1029
:1001000004161B202500AFF2A840FEF7A4FF04460A
:100110001EE0AFF2AC40FEF79EFF044618E0AFF2DF
:10012000B040FEF798FF044612E00021FFF7D6F832
:1001300004460DE00021FFF771FB044608E00023B0
:10014000FFF79AFE044603E00023FFF7C3FC0446D2
:10015000204670BD00230122194682E700231A467B
:1001600019467EE7FEB505460C461646204602F0C7
:1001700079FB00900194002002906B4632460021EA
:100180002846FFF76EFFFEBD8168002001E0401C9D
:1001900009680029FBD17047806801E0491E0068AA
:1001A000002801D00029F9DC704770B50D4684683D
:1001B00000E024682CB12946206AFEF726FF0028BB
:1001C000F7D1204670BD01604860704770B50546A4
:1001D000FEF758FF044674B12822294620460AF04B
:1001E000CAFE00202062E16841F48071E160606035
:1001F0002060204670BD002070BD02469068002936
:1002000001D010B991607047104610B10268002A01
:10021000FAD1D8E770B505460E461446002C0CD02E
:10022000206A08B102F058FB3046FEF714FF206246
:1002300021462846BDE87040DFE770BD70B5064630
:100240000D461446002C10D0A089800503D4206AE6
:1002500008B102F041FB2562E06840F40070E06004
:1002600021463046BDE87040C7E770BD10B5044672
:100270000846FFF7ABFF01462046BDE81040BCE74B
:1002800070B504460D461046FFF7A0FF024629460A
:100290002046BDE87040BDE70246906801E0006876
:1002A000491E08B10029FADC90B1416809B1036820
:1002B0000B60016809B143684B609168814201D1CC
:1002C0000168916000210160416070475B5D000042
:1002D0000020FAE710B5FFF7DFFFBDE81040FEF79A
:1002E000DDBE2DE9F04106460F460025B46801E069
:1002F0006D1C24682CB13946206AFEF786FE002862
:10030000F6D124B129463046BDE8F041C4E70020CB
:10031000BDE8F08110B5FFF7E4FFBDE81040FEF73F
:10032000BDBE30B40C461146836801E01B68641EF4
:100330000BB1002CFADC4BB10B605A684A60596073
:1003400082689A4204D1816030BC704730BC54E767
:1003500048680160F8E730B40346986801E0006837
:10036000491E08B10029FADC0028EDD001681160AF
:100370004468546001B14A609968814201D19A6031
:1003800001E051680A6000214160016030BCFEF765
:1003900085BED9E72DE9F041064688461746002577
:1003A000B46801E06D1C24682CB14146206AFEF758
:1003B0002CFE0028F6D1002CAAD04046FEF74BFEBA
:1003C00038623A4629463046BDE8F041C3E79FE728
:1003D00010B5FEF757FE002801D00221C16010BD04
:1003E00010B5FEF74FFE002801D00121C16010BDFD
:1003F00010B5FEF747FE002801D00021C16010BDF6
:1004000010B50446FEF73EFE002804D00CB10121D1
:1004100000E00021C16010BD70B504460D46FEF736
:1004200031FE064646B10320F060C6E90645204687
:1004300029460DF021FB7061304670BD70B5054650
:10044000FEF720FE04462CB10420E0602846FEF7AB
:1004500002FE2061204670BD10B5FEF713FE002895
:1004600001D00521C16010BD10B5FEF70BFE0028BC
:1004700001D00621C16010BD2DE9F04780468946B4
:100480000027FFF7E9FF064600240DE058F8240096
:100490000DF04FFBFFF7C0FF05465CB1294638461B
:1004A000FFF791FE2F46641C0EB14C45EEDB304643
:1004B000BDE8F087B560F5E72DE9F047804689464D
:1004C0000027FFF7C9FF064600240DE058F8240076
:1004D0000DF0A6FEFFF7A0FF054654B129463846A9
:1004E000FFF771FE2F46641C0EB14C45EEDB304623
:1004F000DEE7B560F6E72DE9F0478046894600273C
:10050000FFF7AAFF064600240CE008EBC40103C96C
:10051000FFF782FF054654B129463846FFF753FEE0
:100520002F46641C0EB14C45EFDB3046C0E7B5608A
:10053000F6E72DE9F047074688464FF00009FFF738
:100540008BFF064600240BE057F82400FFF776FFE8
:10055000054654B129464846FFF735FEA946641CB6
:100560000EB14445F0DB3046A2E7B560F6E72DE971
:10057000F04106460F460024002E1DD0FEF782FDF6
:10058000054628001AD0F06820F48070E860706991
:100590006861D6E90601C5E90601306918B1FEF7C0
:1005A0005AFD286160B1306A18B1FEF754FD286227
:1005B00058B17FB1B66821E00020A9E60020A7E687
:1005C0002846FEF76BFD0020A2E62846FEF766FDF2
:1005D00000209DE628469BE601213046FFF7C7FF35
:1005E00020B144B120604460044606E02846FEF78E
:1005F00055FD00208CE6A86004463668002EEBD13D
:10060000284685E6014626E0202A08D0092A08D097
:100610000D2A08D00A2A08D02F2A08D00AE0401C48
:1006200019E0401C17E0401C15E0401C13E0437823
:100630002F2B03D02F2A06D008E0401C027852B19D
:100640000A2A08D0F9E743782A2B0BD0222A12D0A5
:1006500001F8012B401C0278002AD5D10020087037
:1006600033E6401C027822B12A2AFAD142782F2A96
:10067000F7D1801CEFE701F8012B401C08E05C2A51
:1006800002D101F8012B401C10F8012B01F8012BBD
:1006900002780AB1222AF2D110F8012B01F8012BBD
:1006A000D9E710220921042003F014BC09210420F9
:1006B00003F076BC10B5FFF7F9FF4FF4C87004F0F3
:1006C000CDF9BDE81040F1E738B506240C234822E7
:1006D00019460020009403F019FC082348220B213E
:1006E0000020009403F012FC082348220921022074
:1006F000009403F00BFC08234822072102200094F9
:1007000003F004FC0823482206210220009403F091
:10071000FDFB082348220F210320009403F0F6FB81
:10072000082348220D210320009403F0EFFB482208
:100730000B21032003F0CEFB48220821002003F008
:10074000C9FB48220921022003F0C4FB48220821EA
:10075000022003F0BFFB48220E21032003F0BAFB66
:10076000BDE8384048220C21032003F0B3BB10221F
:100770000A21042003F0AEBB0A21042003F010BCC0
:1007800010B5FFF7F9FF4FF4C87004F067F9BDE842
:100790001040F1E710B50A460146114802F07DF914
:1007A000002804D0BDE810400EA002F0F3B810BD40
:1007B00010B504460A4802F067F905230C222146C9
:1007C000002002F061FCAFF23301BDE810400020D0
:1007D00002F02EBC0A460146002002F08ABD00004D
:1007E0006C100020735573625175657565D2E7B35F
:1007F000F6A3A10010B50A460146114802F04DF9D2
:10080000002804D0BDE810400EA002F0C3B810BD0F
:1008100010B504460A4802F037F905230C22214698
:10082000042002F031FCAFF23301BDE81040042097
:1008300002F0FEBB0A460146042002F05ABD000049
:10084000721400207352533233325175657565D27C
:10085000E7B3F6A3A100000010B50A460146184808
:1008600002F01BF9002804D0BDE8104015A002F0EA
:1008700091B810BD10B5044610220021032003F0EA
:1008800029FB154B00221A600D4802F0FDF80523E4
:100890000C222146032002F0F7FBAFF24301BDE832
:1008A0001040032002F0C4BB10B50A460A4C0121D7
:1008B00021600146032002F01CFD0020206010BDD5
:1008C000781800207352533438355175657565D2E8
:1008D000E7B3F6A3A10000008081224270B5002496
:1008E00000250126F84B01290CD00022C3F89851AD
:1008F000C3F89051C3F894513AB101060DD5C3F82D
:100900009C510CE0C3F89861F2E7010602D5C3F8E8
:100910009C6104E0C3F89C5101E0C3F89C61C3F8FA
:1009200094614006000E641CE4B2082CE2D3C3F8C4
:100930009061C3F8986170BD10B50446B031C8B27B
:1009400000221146FFF7CAFFA41CC4F303100022C3
:1009500040F010001146FFF7C1FF04F00F00002225
:10096000BDE810401146B9E730B5002505F1B000EB
:100970000022C0B21146FFF7B1FF0022114602204B
:10098000FFF7ACFF002211461020FFF7A7FF00245D
:10099000002201211046FFF7A1FF641CE4B2802C65
:1009A000F6D36D1CEDB2082DE0D330BD70B510222A
:1009B0000421002003F08EFA10220521002003F00C
:1009C00089FA10220621002003F084FA1022072160
:1009D000002003F07FFA10220521022003F07AFAAA
:1009E000BA4C01252560642004F038F8002020600E
:1009F000642004F033F8256000221146AE20FFF792
:100A00006DFF002211460220FFF768FF0022114609
:100A10001020FFF763FF002211464020FFF75EFF22
:100A2000002211468120FFF759FF00221146FF20C6
:100A3000FFF754FF00221146A120FFF74FFF0022CD
:100A40001146C820FFF74AFF00221146A620FFF7F3
:100A500045FF00221146A820FFF740FF0022114663
:100A60003F20FFF73BFF00221146D320FFF736FF60
:100A7000002211461046FFF731FF00221146D52013
:100A8000FFF72CFF002211468020FFF727FF0022EE
:100A90001146D920FFF722FF00221146F120FFF76F
:100AA0001DFF00221146DA20FFF718FF0022114631
:100AB0001220FFF713FF00221146DB20FFF70EFF85
:100AC000002211464020FFF709FF00221146202096
:100AD000FFF704FF002211460220FFF7FFFE00226D
:100AE00011468D20FFF7FAFE002211461420FFF771
:100AF000F5FE00221146A420FFF7F0FE0022114669
:100B0000A620FFF7EBFE00221146AF20FFF7E6FE1E
:100B100000221146AF20FFF7E1FEFFF725FFBDE8F9
:100B200070400021084607E72DE9F041804606980D
:100B30000E461F4600242038C5B2B8F17F0F02D9F7
:100B4000A046B61CF6B20C2A06D0102A19D0BDE871
:100B5000F0415FA001F01EBF761CF1B24046FFF7E6
:100B6000EBFE604905EB450001EB40053A46285D88
:100B70000121FFF7B3FE641CE4B2062CF6D3BDE8F6
:100B8000F08131464046FFF7D7FE574800EB051588
:100B90003A46285D0121FFF7A1FE641CE4B2082C4F
:100BA000F6D3761CF1B24046FFF7C6FE00242819A2
:100BB0003A46007A0121FFF791FE641CE4B2082C4A
:100BC000F5D3DCE72DE9F8430446DDF820800E4636
:100BD00091461F46002510E000904B4642463146A4
:100BE0002046FFF7A1FF04EB5800C4B2782C02D9CD
:100BF0000024761CF6B26D1CEDB2785D0028EBD1B6
:100C0000BDE8F88308B5102140060091010E0022CE
:100C100036A31046FFF7D6FF08BD0FB42DE9FE4FEF
:100C20000C46934600254FEA54088020B0FBF8F6A6
:100C30004FEA4B07102C1BD0042002900DF1440901
:100C4000CDF80490701C01F00DFE82464B46711CDD
:100C50005046109A09F0A2FD8146B1450BD90AEB26
:100C6000060010F8010C7F2805D9A6F1010905E05E
:100C700041200290E2E7B14500D9B1460C98012825
:100C800002D002280AD105E0A6EB0900400808FBC3
:100C900000F503E0A6EB090008FB00F5B9F1000F31
:100CA0007DDD5846FFF7AEFF0026A8E01AF80610D3
:100CB0007F2925D80091F9B2E8B222460F9BFFF7B1
:100CC00033FF05EB540599E00000214294012242D4
:100CD0004E6F202043484152484947485F65202EC7
:100CE00000000000F8ED040820F004082020202077
:100CF0002020202020202020202020200000000074
:100D0000002078E0102C02D00C2C38D072E0C0EB20
:100D1000C00202EB8203DA4A03EB020898F82020B3
:100D2000914267D10AEB060298F8213052789A4234
:100D300060D1F9B2E8B2FFF7FFFD4FF0000B07E01A
:100D400018F80B0001210F9AFFF7C8FD0BF1010BFA
:100D5000A345F5D3781CC1B2E8B2FFF7EDFDA34679
:100D600007E018F80B0001210F9AFFF7B7FD0BF110
:100D7000010BBBEB440FF4D32544761C3EE000EBA3
:100D8000C00202EB4203BE4A6C3A03EB020898F839
:100D9000182091422ED10AEB0602527800E032E090
:100DA00098F819309A4225D1F9B2E8B2FFF7C4FD9C
:100DB0004FF0000B07E018F80B0001210F9AFFF726
:100DC0008DFD0BF1010BA345F5D3781CC1B2E8B240
:100DD000FFF7B2FDA34607E018F80B0001210F9AB8
:100DE000FFF77CFD0BF1010BBBEB440FF4D3254463
:100DF000761C03E0401C029A904283D3761C4E4539
:100E0000FFF454AF09E008D0B1229EA1A3A009F0DD
:100E1000DFFCAFF2341009F0DBFC5046BDE8FE0FFA
:100E20005DF814EB01F058BD00B5002211468D208D
:100E3000FFF754FD002211461420FFF74FFD00225A
:100E40001146AF205DF804EB48E500B500221146DD
:100E50008D20FFF743FD002211461020FFF73EFDD5
:100E600000221146AE205DF804EB37E52DE9FF5F67
:100E700080460E9D8B461F46002459464046FFF78C
:100E80005BFD0BF101090C2D08D0102D4FD0AFF2F6
:100E9000C01004B0BDE8F05F01F07CBDDFF8E0A158
:100EA000AAF16C0A3CE06C221B2300203D1932E0C1
:100EB00000EBC00606EB46065644395D96F818C0AE
:100EC000614527D1697896F819C0614522D1594604
:100ED0004046FFF731FD00250121705D029AFFF7C2
:100EE000FDFC6D1CEDB20C2DF6D309F0FF01404660
:100EF000FFF722FD0C250121705D029AFFF7EEFC41
:100F00006D1CEDB2182DF6D308F10C0808F0FF089F
:100F1000641C04E0401C92FBF3F18142C8D8641CBD
:100F2000384609F06DFFA042BDD8BDE8FF9FDFF84D
:100F300050A138E000203A5D3B19C0EBC00101EB45
:100F4000810101EB0A0696F820108A4227D15978D0
:100F500096F82150A94222D159464046FFF7ECFCB1
:100F600000250121705D029AFFF7B8FC6D1CEDB2FF
:100F7000102DF6D309F0FF014046FFF7DDFC1025E8
:100F80000121705D029AFFF7A9FC6D1CEDB2202DC6
:100F9000F6D308F1100808F0FF08641C02E0401CBA
:100FA0004128CAD3641C384609F02AFFA042C1D8A0
:100FB000BBE72DE9F04F8146DDE909BA0E46002571
:100FC000580705D0012000EBD30702EB090815E014
:100FD000DF08FAE731464846FFF7AEFC4C4609E029
:100FE00028466D1C1AF800005A460121FFF776FCCE
:100FF000641CE4B2A045F3D8761CF6B2BE42E9D335
:10100000BDE8F08F10B586B00121080304F01BFC89
:1010100004220621002002F05DFF18220521002095
:1010200002F058FF18220721002002F053FF10227F
:101030000421002002F04EFF0020ADF804004FF420
:101040008271ADF80610ADF80800ADF80A00ADF8F1
:101050000C004FF40071ADF80E100821ADF810101F
:10106000ADF812000720ADF81400104C01A920467D
:1010700006F00AFC0121204606F08BFC06B010BDEC
:1010800015E504082E2E5C48415244574152455CF8
:101090004F4C45445C6F6C65642E63004C6F674534
:1010A00072723A2025732C25640000000030014044
:1010B00010B57E4C204605F0C7FF2046BDE8104025
:1010C00014227B4903F0E9BE70B505F084FF0024CB
:1010D000784D05EBC42005F0B7FF641CE4B2002C8A
:1010E000F7D0734800214160C160FFF7E1FFBDE820
:1010F000704005F07CBF2DE9F04105460E464FF4E7
:101100000067384601F0AEFB8046C6F3CF240BE003
:101110003A464146284603F01DFE3A464146002025
:1011200002F0E7F805F50065641EA4B2F0D2394676
:10113000404609F05AFFC6F30A04224641462846B3
:1011400003F008FE22464146002002F0D2F8404655
:10115000BDE8F04101F0C0BB70B5142254495348BA
:1011600003F0F8FD524C4FF0503000252268011179
:1011700082420ED122698A420BD121894EA001F010
:10118000AFFB4C486168FFF7B6FF2581BDE87040B2
:101190008EE7206021612581BDE8704094E72DE94C
:1011A000F84F0546284609F02BFE00287BD028463C
:1011B00009F026FE14301FFA80F8404601F052FB79
:1011C000074600260024464B46A241463846009575
:1011D00009F020FB80B200F0010101EB500505F0A1
:1011E000FAFE352006F01BF910E00A2003F036FC69
:1011F0000A2C09D93EA001F0CDFB05F0ECFE3846E3
:10120000BDE8F84F01F068BB641CA4B2012006F0F1
:10121000F7F80128E9D0DFF89890DFF898A031E0DE
:10122000202006F0FCF8701C81B2B85D08B940F0CF
:101230002D004A1C795C96B240EA0124200A01D1B3
:1012400044F43454D9F80400C8F50061884207D347
:101250000020C9F80400B9F80800401CA9F80800EB
:10126000D9F804005044410501D105F0EDFED9F84C
:1012700004002146504405F0B7FFD9F80400801C53
:10128000C9F804006D1EADB2CAD2FFF711FF05F018
:10129000AEFE1CA0D9F8041001F022FB3846BDE8D0
:1012A000F84F01F019BBBDE8F88F000000F0070807
:1012B000801C002000F80708B1BEB5D8C8D5D6BE3E
:1012C000B4E6B4A2D2E7B3F6A3BA2564B4CE202E16
:1012D0000D0AB1BEB5D8C8D5D6BE3A200000000070
:1012E0000F5C00202A25732025732A2000000000AF
:1012F000D0B4466C617368C3A6B5C8B4FDB3ACCABC
:10130000B1A3A100466C617368C6ABD2C6B3A4B6E4
:10131000C83A252378000000072813D2DFE800F040
:101320000406080A0C0E1000E3A07047E4A0704702
:10133000E6A07047E8A07047EAA07047ECA07047AD
:10134000EEA07047F1A070474FF4A071F24809F089
:101350004CBE4FF4A071F14809F047BE70B5054688
:101360000C46EF480078002806D022462946BDE802
:101370007040EA4809F0D7BCEAA1284601F01AFDFE
:10138000002821DBE9A1284601F014FD00280DDB2F
:1013900022462946E94801F080FB002830D0BDE80C
:1013A00070407122E6A1EFA001F0F4BA224629466E
:1013B000F34801F072FB002822D0BDE8704078228B
:1013C000DFA1F0A001F0E6BAD34809F019FDC0F59D
:1013D000A070A04205D92946BDE87040CE4809F06A
:1013E00079BD8422D6A1EEA001F0D4FAFFF7ACFFBC
:1013F0002946BDE870404FF4A072C74809F03EBED0
:1014000070BD0FB42DE9F84F82464FF00408C44870
:10141000CAEBCA01001D00EB8104667E60680B9078
:101420004FF4A165284601F01DFA83460CAB0093EA
:10143000294658460B9A09F0B1F907464FF00009C2
:10144000002F01DDAF423EDDB622BDA1DBA001F0E1
:10145000A1FA584601F040FA0220BDE8F80F5DF805
:1014600014FBFFF771FF0025BAB25946022001F0C4
:1014700040FF16E0642003F0F1FAE168A64801F0AD
:1014800099FC20612069002802DB4FF003081DE071
:101490006169A14801F08EFC002802DB4FF00208D0
:1014A00014E028466D1C2189EDB28842E2D3607EAB
:1014B000801B00EBC00101EB00104FF4FA7101EB4F
:1014C000800003F0CBFA761EF6B2CAD2584601F07D
:1014D00003FACDF80090B8F1050F0ED2DFE808F05E
:1014E000030507090B00BCA408E0BEA406E0C0A4E5
:1014F00004E0C1A402E0C2A400E0C3A45046FFF788
:101500000BFF01462246C3A001F018FA4046A4E7AB
:1015100070B5044600202060207100210620FFF7EE
:1015200070FF0546032D05D0BCA1204609F039FC0B
:10153000284670BD2C21784809F057FC411C042333
:101540000D22204601F059FBF2E770B50546152142
:10155000284609F04AFD00210520FFF752FF044606
:10156000032C09D10D216C4809F0D3FB811C1423F5
:101570000D22284601F041FB204670BD10B5002128
:101580000220FFF73EFF032808D000210320FFF7C9
:1015900038FF0021BDE81040022032E710BD0021D5
:1015A00001202EE79F4901200860704770B5002494
:1015B0000425FFF7F7FFFFF7C7FE4FF47A7610E038
:1015C000641CE4B2304603F049FA97A1524801F096
:1015D000F1FB002805DB214694A001F0AFF90325BB
:1015E00001E0142CECD3284670BD8E490020086021
:1015F00040F6B83003F032BA10B510220F210420A3
:1016000002F068FCFFF7F1FF10220B21042002F02A
:1016100061FC844900201039086010BD10B5012319
:101620000C224FF4E131022001F02EFDFFF78CFE79
:10163000FFF78FFE414801F027FA514801F024FAE4
:10164000AFF2E721BDE81040022001F0F1BC70B517
:10165000FFF7E4FFFFF7D0FFFFF7A8FFFFF79FFFBB
:10166000FFF78CFF04462C483838FFF76EFF2A4AF4
:101670001421383A73A001F033F92748233805467E
:10168000FFF746FF294674A001F02AF9204670BDF5
:1016900010B500210846FFF7B4FE0446032C02D023
:1016A00073A001F077F94FF47A7003F0D7F9FFF7E0
:1016B0009CFF204610BD00005455524E4F46460038
:1016C00048414E445348414B450000005155455256
:1016D00059434F4E46494700434C4F534545434FAE
:1016E0000000000053415645434F4E464947000015
:1016F000515545525952454C455345005155455257
:1017000059564F4C5441474500000000CEDEB4CB43
:10171000C3FCC1EE00000000CC1C00200C1E002009
:10172000D40100202B51495552433A002B514955C1
:1017300052433A2022726563762200004C1F00203B
:101740002E2E5C48415244574152455C4C54455CF6
:10175000454332305C656332306D6F64756C652E65
:101760006300000025732C25643A7354637051752F
:10177000657565207370696C6C6F766572A3A100E6
:101780005223002025732C25643A735572635175DA
:10179000657565207370696C6C6F766572A3A100C6
:1017A00025732C25643A6563323041744275662096
:1017B0007370696C6C6F7665722E200025732C2512
:1017C000643A636D645061636B207370696C6C6F15
:1017D000766572A3A1000000496E506172616D458B
:1017E000727200004F7574506172616D45727200C3
:1017F00052554E455252000052554E4F4B0000007C
:1018000054494D454F555400CEB4D6AAB4EDCEF34D
:1018100000000000257320257300000033353030B0
:1018200000000000BC0123425244590045433230BD
:10183000205374617274205761697465643A256439
:10184000205300004543323020C8EDBCFEB0E6B165
:10185000BEA3BA252E2A73004543323020B9A9B55C
:10186000E7B5E7D1B9A3BA2573206D560000000093
:101870004543323020C8EDB9D8BBFACAA7B0DCA3C3
:10188000ACBCB4BDABB6CFB5E7B9D8BBFAA3A10029
:101890000FB42DE9F84F81460427F348C9EBC9017D
:1018A00000EB8104667E60680B90802000F0DAFF18
:1018B00082460CAB0093802150460B9A08F06EFFD5
:1018C0008046B8F1000F02DDB8F1800F2FDD6522F0
:1018D000E6A1EEA001F05EF802272BE0FFF734FD51
:1018E00000251FFA88F25146022001F002FD14E0A3
:1018F000642003F0B3F8E168EB4801F05BFA206183
:101900002069002801DB032714E06169E64801F043
:1019100051FA002801DB02270CE028466D1C2189C2
:10192000EDB28842E4D34FF47A7003F097F8761E54
:10193000F6B2D3D2504600F0CFFF00200090052F22
:101940000ED2DFE807F0030507090B00D7A408E073
:10195000D9A406E0DBA404E0DCA402E0DDA400E0FE
:10196000DEA4484600F05AF901462246DEA000F007
:10197000E5FF3846BDE8F80F5DF814FB024600218C
:10198000DBA3072084E702460021082080E7024607
:10199000002109207CE72DE9F04104460F4622464C
:1019A00000210A20FFF774FF0646032E20D1AE4D1A
:1019B000012C20D0022C25D0032C2AD0CEA1BA484D
:1019C00001F0F8F9C5F82801D5F8280100280EDB48
:1019D000D5F82811B44830340830085CA04206D14C
:1019E000D5F82811B0480A30085C312818D00226F2
:1019F0003046BDE8F081C0A1AB4801F0DBF9C5F885
:101A00002801E1E7BFA1A84801F0D4F9C5F82801F1
:101A1000DAE7BFA1A44801F0CDF9C5F82801D3E762
:101A2000D5F82811A04810230F300144222238464F
:101A300001F0E3F8DCE72DE9F04104252D24002135
:101A40000120FFF725FF984E874F09364FF4FA68BB
:101A500015E0404603F002F800210220FFF718FFCE
:101A60000546032D0BD1B86C002807DDB86C805DEE
:101A7000312807D0B86C805D352803D00225641E5C
:101A8000601CE6D12846B4E72DE9F04104251E2468
:101A900000210320FFF7FCFE834E734F0A364FF4FC
:101AA000FA6818E0404602F0D9FF00210420FFF751
:101AB000EFFE0546032D0ED1D7F88000002809DD82
:101AC000D7F88000805D312808D0D7F88000805D8D
:101AD000352803D00225641E601CE3D1284688E720
:101AE00070B505461921284609F07FFA00210846FD
:101AF000FFF7CEFE0446032C09D15B4801696A4812
:101B00001923083001440D22284601F076F82046BA
:101B100070BD10B500210520FFF7BAFE032801D0E3
:101B20007EA010BD504C9C3420685F4908440D21B4
:101B300009F0EFF80021017021685B480A30084481
:101B400010BD70B505460020286000210620FFF773
:101B50009FFE0446032C0AD14348D0F8B8105248DF
:101B60001923801D01442C22284601F046F8204606
:101B700070BD2DE9F04105460E466D480446FFF75D
:101B8000AFFF032809D06BA23146284608F042FE79
:101B90006BA000F0FFFE02202BE7224619216CA06B
:101BA00000F09EFEFFF747FF0446032C09D06DA20C
:101BB0003146284608F02EFE6DA000F0EBFE022014
:101BC00017E7FFF761FFFFF7A4FF01466EA000F0E3
:101BD00087FE5748001F0746FFF7B3FF3B466EA23C
:101BE0003146284608F016FE3A4603216DA000F063
:101BF00077FE2046FDE670B505460E462846FFF7FF
:101C0000BDFE2846FFF7BFFE0446032C03D1314634
:101C10002846FFF7C0FE204670BDB8E610B50B2879
:101C20001DD2DFE800F006080A0C0E101214161878
:101C30001A0060A010BD62A010BD63A010BD64A01A
:101C400010BD65A010BD66A010BD69A010BD6BA041
:101C500010BD6DA010BD6FA010BD72A010BD75A00D
:101C600000F098FE79A010BD9C0200202E2E5C484A
:101C7000415244574152455C4C54455C45433230D7
:101C80005C656332306E65742E63000025732C250D
:101C9000643A636D645061636B207370696C6C6F40
:101CA000766572A3A1000000CC1C0020496E506133
:101CB00072616D45727200004F7574506172616D92
:101CC0004572720052554E455252000052554E4FC9
:101CD0004B00000054494D454F555400CEB4D6AA90
:101CE000B4EDCEF300000000257320257300000042
:101CF000434D494F540000002B51494143543A2071
:101D0000310000002B51494143543A203200000079
:101D10002B51494143543A2033000000BBF1C8A184
:101D2000CDF8C2E7D0C5CFA2CAA7B0DC2100000021
:101D3000B21C0020C7EBB2E5C8EB53494DBFA80069
:101D4000CEB4BCECB2E2B5BD53494DBFA800000013
:101D500053696DBFA84943434944A3BA252E2A734A
:101D60000000000053494DBFA8C7B7B7D10000001D
:101D700053494DC7B7B7D1CEDEB7A8D7A2B2E1C994
:101D8000CFCDF8C2E7000000CDF8C2E7D0C5CFA2A2
:101D9000A3BA257300000000D0C5BAC5D6CAC1BF1A
:101DA0003A2573004C544520435351A3BA252E2A9B
:101DB00073000000515545525949434349440000BE
:101DC0005345544353000000515545525943530065
:101DD000534554505300000051554552595053003B
:101DE00051554552594E4554494E464F000000004A
:101DF000515545525943535100000000434F46434B
:101E00004F4E544558540000414354434F4E54459F
:101E1000585400004445414354434F4E5445585490
:101E2000000000005155455259434F4E54455854F7
:101E3000000000004543323020CEDED0A7654E655D
:101E400074436D644E756D2100000000CEDEB4CB8E
:101E5000C3FCC1EE0000000005280ED2DFE800F050
:101E6000030507090B00D7A07047D9A07047DBA076
:101E70007047DCA07047DDA07047DEA070470528E2
:101E80000ED2DFE800F0030507090B00DCA0704765
:101E9000DEA07047E0A07047E2A07047E4A0704762
:101EA000E6A0704770B5102000F0DCFC054629461E
:101EB0000120FFF770FD032807D029460120FFF716
:101EC0009AFE0446032C02D005E0032070BD29468B
:101ED000DDA000F005FD284600F0FEFC204670BDA8
:101EE0000FB42DE9F84F81464FF00408DA48C9EBEA
:101EF000C90100EB8104667E60680B90802000F0D1
:101F0000B1FC82460CAB0093802150460B9A08F03E
:101F100045FC0746002F01DD802F2FDDCFA000F00C
:101F200039FD4FF002082CE0FFF70EFA0025BAB297
:101F30005146022001F0DDF916E0642002F08EFD2A
:101F4000E168D24800F036FF20612069002802DBFA
:101F50004FF0030815E06169CC4800F02BFF002822
:101F600002DB4FF002080CE028466D1C2189EDB21F
:101F70008842E2D34FF47A7002F070FD761EF6B21A
:101F8000D2D2504600F0A8FC4046FFF765FF044659
:101F90004846FFF774FF01462246BDA000F0CEFC84
:101FA0004046BDE8F80F5DF814FB7CB50246002101
:101FB0000220FFF795FF0646032E2BD1002000904C
:101FC0000190162000F04EFC0446A34DA96CAF48CA
:101FD0000A30085C2070A96CAC481023133001440F
:101FE0002C22601C00F009FE601C08F009FFA96C9F
:101FF0001430A64A0523114401442C22684600F0FF
:10200000FCFD21786B46621CA3A000F097FC2046E3
:1020100000F062FC30467CBD1CB50446CDE90023CF
:102020000B46002122460846FFF75AFF03280ED12F
:1020300089490B69954A303409329A5CA24205D12C
:102040000A6992490B31515C302900D002201CBD35
:1020500002460021012043E770B504462078FFF7CF
:10206000F7FF03280CD1A38A628A2078611CFFF74E
:10207000D3FF0546032D02D12078FFF796FF2846AF
:1020800070BD2DE9F84F06468A469146B9F1000F1A
:102090000DD00025A84600240427FFF755F9327813
:1020A0006D4EB16D4B46022001F06CF90DE003203E
:1020B000BDE8F88F142002F0D1FC3E21734808F0EF
:1020C00028FE10B14FF0010804E028466D1CEDB267
:1020D0004628EFD3B8F1010F10D03846FFF7BCFE09
:1020E00004460320FFF7CBFE01466848009077A323
:1020F000224679A000F04EFC3846D9E74A465146C0
:10210000022001F0F6F830E0642002F0A7FCF16F45
:102110005E4800F04FFEC6F88000D6F88000002828
:102120000DDB03273846FFF797FE04460420FFF730
:10213000A6FE0146224656A000F000FCDCE7D6F8D9
:102140008410524800F036FE00280EDB0227384685
:10215000FFF782FE04460420FFF791FE01464B4B39
:10216000224660A000F016FCC6E72046641CB6F8C4
:102170007810A4B28842C7D3BEE770B505460524DF
:102180005BA1284600F016FE002801DD002416E0C1
:102190005CA1284600F00EFE002801DD04240EE0BC
:1021A0005DA1284600F006FE002801DD022406E0BD
:1021B0005EA1284600F0FEFD002800DD0324204635
:1021C00070BD0000496E506172616D457272000011
:1021D0004F7574506172616D4572720052554E4573
:1021E0005252000052554E4F4B00000054494D458D
:1021F0004F555400CEB4D6AAB4EDCEF30000000083
:102200004F50454E534F434B45540000434C4F53A2
:1022100045534F434B4554005155455259534F4335
:102220004B45540054435053454E44434D440000E5
:1022300054435053454E444255460000CEDEB4CB85
:10224000C3FCC1EE00000000544350B1BEB5D849F4
:1022500050A3BA2573000000D003002054637020FF
:10226000636D645061636B20D2E7B3F6A3A12D2D9B
:10227000D4F6BCD35443505F434D445041434B5F6D
:102280004C454ECAFDD6B5A1A3000000CC1C0020D1
:102290002573202573000000544350204368616E6D
:1022A0006E616CA3BA256320A1A320B7FECEF1C650
:1022B000F74950A3BA2573A1A320B7FECEF1C6F704
:1022C000B6CBBFDAA3BA257300000000CEB4CAD5DE
:1022D000B5BD223E22000000257320257320257302
:1022E000202573002573202573202573000000002E
:1022F0002B51495552433A2022636C6F7365642217
:10230000000000002B51495552433A20227064705E
:1023100064656163742200002B51495552433A2091
:1023200022696E636F6D696E672200002B514955FB
:1023300052433A2022696E636F6D696E672066753D
:102340006C6C220005280ED2DFE800F003050709B7
:102350000B00D5A07047D7A07047D9A07047DAA06E
:102360007047DBA07047DCA07047092818D2DFE86F
:1023700000F00507090B0D0F11131500D9A07047C8
:10238000DBA07047DDA07047DFA07047E1A0704779
:10239000E3A07047E4A07047E6A07047E8A070474C
:1023A000EAA070470FB42DE9F84F81464FF00408BA
:1023B000E948C9EBC90100EB8104667E60680B90B7
:1023C0004FF49675284600F04DFA82460CAB009308
:1023D000294650460B9A08F0E1F90746002F01DD27
:1023E000AF422EDDDDA000F0D5FA2DE0FEF7ACFF08
:1023F0000025BAB25146022000F07BFF16E03220E1
:1024000002F02CFBE168E14800F0D4FC2061206977
:10241000002802DB4FF0030816E06169DB4800F09A
:10242000C9FC002802DB4FF002080DE028466D1CB5
:102430002189EDB2B0EB410FE1D34FF47A7002F095
:102440000DFB761EF6B2D1D2504600F045FA40465A
:10245000FFF778FF04464846FFF787FF014622460C
:10246000CBA000F06BFA4046BDE8F80F5DF814FB16
:1024700010B500210846FFF795FF032809D1002178
:102480000120FFF78FFF032803D1BDE81040002192
:1024900088E710BD70B5102000F0E4F90546294624
:1024A0000220FFF778FA032807D029460220FFF719
:1024B000A2FB0446032C02D005E0032070BD294690
:1024C000B5A000F00DFA284600F006FA204670BDCF
:1024D000F8B50446204608F093FC0A30064600F0A2
:1024E000C1F90546B0A3B2A231462846009408F0CF
:1024F00091F9284608F084FC024600210420FFF7E9
:1025000051FF0446032C0BD12A4600210520FFF77A
:1025100049FF0446032C03D12946A7A000F0E0F9A7
:10252000284600F0D9F92046F8BD10B50424FFF77D
:102530009FFF032801D0204610BDBDE81040A9E749
:102540002DE9FF4104460F466068FFF7C1FF4FF4D5
:102550009676304600F086F90546384608F050FC7D
:10256000D4E90131CDE90207CDE90013314628460F
:10257000226808F04FF90246002A01DDB24204DD6C
:10258000022491A000F006FA0CE000210620FFF7DB
:1025900009FF0446032C05D12A4600210720FFF736
:1025A00001FF0446284600F097F904B02046BDE834
:1025B000F081002808D0A0F50070BD3807D00128B0
:1025C00008D08EA000F08CB992A000F089B998A034
:1025D00000F086B99CA000F083B92DE9F0410024F9
:1025E0000426FEF7B6FE9D4F012038705A4DD5F8EF
:1025F000E40008F005FCD5F8E41082B2022000F0F7
:1026000078FE39E0642002F029FA55F8EC1F94486E
:1026100000F0D0FB68606868EC3D002823DBD5F84B
:10262000F0108F480C30085C302819D055F8F01F96
:102630008B482A68401C095C642030394143884833
:10264000801C105C2A68303800EB800001EB4001F0
:102650008348C01C105C08440226FFF7AAFF12E062
:1026600000200326F9E7D5F8F410484800F0A2FB53
:10267000002801DB022606E02046641CB5F8E810BD
:10268000E4B28842BED3002038703046FFF75AFECD
:1026900004460820FFF769FE014622463CA000F0F0
:1026A0004DF9304683E70000496E506172616D4517
:1026B000727200004F7574506172616D45727200E4
:1026C00052554E455252000052554E4F4B0000009D
:1026D00054494D454F555400CEB4D6AAB4EDCEF36F
:1026E0000000000048545450434F4E54455354008A
:1026F000454E52455148454144455200434C4F5385
:102700004554494D45000000424F445954595045E5
:102710000000000053455455524C434D4400000006
:102720004854545055524C00504F53545245514305
:102730004D440000504F53545245514255460000FD
:10274000485454505245414400000000CEDEB4CB02
:10275000C3FCC1EE000000005C04002048747470EB
:1027600020636D645061636B20D2E7B3F6A3A12DA3
:102770002DD4F6BCD3485454505F434D445041438C
:102780004B5F4C454ECAFDD6B5A1A300CC1C002022
:10279000257320257300000048545450B1BEB5D8AD
:1027A0004950A3BA25730000687474703A2F2F0043
:1027B0002573257300000000504F53542055524C90
:1027C0003A25732E00000000686561646572426FEF
:1027D000647942756620D2E7B3F6A3A12D2DD4F615
:1027E000BCD3485454505F434D445041434B5F4C1D
:1027F000454ECAFDD6B5A1A3000000004854545070
:10280000285329206F74686572206572726F722E6A
:102810000000000048747470204F70657261746924
:102820006F6E207375636365737366756C2E00003D
:102830004854545028532920756E6B6E6F776E2064
:102840006572726F722E000048545450285329202C
:1028500074696D656F75742E00000000D40100204E
:102860000C1E002070B506463146002000F0AEFB7D
:102870000446002000F017FB05464B2D08D918220E
:102880005AA161A007F0A4FF294663A007F0A0FFAA
:1028900024B13146204608F0A8FB1BE0202253A1BA
:1028A00059A007F095FF294663A007F091FF00208B
:1028B00000F0E0FA3146002000F088FB04464CB9F5
:1028C00025224AA150A007F083FF68A007F080FFEF
:1028D00004F0E6FE204670BD0146002000F06DBB0E
:1028E0000FB4F8B507AD00954FF400742046FFF71C
:1028F000B9FF06465EA22146304607F08BFF04462C
:10290000C4F5007130192B46069A07F047FF0028DE
:1029100006DD204482B23146002000F0EAFC07E0E8
:10292000502232A138A007F053FF50A007F050FF0B
:102930003046FFF7D1FFF8BC5DF814FB0FB4F8B5D3
:1029400007AD00954FF400742046FFF78BFF064655
:1029500049A22146304607F05DFF0446C4F50071E8
:1029600030192B46069A07F019FF002806DD20448F
:1029700082B23146002000F0BCFC07E06E221BA1B1
:1029800021A007F025FF39A007F022FF3046FFF70E
:10299000A3FFD0E70FB4F8B507AD00954FF400746E
:1029A0002046FFF75FFF064635A22146304607F076
:1029B00031FF0446C4F5007130192B46069A07F022
:1029C000EDFE002806DD204482B23146002000F0F2
:1029D00090FC07E08B2205A10BA007F0F9FE23A0D5
:1029E00007F0F6FE3046FFF777FFA4E72E2E5C5384
:1029F000595354454D5C535953504F52545C73795D
:102A000073706F72742E63004C6F674572723A2058
:102A100025732C25640000000D0AB6AFCCACC4DAD7
:102A2000B4E6D5BCD3C3D2D1B3ACB9FDA3BA256447
:102A30002525A3A10D0A00000D0AC4DAB4E6D5BC11
:102A4000D3C3A3BA256425252D2DB6AFCCACC4DAEB
:102A5000B4E6D2E7B3F6A3A1B3F5CABCBBAFB6AF39
:102A6000CCACC4DAB4E6BFD5BCE4A3A1000000003E
:102A70004C6F674170703A004C6F674465623A0072
:102A80004C6F674572723A0000210180418081805D
:102A90004FF48061801D08F0A8BA2DE9F0418388C9
:102AA000161D33444FF48067BB4202D30120BDE8BA
:102AB000F08145881223841D2B5543885B1CC3F38A
:102AC00009034380458834232B5543885B1CC3F39B
:102AD0000903438000230BE011F8015BB0F802C04A
:102AE0000CF8045045886D1CC5F3090545805B1C36
:102AF0009342F1DB4288562111554188491CC1F3AC
:102B0000090141804288782111554188491CC1F34F
:102B1000090141808188314481808188B94209D38B
:102B2000FFF7B2FF4322BFA1C5A007F051FEC8A026
:102B300007F04EFE0020BAE770B58388002B08D05E
:102B400003889B1CC3F30903038000231380831DA8
:102B500021E0022070BD1488641C14800488E45CA9
:102B600001F8014B0488641CC4F309040480148830
:102B70008588AC4203D20488B4F5806F0BD3FFF78D
:102B800083FF6622A7A1AEA007F022FEB0A007F047
:102B90001FFE022070BD0488E45C562CDBD1048843
:102BA000641CC4F309040444A479782CD3D10188AB
:102BB000891CC1F30901018081881288891A091FC3
:102BC0008180002070BD2DE9F04105460C46174676
:102BD000284608F015F90646384608F011F931186C
:102BE000A14204DB00212A19101A00F8011C394601
:102BF0002846BDE8F04108F06DB930B50546002023
:102C00005B1E04E02C54984204DA401C80B20C5C39
:102C10009442F7D130BD70B50446084611461D46B2
:102C2000049E08F076F80246012006E0231803F817
:102C3000011CB04204D8401C80B2115CA942F5D1FD
:102C400070BD30B500231144491E18E00C782409EA
:102C50000A2C01D2302500E037252C4400F813401F
:102C60000C7804F00F040A2C01D2302500E037253F
:102C70002C4400EB43056C705B1C9BB2491E9342D5
:102C8000E4D330BD30B500231AE0CD5C2C0905F04B
:102C90000F053034392C03D9E41D00F8134001E04E
:102CA00000F813403035ECB2392C04D900EB430561
:102CB000E41D6C7002E000EB43056C705B1C9BB282
:102CC0009342E2D330BDF0B5034600250846002606
:102CD0000A2A01D00670F0BD002B1DD005DA4FF096
:102CE0002D0200F8012BC3F1000342F210724FF0E5
:102CF0000A0793FBF2F454EA050C06D004F1300500
:102D000000F8015B04FB1233012592FBF7F2002A65
:102D1000EFDC06700846F0BD3022027046700846AF
:102D2000F0BDF0B505460023002042F210720A26DD
:102D3000B5FBF2F4E4B254EA000704D0303407469D
:102D4000401CC0B2CC55B5FBF2F402FB1455B2FBEB
:102D5000F6F25B1CDBB2052BEAD308B93020087011
:102D60000846F0BD2DE9F04105460C46284608F01E
:102D700047F880B2002100B121700122002312E047
:102D8000AE5CEF5CBE420CD1521C92B25B1C9BB29B
:102D9000AE5CEF5CBE4201D0A35404E0E65CA654F6
:102DA00001E01BB1E35C8242EAD380E6521C92B29E
:102DB000A154F8E72DE9F04782468946504608F0CD
:102DC0001FF887B2484608F01BF886B20025002499
:102DD0003046FFF747FD804641464846FFF7C2FFB1
:102DE0000DE01AF8050019F80410884204D16D1C92
:102DF000ADB2641CA4B202E06CB118F80440BD424C
:102E000001D2B442EDD34046FFF766FDB44205D38C
:102E1000A81BBDE8F0876D1CADB2F0E74FF0FF30A6
:102E2000F7E700002E2E5C53595354454D5C53591F
:102E3000534C49425C7379736C69622E63000000E5
:102E40004C6F674572723A2025732C256400000090
:102E50000000000003E011F8013B00F8013B521EA6
:102E6000531CF8D1704701E000F8011B521E531C9F
:102E7000FAD1704770B504466B486C4E002150F88B
:102E8000240006EB840542002869FFF7ECFF664842
:102E90000021103050F82420A868FFF7E4FF01203B
:102EA0003119087670BD10B5002200215E4B5F4CD1
:102EB00053F8203004EB800005E0046934F8114039
:102EC00004B1521C491C8B42F7D864204243B2FB28
:102ED000F3F0C0B210BD2DE9F04105460F460024C5
:102EE000DFF8488108EB0500007E002803D1D8F800
:102EF0000010284688474FF0FF32FFB14A4E08368F
:102F000056F82500B7FBF0F3B7FBF0F100FB1170AA
:102F100000B15B1C444850F82510491E002921DBF4
:102F200008EB8507386930F811C0BCF1000F08D0F4
:102F300000249C4213D1002298B20AE01046BDE85A
:102F4000F081641CF5E73C6901EB020C24F81C00DD
:102F5000521C9A42F7D356F825004843EFE7491E22
:102F60000029E0DA1046EAE770B5304A13181B7EF4
:102F7000002B13D02C4B103353F820308B421AD92E
:102F8000294B083353F82030B1FBF3F102EB8002F8
:102F9000106930F811300020002408E011688847DB
:102FA000012070BD15690E1825F81640401C984286
:102FB000F8DB002070BD022070BD002905D01B4A3F
:102FC00002EB80029268891ACEE7704710B504467A
:102FD0002046FFF780FF411C05D0144901EB840116
:102FE0008968084410BD002010BD2DE9F041064657
:102FF0008846174639463046FFF76DFF0446601C89
:103000000FD00A483A4600EB86054146A86820449E
:10301000FFF720FF41463046FFF7CFFFA868204466
:103020008DE700208BE7000010F60408580500200B
:1030300010B50C46F24A52F82030002B09D052222B
:10304000F0A1F6A007F0C4FBF8A007F0C1FB2046F2
:1030500010BD42F82040FAE730B40C46E84951F878
:103060002030002B03D0204630BC1146184730BC1E
:10307000704770477047F449C2B20B689A8009687C
:103080000A885206FCD570472DE9F04387B0044604
:103090000D46164698460121084602F0D4FBEA4840
:1030A00018220F38015D401F005D00F013FFE64855
:1030B0000422401F015D401F005D00F00BFFE3484C
:1030C000002C7CD050F82400012102F0C7FB0295AF
:1030D0000025ADF80C50ADF80E50ADF81050ADF81D
:1030E0001450ADF81260D84E02A956F8240002F030
:1030F00049FC56F824004FF4587102F093FDBDF8D6
:10310000120006F11409000722D5042C20D056F82D
:1031100024000122802102F0D7FCCC4F00950195BC
:10312000183F59F82410385D1023002200F02BFCC2
:1031300006F12400002150F82420385D00F01CFB2B
:10314000AF480121303850F82420385D00F014FBDE
:10315000BDF81200400759D5BC481038005D8DF805
:1031600018008DF819808DF81A5001208DF81B0079
:1031700006A802F0A2F856F82400012240F22441E9
:1031800002F087FC042C3BD056F824000122402199
:1031900002F09AFCCDE90058AC4859F824101430DC
:1031A000A0F1280550F82420285D002300F0EBFB57
:1031B00005F10A00A64F30F81410285D00E01AE06F
:1031C00057F8200004F0FCF98D480021203850F811
:1031D0002420285D00F0D0FA89480121103850F8E9
:1031E0002420285D00F0C8FA285D012157F820004E
:1031F00004F0CFF90AE00068012102F024FB66E741
:10320000012240F22551306902F043FC56F82400B7
:10321000012102F032FC07B0BDE8F0831CB5044682
:1032200089480122802150F8240002F04DFC06203C
:103230000021CDE90010844810231430002250F8FA
:10324000241082481838005D00F09DFB1CBD7CB541
:1032500004467D480122402150F8240002F034FC4D
:1032600006200021CDE900107848784D1430143D37
:1032700050F8242074480023143050F82410285D9E
:1032800000F081FB05F10A00714E30F81410285D42
:1032900056F8200004F094F9285D012156F820002A
:1032A000BDE87C4004F075B92DE9F0410446674D56
:1032B000674E143D0021285D56F8200004F069F99E
:1032C00005F10A0705F1280037F8141050F824001A
:1032D00007F08BFE285D37F8141056F8200004F034
:1032E0006FF9285D012156F82000BDE8F04104F097
:1032F00050B92DE9F047044688461646B8F1000F4C
:1033000025D0002E23D0042C23D0504FDFF840913D
:10331000183F0021385D59F8200004F03AF94A4D71
:103320000020183D2855385D59F82000C0F80C8061
:10333000385D314659F8200004F042F9385D01212A
:1033400059F8200004F025F9285D0028FCD0BDE8DC
:10335000F08700253C4F4021386902F05CFC0EE00C
:1033600018F8051057F8240002F0E8FB57F824007D
:10337000402102F050FC0028F8D06D1CADB2B542DF
:10338000EED3E4E70FB470B586B004460CA8019004
:103390002D4E10E05C2916D025295BD0401C0B90E7
:1033A00056F8240002F0CAFB56F82400402102F02F
:1033B00032FC0028F8D00B9801780029EAD106B039
:1033C00070BC5DF814FB401C0B9001786E290DD089
:1033D000722902D0401C0B90E6E756F824000D211C
:1033E00002F0ACFB0B98401C0B90DDE756F8240074
:1033F0000A2102F0A3FB0B98401C0B90D4E70000BD
:10340000505600202E2E5C53595354454D5C555355
:103410004152545C75736172742E63004C6F674542
:1034200072723A2025732C25640000005561727475
:103430002043616C6C6261636B20726570656174BE
:1034400020726567210000009005002040F6040806
:10345000C8050020401C0B90017864291BD07329FB
:1034600002D0401C0B909FE7019820C801900BE010
:1034700056F8240002F062FB56F82400402102F0C6
:10348000CAFB0028F8D06D1C29780029F0D10B98D0
:10349000401C0B9088E7019808C801900A2202A9F5
:1034A0001846FFF710FC02AD0BE056F8240002F0BE
:1034B00045FB56F82400402102F0ADFB0028F8D06F
:1034C0006D1C29780029F0D10B98401C0B906BE7FC
:1034D00070B59D4C40F22441204602F0A7FBA0B1FC
:1034E0009A4D0021286904F054F82088201D008896
:1034F000286904F067F8C0F5807082B29449002012
:10350000FFF7AAFD0020FFF7CFFE40F22555294620
:10351000204602F08BFB18B12946204602F0A6FB9C
:1035200040F227752946204602F080FB002806D08D
:1035300029462046BDE87040002202F0AABA70BDBC
:1035400070B5844C40F22441204602F06FFBA0B1DC
:103550007E4D0021686904F01CF82088201D008839
:10356000686904F02FF8C0F5807082B27A490120B2
:10357000FFF772FD0120FFF797FE40F2255529461F
:10358000204602F053FB18B12946204602F06EFB9C
:1035900040F227752946204602F048FB002806D055
:1035A00029462046BDE87040002202F072BA70BD84
:1035B00070B56A4C40F22441204602F037FBA0B1BE
:1035C000624D0021A86803F0E4FF2088201D0088D8
:1035D000A86803F0F7FFC0F5807082B2604902204E
:1035E000FFF73AFD0220FFF75FFE40F2255529461E
:1035F000204602F01BFB18B12946204602F036FB9C
:1036000040F227752946204602F010FB002806D01C
:1036100029462046BDE87040002202F03ABA70BD4B
:1036200070B5504C40F22441204602F0FFFAA0B1A0
:10363000464D0021686A03F0ACFF2088201D0088F9
:10364000686A03F0BFFFC0F5807082B2464903206C
:10365000FFF702FD0320FFF727FE40F2255529461C
:10366000204602F0E3FA18B12946204602F0FEFA9D
:1036700040F227752946204602F0D8FA20B10022F0
:103680002946204602F005FA2046BDE87040402158
:1036900002F0C8BA2DE9F041344D40F225512846D8
:1036A00002F0C4FA324C002658B1AA882168481C9E
:1036B000206030484254216846542068FF2800DBCF
:1036C000266040F224473946284602F0AFFA88B116
:1036D0002888A8882068274982B20420FFF7BCFC0C
:1036E0004FF48071234807F0A2FC26603946284633
:1036F00002F0BCFA40F227742146284602F096FAFE
:10370000002806D021462846BDE8F041002202F0FC
:10371000C0B9BDE8F08116490120091D0870704745
:1037200013490120091D4870704711490120091DE6
:10373000887070470E490120091DC8707047704796
:10374000704770477047000000380140C8050020EE
:1037500064560020004400406457002000480040A8
:1037600064580020004C0040645900200050004084
:1037700074050020645A002010B5144600290BD0AF
:10378000012919D04E22E9A1EDA007F021F8F0A0FF
:1037900007F01EF8204610BDF64951F8202042B12E
:1037A0004322E2A1E6A007F013F8F3A007F010F817
:1037B000F0E741F82040EDE7EE49303151F82020A4
:1037C00042B14A22D9A1DEA007F002F8F1A006F02A
:1037D000FFFFDFE741F82040DCE730B4E549B0F116
:1037E000007F01F1300271D036DCB0F5005F6ED0A1
:1037F00018DC80287AD00ADC02286DD0082870D026
:10380000202868D14868002865D030BC0047B0F552
:10381000007F71D0B0F5006F5DD1906800285AD05C
:1038200030BC0047B0F5002F77D00ADCB0F5004F70
:103830006ED0B0F5003F4ED1086900284BD030BCA7
:103840000047B0F5001F6DD0B0F5000F43D15069AF
:10385000002840D030BC0047D54C031BA0427CD090
:103860001ADCD44CA0EB0403A0426CD00BDCB0F10A
:10387000006F61D0A0F18050801E2CD1C869002853
:103880007FD030BC0047182B62D0782B79D1106ADA
:10389000002876D030BC0047B3F5FC4F67D00ADC77
:1038A000B3F5C06F5ED0B3F5F05F6AD1886A0028C7
:1038B00067D030BC0047B3F5FF3F5DD0BE48C34280
:1038C0005FD1D06A00285CD030BC00472FE018E000
:1038D0000CE001E005E054E00868002851D030BC5D
:1038E0000047106800284CD030BC004750680028C2
:1038F00047D030BC0047FFE78868002841D030BC83
:103900000047C86800283CD030BC004705E0FFE70E
:10391000D068002835D030BC00471069002830D06E
:1039200030BC0047486900282BD030BC004788696C
:10393000002826D030BC00479069002821D030BC38
:1039400000470AE0FFE7D06900281AD030BC0047E2
:10395000086A002815D030BC0047486A002810D0FB
:1039600030BC0047506A00280BD030BC0047906A3A
:10397000002806D030BC0047C86A002801D030BCFF
:10398000004730BC70472DE9F0478CB00446DDE9B4
:1039900014980D4617469A46072C04D20121084672
:1039A00001F046FF03E00121022001F041FF834EB8
:1039B00056F8240003F04CFD01950297CDF80CA0B9
:1039C0000025049505958020069007950895CDF86B
:1039D000249040010A900B9556F8240001A903F0A9
:1039E000AEFD774810F824008DF800008DF80180B6
:1039F0008DF8025001208DF80300684601F05DFC4F
:103A000056F824000122022103F0D0FD0CB0BDE8DD
:103A1000F08710B5022003F0D8FD012805D102205F
:103A200003F0FBFD0220FFF7D8FE082003F0CDFDD8
:103A300001280ED1082003F0F0FDD5223BA140A0C3
:103A400006F0C6FE5FA006F0C3FEBDE810400820E9
:103A5000C3E610BD10B5202003F0B7FD012805D145
:103A6000202003F0DAFD2020FFF7B7FE802003F0CE
:103A7000ACFD01280ED1802003F0CFFDEB222BA15D
:103A80002FA006F0A5FE52A006F0A2FEBDE8104051
:103A90008020A2E610BD10B54FF40074204603F05C
:103AA00094FD012805D1204603F0B7FD2046FFF71D
:103AB00094FE4FF40064204603F087FD01280FD1E7
:103AC000204603F0AAFD40F2011218A11CA006F046
:103AD0007FFE42A006F07CFE2046BDE810407CE65A
:103AE00010BD10B54FF40054204603F06EFD0128C0
:103AF00005D1204603F091FD2046FFF76EFE4FF4FE
:103B00000044204603F061FD012874D1204603F0F3
:103B100084FD40F2171205A109A006F059FE32A05B
:103B200006F056FE2046BDE8104056E62E2E5C53A9
:103B3000595354454D5C444D415C646D612E6300A6
:103B40004C6F674572723A2025732C256400000083
:103B5000446D6154652043616C6C6261636B20222B
:103B6000654972715479706522206572726F722195
:103B700000000000645B0020446D615463204361D9
:103B80006C6C6261636B2072657065617420726534
:103B900067210000446D6154652043616C6C626173
:103BA000636B207265706561742072656721000027
:103BB00000020010080000100002F8FFC8050020F5
:103BC00064F60408444D41315F5445312100000042
:103BD000444D41315F54453221000000444D413194
:103BE0005F54453321000000444D41315F5445345A
:103BF00021000000FFE710BD10B54FF4003420464F
:103C000003F0E3FC012805D1204603F006FD204621
:103C1000FFF7E3FD4FF40024204603F0D6FC012813
:103C200011D1204603F0F9FC40F22D12AFF204113D
:103C3000AFF2F40006F0CCFD8AA006F0C9FD2046E4
:103C4000BDE81040C9E510BD10B54FF40014204682
:103C500003F0BBFC012805D1204603F0DEFC204622
:103C6000FFF7BBFD4FF40004204603F0AEFC012833
:103C700011D1204603F0D1FC40F24312AFF25411AF
:103C8000AFF2441006F0A4FD79A006F0A1FD204695
:103C9000BDE81040A1E510BD10B54FF000742046FE
:103CA00003F093FC012805D1204603F0B6FC204622
:103CB000FFF793FD4FF00064204603F086FC0128D7
:103CC00011D1204603F0A9FC40F25912AFF2A41121
:103CD000AFF2941006F07CFD68A006F079FD204656
:103CE000BDE8104079E510BD10B5674C204603F0E3
:103CF0006CFC012805D1204603F08FFC2046FFF71D
:103D00006CFD614CA41D204603F05FFC012811D11D
:103D1000204603F082FC40F26F12AFF2F011AFF2D6
:103D2000E01006F055FD59A006F052FD2046BDE812
:103D3000104052E510BD10B5534C1E34204603F020
:103D400044FC012805D1204603F067FC2046FFF71C
:103D500044FD4D4C7E34204603F037FC012811D140
:103D6000204603F05AFC40F28512AFF24021AFF238
:103D7000302006F02DFD45A006F02AFD2046BDE8C6
:103D800010402AE510BD10B5434C204603F01DFC41
:103D9000012805D1204603F040FC2046FFF71DFD19
:103DA0003E4C204603F011FC012811D1204603F0BF
:103DB00034FC40F29B12AFF28C21AFF27C2006F073
:103DC00007FD37A006F004FD2046BDE8104004E5DD
:103DD00010BD10B5354C204603F0F7FB012805D186
:103DE000204603F01AFC2046FFF7F7FC304C204633
:103DF00003F0EBFB012810D1204603F00EFC40F24B
:103E0000B112AFF2D821AFF2C82006F0E1FC29A030
:103E100006F0DEFC2046FFF7E0FC294C204603F0CC
:103E2000D4FB012805D1204603F0F7FB2046FFF71D
:103E3000D4FC244C204603F0C8FB012811D12046B5
:103E400003F0EBFB4FF4DF72AFF22031AFF2103032
:103E500006F0BEFC1CA006F0BBFC2046BDE81040EE
:103E6000BBE410BD444D41315F5445352100000095
:103E7000444D41315F54453621000000444D4131ED
:103E80005F5445372100000002000010444D4132CC
:103E90005F544532210000000002001000080010AD
:103EA000444D41325F544533210000000020001092
:103EB00000800010444D41325F5445342100000021
:103EC0000000021000000810444D41325F54453597
:103ED00021000000F8B504460D4616469848012119
:103EE00050F8240001F0AFFC95481C3030F8150064
:103EF000ADF800008DF8036003208DF802009148B2
:103F0000694650F8240001F098FAF8BD2DE9FE4307
:103F10000646DDF828900C46154698462A46214666
:103F20003046FFF7D7FF282D01D0482D36D101218B
:103F3000084601F088FC824F8C37385D8DF8000010
:103F40008DF8019000258DF802508DF803506846D9
:103F500001F0B3F9A7F15000015D4438805D01F034
:103F600028FBA7F1400656F8240001908DF8085070
:103F70008DF8098001258DF80A5001A802F0C6F8D5
:103F800056F8240002F021F9385700F01F018D4047
:103F90004009800000F1E020C0F80051BDE8FE8338
:103FA000684A52F82000C268654B1C3333F8111080
:103FB0004A40C260704710B50C46634A52F8203040
:103FC000002B09D0972261A165A006F001FC68A032
:103FD00006F0FEFB204610BD42F82040FAE770B51F
:103FE000064600204FF0804108F00AFC04460D46CA
:103FF000304609F0B5FD08F003FC22462B4609F0D7
:10400000A7FB09F039FD504951F82000002802D0E3
:10401000BDE87040004770BD10B5012002F0BAF84D
:1040200028B1012002F0BFF80120FFF7D8FFBDE85A
:104030001040012002F0C9B810B5022002F0AAF821
:10404000012805D1022002F0AEF80220FFF7C7FFD9
:10405000BDE81040022002F0B8B810B5042002F00C
:1040600099F828B1042002F09EF80420FFF7B7FF6A
:10407000BDE81040042002F0A8B810B5082002F0F6
:1040800089F8012805D1082002F08DF80820FFF7F3
:10409000A6FFBDE81040082002F097B810B5102028
:1040A00002F078F828B1102002F07DF81020FFF718
:1040B00096FFBDE81040102002F087B830B591B0EF
:1040C00005241F4D4C3555F8240002F070F888B1D6
:1040D00055F8240002F067F8402101A806F0A7FF78
:1040E000234629A2402101A806F094FB55F824009C
:1040F000FFF775FF641C092CE5DD11B030BD30B54C
:1041000091B00A240E4D4C3555F8240002F04FF8BA
:1041100088B155F8240002F046F8402101A806F0C5
:1041200086FF234618A2402101A806F073FB55F82C
:104130002400FFF754FF641C0F2CE5DDDDE70000D1
:104140009CF60408F8050020C45B00202E2E5C536A
:10415000595354454D5C494F5C696F2E6300000014
:104160004C6F674572723A2025732C25640000005D
:10417000494F2043616C6C6261636B2072657065AE
:1041800061742072656721004558544925642049AF
:1041900052512100002101604160018181720B2296
:1041A00010A106F06BBF0EB5114A12680092104ABA
:1041B000121D126801920E4A0832126802920029FA
:1041C0000BD0012904D00C226946FEF75BFD0EBD21
:1041D0000C226946FEF756FD0EBD0C22694606F01C
:1041E0004DFF0EBD4E6F762032302032303230001F
:1041F000E8F7FF1F10B50C46F54901280BD002283F
:1042000016D03D22F3A1F8A006F0E2FAFAA006F0DB
:10421000DFFA204610BD486840B13222EDA1F2A07D
:1042200006F0D6FAFBA006F0D3FAF2E74C60F0E70E
:10423000886840B13922E7A1EBA006F0C9FAFDA0D9
:1042400006F0C6FAE5E78C60E3E7E149012805D00E
:10425000022807D18868002804D000474868002851
:1042600000D00047704710B5012002F06EF838B159
:10427000012002F078F802F049F80120FFF7E5FF8D
:10428000022002F062F8002808D0022002F06BF849
:1042900002F03CF8BDE810400220D6E710BD10B592
:1042A000022002F052F800280CD04FF4003001F048
:1042B0008CFF022002F057F802F028F8BDE8104009
:1042C0000220C2E710BD30B56423B0FBF3F4E4B2C2
:1042D000B0FBF3F503FB1500132C01D96430C0B219
:1042E00000EB90030724B3FBF4F504FB1533D94D21
:1042F0001A440D4415F8015C2A4492B2800703D198
:10430000032901D2521E92B2B2FBF4F004FB10203A
:1043100030BD810701D0002070476421B0FBF1F26D
:1043200001FB120109B1012070474FF4C871B0FBC5
:10433000F1F201FB120008B1002070470120704724
:104340002DE9F04788B0044601F0E6FF01F0B5FF23
:104350000646DFF80483B6FBF8F39D480A27018878
:10436000994279D0038040F2B2754FF4B7794FF497
:10437000B67A0FE02846FFF7CCFF38B14B4502D3A1
:10438000A3F5B77304E06D1CADB205E0A3F26D13A5
:104390006D1CADB25345EDD80195BDF804104FF436
:1043A0007A70B1FBF0F130312170BDF80410B1FB2F
:1043B000F0F200FB12126421B2FBF1F230326270B3
:1043C000BDF80420B2FBF0F500FB1520B0FBF1F2C4
:1043D00001FB1200B0FBF7F03030A070BDF8040014
:1043E000B0FBF7F107FB11003030E0700025DFF87B
:1043F000649209F10C090DE0BDF80400FFF789FF94
:1044000008B1012D7AD019F80500984204D81B1A7A
:104410006D1CADB21C2BEFD26D1C04955B1C03937D
:104420009DF81000B0FBF7F0303060719DF810007F
:10443000B0FBF7F107FB11003030A0719DF80C00C4
:10444000B0FBF7F0303020729DF80C00B0FBF7F1B4
:1044500007FB110030306072B6FBF8F008FB10600B
:104460004FF46161B0FBF1F20792B0FBF1F201FB96
:1044700012033C22B3FBF2F30693B0FBF1F301FB12
:104480001300B0FBF2F102FB110005909DF81C0037
:10449000B0FBF7F03030E0729DF81C00B0FBF7F194
:1044A00007FB1100303020739DF81800B0FBF7F0C7
:1044B0003030A0739DF81800B0FBF7F107FB110036
:1044C0003030E0739DF81400B0FBF7F030306074CA
:1044D0009DF81400B0FBF7F107FB11003030A07419
:1044E0009DF80C209DF81010BDF80400FFF7EBFEBE
:1044F000029008B00320BDE8F087FFE71D2B8BD3A7
:104500001D3B85E755481BE708B503218DF80010D2
:104510008DF8010000208DF8020001208DF80300C5
:10452000684600F0CAFE08BD2DE9F04107460024A8
:104530004A48202181722D21C17101713A210174F3
:10454000417301214FF0C05001F088F90121084664
:1045500001F079F9012001F04DFE042001F0A4FDE5
:1045600045F25006B04232D001F074FD012001F056
:10457000F4F801F094FE01F0C9FE6FF07F4500E011
:10458000641C412001F06EF808B9AC42F8D3DFF8A2
:10459000D080444505D24FF4807001F0F3F8012437
:1045A00066E00024012001F0EAF800E0641C6120CC
:1045B00001F058F808B9AC42F8D3444570D24FF432
:1045C000007001F0DFF8CA2202A107A04AE079E0FA
:1045D000140600202E2E5C53595354454D5C525402
:1045E000435C7274632E63004C6F674572723A20AD
:1045F00025732C25640000005274635F5265674880
:104600006F6F6B43616C6C6261636B204661696CB8
:1046100065642100527463205365635469204361CB
:104620006C6C6261636B2072657065617420726589
:104630006721000052746320416C72546920436109
:104640006C6C6261636B2072657065617420726569
:104650006721000038F7040880510100045C002045
:10466000F0FFFF0006F0B4F8C9A006F0B1F800248E
:10467000012001F08CF801F049FEF4B147F6FF701B
:1046800001F02BFE01F042FE01F040FE01F00EFEB3
:1046900001F03CFE3146042001F0FEFC18E0FFE78B
:1046A000CF22AFF2D001AFF2C00006F091F8B8A06F
:1046B00006F08EF80220BDE8F08149F6404001F096
:1046C0000CFEDFE701F022FE0121084601F0DCFDCF
:1046D00001F01CFE0121084601F0D6FD01F016FE96
:1046E0000121022001F0D0FD01F010FE002001F0B8
:1046F00081FD3846FFF708FFA648FFF721FEAFF21D
:10470000FB110120FFF776FD0320D4E72DE9F05FD0
:1047100000230178C278303901EB4104C4EBC111A8
:1047200002EBC10442786421303A4A43817830393F
:1047300001EB810102EB4101214430398DB2417915
:104740008279303901EB81046FF02F0101EB4404D1
:104750002244D7B2027A447A303A02EB820201EB69
:1047600042022244D6B2C27A047B303A02EB820281
:1047700001EB4202224402F0FF08827BC47B303A04
:1047800002EB820201EB4202224402F0FF09827C2A
:10479000407C303800EB800001EB4000104400F01A
:1047A000FF0AA5F2B270822802D30220BDE8F09F72
:1047B00040F2B274DFF8E0B109E02046FFF7A9FD4E
:1047C00008B15B4401E075480344641CA4B2AC42E8
:1047D000F3D37F1EFFB20024DFF8C4B110E01BF852
:1047E000040040F2A321484303EBC0132846FFF71F
:1047F00090FD18B1012C01D16A480344641CA4B295
:10480000BC42ECD3761E40F2A320464303EBC61015
:10481000C8EB4811C1EB082100EB0110C9EB0911ED
:1048200000EB810000EB0A04012001F0E3FC01F041
:1048300036FD01F06BFD204601F048FD01F066FDFC
:1048400001F034FD01F062FD0320AFE72DE9F05FD8
:1048500000230178C278303901EB4104C4EBC11167
:1048600002EBC10442786421303A4A4381783039FE
:1048700001EB810102EB4101214430398DB24179D4
:104880008279303901EB81046FF02F0101EB440490
:104890002244D7B2027A447A303A02EB820201EB28
:1048A00042022244D6B2C27A047B303A02EB820240
:1048B00001EB4202224402F0FF08827BC47B303AC3
:1048C00002EB820201EB4202224402F0FF09827CE9
:1048D000407C303800EB800001EB4000104400F0D9
:1048E000FF0AA5F2B270822801D302205EE740F2EF
:1048F000B274DFF8A4B009E02046FFF70AFD08B162
:104900005B4401E025480344641CA4B2AC42F3D3E9
:104910007F1EFFB20024DFF888B010E01BF804000F
:1049200040F2A321484303EBC0132846FFF7F1FCF4
:1049300018B1012C01D11B480344641CA4B2BC4231
:10494000ECD3761E40F2A320464303EBC610C8EB1F
:104950004811C1EB082100EB0110C9EB091100EB74
:10496000810000EB0A04012001F044FC01F097FCF7
:1049700001F0CCFC204601F0B8FC01F0C7FC01F0CE
:1049800095FC01F0C3FC002001F034FC03200DE78E
:1049900000000000045C00200085E2018033E1019A
:1049A00044F704088051010010B505F057F90128BB
:1049B0000CD003F037FA3C48416811F1020F01D3E3
:1049C000002141604168491C416010BDBDE81040B4
:1049D00000F0BEB910B5042000F0B2FC33483449F1
:1049E000314A0068B0FBF1F31370B0FBF1F142F211
:1049F000107041430A2050804FF0E020026942F0DD
:104A0000020202614161016941F00101016110BDD1
:104A100070B505462748854208D90546612226A17A
:104A20002CA005F0D5FE2FA005F0D2FE00214FF0FE
:104A3000E02674691C4800784543B369B2699A421C
:104A4000FCD003D2A3EB0200014403E0A4EB02007C
:104A5000184401441346A942F0D370BD70B5044612
:104A600005F0FCF801280CD00F4D6888844203D370
:104A7000B4FBF0F004F076FC6888B4FBF0F100FBC6
:104A800011444FF47A706043BDE87040C0E770B5E0
:104A9000054600244FF47A7603E03046FFF7B8FF6E
:104AA000641CAC42F9D370BD2006002054060020DF
:104AB00040420F00E3388E032E2E5C535953544569
:104AC0004D5C5359535449434B5C73797374696318
:104AD0006B2E63004C6F674572723A2025732C254C
:104AE000640000000000000010B50C46794A52F83E
:104AF0002030002B09D0342277A17DA005F068FE7C
:104B00007FA005F065FE204610BD42F82040FAE780
:104B1000704951F82000002800D0004770472DE967
:104B2000FF4104460F4615461E4641F6991087423E
:104B300008D907465E2268A16DA005F049FE70A065
:104B400005F046FE6F48012150F8240000F086FE73
:104B50006C480838005D8DF80C008DF80D5000256C
:104B60008DF80E5001208DF80F0003A800F0A5FB72
:104B700041F61F40ADF80000ADF80650ADF8025008
:104B8000384608F0EDFF604A604B08F0E1FD002276
:104B90005F4B09F05BFA08F09FFFADF804008DF859
:104BA00008505C4D694655F8240001F0CDFC012207
:104BB00055F82400114601F0B2FF55F824003146A3
:104BC00001F093FF55F82400012102F0E7F9BDE858
:104BD000FF81504951F82000002102F0A7B970B5BB
:104BE00004464C4D002155F8240002F09FF955F879
:104BF0002400BDE87040012101F077BF454951F81C
:104C00002000002101F071BF10B501218C07204662
:104C100002F0B8F9012807D10121204602F0BEF9BF
:104C2000BDE81040002073E710BD10B53A4C0121DB
:104C3000204602F0A7F9012807D10121204602F001
:104C4000ADF9BDE81040012062E710BD10B5334C4E
:104C50000121204602F096F9012807D101212046C2
:104C600002F09CF9BDE81040022051E710BD10B5DC
:104C70002B4C0121204602F085F9012807D10121A2
:104C8000204602F08BF9BDE81040032040E710BD3C
:104C900010B5244C0121204602F074F9012807D1F7
:104CA0000121204602F07AF9BDE8104004202FE7E8
:104CB00010BD10B51C4C0121204602F063F90128FB
:104CC00007D10121204602F069F9BDE81040052016
:104CD0001EE710BD185C00202E2E5C53595354451E
:104CE0004D5C54494D45525C74696D65722E63008C
:104CF0004C6F674572723A2025732C2564000000C2
:104D00000000000058F704089A9999999999B93FB9
:104D10000000F03F2806002000040040000800408A
:104D2000000C0040001000400014004010B545F297
:104D3000555001F071F9062001F071F940F20D3083
:104D400001F070F901F071F9BDE8104001F072B99D
:104D500001F06BB903E010F8013B01F8013B521E72
:104D600092B2F8D270472DE9F04105460E4617463B
:104D7000002407E0284602F035FA26F81400AD1C9E
:104D8000641CA4B2BC42F5D3BDE8F0812DE9F0412A
:104D90000E4617460546002409E036F8141028464A
:104DA00002F022FA0428EFD1AD1C641CA4B2BC426C
:104DB000F3D3E9E72DE9F04FADF6040D82460F4637
:104DC0001546AAF10064B4F1005F04D300200DF68B
:104DD000040DBDE8F08F212000F044FC012809D02B
:104DE0006B22A3A1A8A005F0F3FCABA005F0F0FC9A
:104DF0000220ECE702F0EFF84FEAD428C4F34906AA
:104E0000C6F58064A54200D82C460DF1040B37E0AE
:104E100032183BF812208A4203D1401C80B2A042D3
:104E2000F6D3A04214D2484602F00EF9002006E064
:104E3000821937F810102BF81210401C80B2A042D3
:104E4000F6D348464FF4806201A9FFF79FFF04E0C4
:104E5000224639465046FFF799FFA54203D102F09A
:104E6000C6F80320B3E708F10108002607EB440762
:104E7000A244281B85B24FF48064A54200D82C467A
:104E80004FF0006000EBC829421401A94846FFF723
:104E90006AFF00204FF6FF71C1E72DE9F041074698
:104EA0000E46002402F0010000EB5205212000F024
:104EB000D9FB012809D0A8226DA173A005F088FCB8
:104EC00075A005F085FC02205EE702F084F8A7F1EA
:104ED0000060B0F5002F01D278050BD0AE2264A19E
:104EE00069A005F075FC6CA005F072FC02F07FF87B
:104EF000022049E7B5F5006F0BD9B4225CA162A08E
:104F000005F066FC64A005F063FC02F070F8022076
:104F10003AE7352002F083FA384602F095F8042883
:104F20001BD0BB2252A158A005F052FC5AA005F09C
:104F30004FFC12E00A20FFF791FD0A2C0BD9C22288
:104F40004BA151A005F044FC53A005F041FC02F038
:104F500042F8022018E7641CA4B2012002F050FAC3
:104F60000128E7D023E0202002F059FA3078717848
:104F7000B61C40EA0121384602F036F9002410E060
:104F80000A20FFF76BFD1E2C09D9D32238A13EA0C1
:104F900005F01EFC40A005F01BFC0220F4E6641C9A
:104FA000A4B2202002F02CFA0128E9D1BF1C6D1E0A
:104FB000ADB2D8D202F01BF80320E5E62DE9F047A8
:104FC0008146884600260024002702F0010000EBFD
:104FD0005205212000F046FB01280AD0F12224A12D
:104FE00029A005F0F5FB2CA005F0F2FB0220BDE89E
:104FF000F08701F0F0FF352002F011FA12E00A20EC
:10500000FFF72CFD0A2C0BD9FB2219A11EA005F0DD
:10501000DFFB21A005F0DCFB01F0DDFF0220E6E76D
:10502000641CA4B2012002F0EBF90128E7D018E0DB
:10503000202002F0F4F9701C18F8061080B2421C0F
:1050400018F8000096B241EA002A09EB070460054F
:1050500002D1204601F0F8FF2046514602F0C4F884
:10506000BF1C6D1EADB2E3D201F0C1FF0320BEE74D
:105070002E2E5C53595354454D5C464C4153485C6D
:10508000666C6173682E63004C6F674572723A20DC
:1050900025732C25640000000000000010B586B0C8
:1050A00001214FF4017000F0CEFB4FF4004000F0FE
:1050B0004DFB494C204600F0EBFD002101918DF89D
:1050C00008108DF809104FF4602203920491012119
:1050D0008DF8141001A9204600F006FE012000F012
:1050E00065FF0121204600F027FE204600F047FE24
:1050F000204600F049FE0028FAD1204600F04BFE81
:10510000204600F04DFE0028FAD106B010BD10B5C3
:10511000314C014607230122204600F06FFE012199
:10512000204600F044FE0221204600F04DFF0028FA
:10513000F9D02046BDE8104000F0A6BE70B50025AD
:1051400000241020FFF7E3FF284485B20A20FFF770
:1051500085FC641CE4B2052CF3D30520B5FBF0F00C
:1051600070BD2DE9F04107460E460025002408E0F9
:105170003846FFF7CCFF05440A20FFF76FFC641C9C
:10518000E4B2B442F4D3B5FBF6F080B2BDE8F081EE
:1051900010B50A211020FFF7E4FF09F06DF809F0BF
:1051A0003FF84FF066320D4B08F02AFD02460B46E1
:1051B0000B480C4908F04AFF0B4A0C4B08F0C8FAA0
:1051C00000220B4B08F008FA00220A4B08F018FDE9
:1051D00008F052FC00B210BD0024014066664A3F50
:1051E000E17A14AE47E1F63F22FDF675E09C713F8F
:1051F0000000394000005940FEB505460E46012129
:10520000084600F020FB4FF48037019700248DF80A
:1052100008408DF8095001258DF80A5001A800F0CA
:1052200075FF384600F0D1FF8DF800508DF8016011
:105230008DF802408DF80340684600F03EF81B49A7
:1052400002200860C02000F0DBFF012000F0D5FF45
:10525000FEBD3EB50121080700F000FB01248DF8DA
:1052600008408DF8094000258DF80A508DF80B4054
:1052700002A800F022F8684600F07FFF20040090AA
:105280008DF8045008208DF805008DF8064068461A
:1052900000F03CFFC02000F0B3FF012000F0ADFFA4
:1052A0003EBD4FF4803000F090BF000000E100E010
:1052B0002A4908432A490860704770B50F23C2780D
:1052C00001260178002A1ED0254A126802F4E06205
:1052D000C2F5E062120AC2F10404D3404578A54049
:1052E00082781A402A43120101F1E02181F800245A
:1052F000007800F01F018E404009800000F1E0209E
:10530000C0F8006170BD01F01F00864048098000B0
:1053100000F1E020C0F8806170BD124A11400143E5
:105320000F48001F016070470D4A121D002903D06D
:105330001168014311607047116881431160704723
:105340004FF0E021042804D0086920F0040008612F
:105350007047086940F00400086170470000FA05D2
:105360000CED00E080FFFF1F10B59C49884209D179
:105370000121042000F07DFA0021BDE81040042046
:1053800000F077BA9649884209D10121082000F03F
:1053900070FA0021BDE81040082000F06ABA914977
:1053A000884209D10121102000F063FA0021BDE8F4
:1053B0001040102000F05DBA8B49884209D10121CC
:1053C000202000F056FA0021BDE81040202000F017
:1053D00050BA8649884209D10121402000F049FA9B
:1053E0000021BDE81040402000F043BA80498842C7
:1053F00009D10121802000F03CFA0021BDE81040D5
:10540000802000F036BA7B4988420AD184150121F8
:10541000204600F02EFA2046BDE81040002100F0A2
:1054200028BA10BD10B50121084600F022FA00216B
:10543000BDE81040012000F01CBA2DE9F041002227
:10544000CC7804F00F03E40601D58C7823430C7864
:105450004FF00F0714F0FF0F4FF0010C1CD0056840
:105460000CFA02F40E882640A64211D1960007FAE3
:1054700006F825EA080503FA06F848EA0505CE7895
:10548000282E02D0482E02D002E0446100E00461E0
:10549000521C082AE4D305600A88FF2A1ED94568F1
:1054A000002202F108060CFA06F40E882640A642F5
:1054B00010D1960007FA06F825EA080503FA06F85F
:1054C00048EA0505CE78282E00D14461CE78482ED2
:1054D00000D10461521C082AE3D34560BDE8F08185
:1054E0004FF6FF710180022181700421C170704765
:1054F0000246002092680A4200D00120704780686E
:1055000080B2704702460020D2680A4200D00120D3
:105510007047C06880B27047016170474161704751
:10552000002A01D00161704741617047C160704736
:1055300041F4803282618161826181698069704752
:1055400010B52D4B1A684FF68074224042EA0010C5
:105550000843186010BD2949C8617047F0B5264C52
:10556000002801DAE36900E06368C0F30346420DF6
:10557000120185B2C0F301579540032F07D0C20234
:105580000CD50322B240934343F0706209E023F04C
:105590007062636823F07063636002E0AB4343F0C2
:1055A000706201B12A43002801DAE261F0BD626055
:1055B000F0BD10B58A07120F0F23934021F00304AA
:1055C0000D4921448C689C438C608B689040034358
:1055D0008B6010BD0949DC3108607047000801404C
:1055E000000C01400010014000140140001801406F
:1055F000001C01400020014000000140000020424A
:10560000B448016841F0010101604168B24A1140AB
:1056100041600168B14A11400160016821F48021B4
:105620000160416821F4FE0141604FF41F01816077
:105630007047A8490A6822F480320A600A6822F496
:1056400080220A60B0F5803F07D0B0F5802F03D1EB
:10565000086840F4A02008607047086840F4803073
:10566000086070470346002059099A4A01290AD068
:1056700002290AD0516A03F01F02012393400B4212
:1056800000D0012070471168F5E7116AF3E718B5FB
:10569000002000904FF4A0643120FFF7E3FF009951
:1056A000491C00910099A14201D00028F4D031207A
:1056B000FFF7D8FF08B1012018BD002018BD854AAA
:1056C000116821F0F80141EAC00010607047844978
:1056D000086070477F4B5A6822F47C1208431043DD
:1056E000586070477E49086670477A4A516821F0D1
:1056F00003010143516070477648406800F00C0098
:105700007047744A516821F0F001014351607047BD
:10571000704A516821F4E0610143516070476D4A5D
:10572000516821F4605141EAC00050607047694AF5
:10573000002903D0517A014351727047517A814355
:10574000517270476649D83108607047614A5168A4
:1057500021F440410143516070475E4900222031ED
:105760000A7001F82029012805D0042802D105205B
:1057700081F820007047012081F8200070475949C6
:105780000860704753490A6A02430A6270475549E4
:1057900044390860704710B54E4A516801F00C0159
:1057A000514B002927D0042927D0082927D003608E
:1057B000516801F0F00109094C4B5C5C0168E14063
:1057C0004160546804F4E064240A1C5D21FA04F486
:1057D0008460546804F46054E40A1B5DD940C160DD
:1057E000526802F44042920B404B1B1F9A5CB1FB83
:1057F000F2F1016110BD0360DAE70360D8E7516898
:1058000001F47011536803F48033022404EB9141D6
:1058100033B153689B0307D5354B59430160C7E744
:10582000334B59430160C3E72F4B59430160BFE736
:10583000284A002903D051690143516170475169D9
:10584000814351617047234A002903D09169014384
:105850009161704791698143916170471D4A0029A8
:1058600003D0D1690143D1617047D1698143D161CE
:105870007047184A002903D0D1680143D1607047AE
:10588000D1688143D1607047124A002903D0116961
:1058900001431161704711698143116170471149DA
:1058A0004039086070470E49C86470470949C8719B
:1058B00070470848416A41F0807141627047014673
:1058C0000020044A92680A4200D001207047014932
:1058D00088727047001002400000FFF8FFFFF6FEDC
:1058E000000042428004424200127A004406002036
:1058F00000093D0010B5E14988420AD101218C031D
:105900002046FFF7B6FF2046BDE810400021FFF714
:10591000B0BFDB4988420AD101214C042046FFF781
:10592000B3FF2046BDE810400021FFF7ADBFD549C9
:1059300088420AD101218C042046FFF7A5FF2046AA
:10594000BDE810400021FFF79FBFCF4988420AD130
:105950000121CC042046FFF797FF2046BDE8104008
:105960000021FFF791BFC94988420AD101210C05E6
:105970002046FFF789FF2046BDE810400021FFF7D1
:1059800083BF10BD30B585B004460D46208A4CF665
:10599000FF710840E98801432182A0894EF6F31186
:1059A0000840A9882A8911436A8902431143A181C9
:1059B000A08A4FF6FF410840A9890143A1826846A9
:1059C000FFF7E9FEAD48844201D1039800E0029858
:1059D000A189090408D500EBC00101EB001029687A
:1059E0004900B0FBF1F007E000EBC00101EB001053
:1059F00029688900B0FBF1F06422B0FBF2F10901E3
:105A00000B096FF018056B4300EB8300A3891D049D
:105A10004FF0320307D503EBC000B0FBF2F000F00B
:105A20000700084306E003EB0010B0FBF2F000F0C3
:105A30000F000843208105B030BD4FF416510160BE
:105A400000218180C18001810C22428181817047C7
:105A500010B5038A4FF2FF0213400A884C88224394
:105A60008C88C9880C4322431A43028210BD00214E
:105A7000018041808180C1807047002904D08189E4
:105A800041F4005181817047818921F40051818165
:105A9000704710B540F66A13C1F3421301F01F04BA
:105AA0000121A140012B07D0022B07D014303AB1BD
:105AB00002680A43026010BD0C30F8E71030F6E7C8
:105AC00002688A43026010BD002A03D0828A0A431A
:105AD00082827047828A8A4382827047028A22F0D9
:105AE0000F020282028A0A4302827047828922F4EC
:105AF0000062828182890A4382817047002904D032
:105B0000818941F0020181817047818921F0020180
:105B100081817047028A22F020020282028A0A43AF
:105B200002827047002904D0018A41F48041018239
:105B30007047018A21F4804101827047C1F3080156
:105B4000818070478088C0F308007047818941F0E8
:105B5000010181817047028BD2B20283028B42EA3B
:105B6000012101837047028B02F47F420283028B82
:105B70000A4302837047002904D0818A41F0200142
:105B800081827047818A21F020018182704700293B
:105B900004D0818A41F0100181827047818A21F00E
:105BA000100181827047002904D0818A41F00801E8
:105BB00081827047818A21F0080181827047002923
:105BC00004D0818941F40041818170478189C1F30A
:105BD0000E0181817047002904D0818A41F400615F
:105BE00081827047818A21F4006181827047828AB4
:105BF00022F004028282828A0A438282704700294C
:105C000004D0818A41F0020181827047818A21F0AB
:105C10000201818270470246002012880A4200D0A9
:105C2000012070478A05C9430180704770B5002480
:105C300040F66A12C1F3421301F01F05012606FA6D
:105C400005F2012B0CD0022B0DD0838A1340090AD8
:105C50008E40008830400BB100B10124204670BD59
:105C600083891340F3E7038A1340F0E740F66A1292
:105C70000A0A01219140C943018070470038014060
:105C80000044004000480040004C004000500040EC
:105C900010B5DB4988420AD1441501212046FFF79F
:105CA000E8FD2046BDE810400021FFF7E2BDD549E0
:105CB00088420AD1041501212046FFF7DAFD20466B
:105CC000BDE810400021FFF7D4BDCF4988420AD17A
:105CD0000121CC032046FFF7CCFD2046BDE8104053
:105CE0000021FFF7C6BD10BD10B54268C74B1A4072
:105CF0000C790B6842EA0422134343608268C44B68
:105D00001A40D1E9024323434C7942EA4402134347
:105D10008360C26A22F47002097C491EC9B242EA59
:105D20000151C16210BD00210160017141718160AA
:105D3000C160012101747047002904D0816841F0DD
:105D4000010181607047816821F001018160704725
:105D5000002904D0816841F48071816070478168B6
:105D600021F4807181607047C9B2002A03D0426873
:105D70000A434260704742688A43426070478168C4
:105D800041F00801816070470146002089680907D9
:105D900000D501207047816841F00401816070479F
:105DA000014600208968490700D501207047002975
:105DB00004D0816841F4A00181607047816821F4BA
:105DC000A00181607047014600208968490200D522
:105DD00001207047426822F46042491E42EA413184
:105DE00041607047002904D0416841F4006141607E
:105DF0007047416821F400614160704770B5072623
:105E000009290AD9C568A1F10A0404EB4404A64093
:105E1000B543A3401D43C56007E0056901EB41049C
:105E2000A640B543A3401D4305611F23072A09D29D
:105E3000446B521E02EB820293409C4391400C4300
:105E4000446370BD0D2A09D2046BD21F02EB82029B
:105E500093409C4391400C43046370BDC46A0D3A67
:105E600002EB820293409C4391400C43C46270BD9C
:105E7000002904D0816841F48011816070478168F5
:105E800021F4801181607047C06C80B270475C481B
:105E90004C3000687047002904D0416841F48061AB
:105EA00041607047416821F480614160704700297A
:105EB00004D0416841F4805141607047416821F449
:105EC000805141607047826822F4E0420A43826058
:105ED0007047002904D0816841F400418160704717
:105EE000816821F4004181607047002904D08168F5
:105EF00041F4021181607047816821F402118160D0
:105F00007047014600208968890200D5012070474A
:105F100070B5072609290AD9C568A1F10A0404EB5E
:105F20004404A640B543A3401D43C56007E005698E
:105F300001EB4104A640B543A3401D430561836BBB
:105F4000C3F30154121B921C02EB82021F249440E3
:105F5000A34391400B43836370BD826B22F44012D4
:105F6000491E42EA01518163704708B500900098CC
:105F7000084400900098026008BD08B500900098A1
:105F80000844283000900098006880B208BD42683C
:105F9000204B1A400A434260704741628262704758
:105FA000426822F01F020A434260704714490831D8
:105FB000002804D0086840F40000086070470868B2
:105FC00020F40000086070470246002012680A4270
:105FD00000D001207047C9430160704710B50246E8
:105FE00000200B0A5468C9B20C401168194202D053
:105FF000002C00D0012010BD090AC9430160704780
:106000000024014000280140003C0140FFFEF0FF59
:10601000FDF7F1FFFFFD3FFF0D49086070470C4998
:10602000486070470A498860704709494AF6AA20C3
:106030000860704706494CF6CC400860704701463E
:106040000020034AD2680A4200D0012070470000B5
:106050000030004010B50120FFF721FCBDE81040E2
:106060000020FFF71CBC2049086070471E49091F2B
:10607000086070471C498431086070471B4A1188CA
:1060800021F46071014311807047184A118821F092
:106090007F0101431180704708B5144A2C3A10441F
:1060A00000900098016008BD08B510492C390844DB
:1060B00000900098008808BD0B489C300068C0B272
:1060C00070470A480830018841F00101018070479B
:1060D0000548A0300068C0B2704704480830018805
:1060E00041F002010180704704860D422C6C004093
:1060F000384900200860091D0860091D0860091D55
:1061000008603449344814310860704730B5314A6A
:1061100083790168002B2AD013688B431360111D0B
:106120000B680468A3430B60017911440B68046891
:1061300023430B60274C083421680368994321608E
:10614000231D19680568A94319604179102905D0F4
:1061500011440A68006802430A6030BD2168026881
:1061600011432160196800680143196030BD00794E
:10617000104402688A43026030BD00210160017151
:106180000C22427181717047124910310A68024332
:106190000A607047014600200E4A143212680A4213
:1061A00000D0012070470B49143108607047014648
:1061B0000020084A12680A40064B14331B680B4241
:1061C00002D0002A00D00120704702491431086033
:1061D0007047000000040140FFFF0F0010B50121CF
:1061E0000C072046FFF750FB2046BDE81040002179
:1061F000FFF74ABB21490862704720490861704790
:106200001F4A116821F0E0010143116070471B49EA
:10621000A031086070471A4B1A6822F0030202434B
:106220001A601848026842F004020260012905D091
:1062300020BF016821F004010160704730BFF8E71A
:106240000F48016841F004010160016841F002015A
:1062500001600C48016841F00401016030BF7047E3
:1062600001460020064A52680A4200D001207047C9
:1062700003490A6842EA80000860704700000E4245
:106280000070004010ED00E03A4A002903D0118868
:106290000143118070471188814311807047354850
:1062A000001D018841F01001018070473148001D38
:1062B000018821F01001018070472E481C300088B1
:1062C0002C491831098840EA01407047294A010CDD
:1062D00018321180111D08807047264AC0F303410F
:1062E00008321180111D0880E0E7224A010C20329B
:1062F0001180111D088070471E481030008800076B
:10630000010B1C4814300088084370471948001DD1
:1063100001888906FCD570471648001D018821F0C8
:106320000801018001880907FCD57047014600205B
:10633000104A121D12880A4200D0012070470D49F0
:10634000091D0A8882430A8070470A49091D098885
:10635000C2B21140074A1288024202D009B101209C
:106360007047002070470349091D0A8882430A804C
:10637000704700000028004010B5FE4988420AD14D
:10638000C41401212046FFF774FA2046BDE81040EE
:106390000021FFF76EBAB0F1804F0CD0F649884269
:1063A00013D101210220FFF76FFA0021BDE8104050
:1063B0000220FFF769BA01210846FFF765FA0021BC
:1063C000BDE810400120FFF75FBAEC49884209D1CF
:1063D00001210420FFF758FA0021BDE810400420F5
:1063E000FFF752BAE649884209D101210820FFF798
:1063F0004BFA0021BDE810400820FFF745BAE149FB
:10640000884209D101211020FFF73EFA0021BDE8A2
:1064100010401020FFF738BADB49884209D101212A
:106420002020FFF731FA0021BDE810402020FFF7BF
:106430002BBAD64988420AD1441401212046FFF7DD
:1064400018FA2046BDE810400021FFF712BAD049E3
:1064500088420AD10121CC042046FFF70AFA2046DF
:10646000BDE810400021FFF704BACA4988420AD1AA
:1064700001210C052046FFF7FCF92046BDE810403D
:106480000021FFF7F6B9C44988420AD101214C0521
:106490002046FFF7EEF92046BDE810400021FFF747
:1064A000E8B9BE49884209D101214020FFF7ECF943
:1064B0000021BDE810404020FFF7E6B9B849884206
:1064C00009D101218020FFF7DFF90021BDE810404C
:1064D0008020FFF7D9B9B34988420AD18415012138
:1064E0002046FFF7D1F92046BDE810400021FFF714
:1064F000CBB9AD4988420AD101210C042046FFF7EF
:10650000B8F92046BDE810400021FFF7B2B9A7490D
:1065100088420AD101214C042046FFF7AAF92046FF
:10652000BDE810400021FFF7A4B9A14988420AD173
:1065300001218C042046FFF79CF92046BDE810405D
:106540000021FFF796B910BD30B50288894C8F4DF8
:10655000A0420DD0A8420BD0B0F1804F08D0864B9E
:10656000984205D0854B984202D0854B984203D182
:1065700022F070034A881A43824B984206D0824B1D
:10658000984203D022F44073CA881A4302808A8852
:1065900082850A880285A0420AD0A84208D0824A91
:1065A000904205D0814A904202D0814A904201D166
:1065B000097A01860121818230BD30B5028C22F03A
:1065C00001020284028C8388048B24F0700424F07E
:1065D00003050C882C4322F002020D8915434A88DA
:1065E0002A43644DA8420BD0684DA84208D06E4D96
:1065F000A84205D06D4DA84202D06D4DA8420FD1E2
:1066000022F008054A892A4322F004058A882A4391
:1066100023F4807323F400738D891D43CB892B43AE
:1066200083800483C9888186028430BD70B5028C62
:1066300022F010020284028C8388048B24F4E0444C
:1066400024F440760D884FF6FF7404EA052535439F
:1066500022F020020E8904EA061616434A8804EA4C
:1066600002123243434EB04202D0484EB04217D1DC
:1066700022F080024E8904EA0616164326F04006F0
:106680008A8804EA0212324323F4806323F400630D
:106690008E8904EA86061E43CB8904EA83033343CA
:1066A00083800583C9880187028470BD70B5028C20
:1066B00022F480720284028C8388848B24F070041C
:1066C00024F003040D88254322F400720E894FF64E
:1066D000FF7404EA062616434A8804EA022232437B
:1066E000244EB04202D0294EB04217D122F40066A7
:1066F0004A8904EA0222324322F480668A8804EA44
:106700000222324323F4805323F400538E8904EA97
:1067100006161E43CB8904EA031333438380858323
:10672000C9888187028470BD70B5028C22F48052C2
:106730000284058C8288838B23F4E04323F4407623
:106740000C884FF6FF7303EA0424344325F4005504
:106750000E8903EA06362E434D8803EA0535354394
:10676000044EB04202D0094EB04226D122F48046F7
:106770008A891FE0002C014000040040000800400E
:10678000000C0040001000400014004000340140A4
:10679000004C0140005001400054014000180040EE
:1067A000001C004000200040004001400044014027
:1067B0000048014003EA8212324382808483C98800
:1067C000A0F84010058470BD828B22F44062828361
:1067D000828B4FF6FF7303EA01210A4382837047DD
:1067E000F0B5048C24F480540484868B048C4FF61A
:1067F000FF7505EA013726F4734605EA02223243A3
:1068000005EA03331343F74A90420ED0F64A90420A
:106810000BD0B0F1804F08D0F44A904205D0F44A32
:10682000904202D0F34A904205D124F400513943FA
:1068300041F4805104E024F402420A4342F48051BE
:1068400083830184F0BD828B22F00C028283828BD1
:106850000A4382837047F0B5048C24F48074048466
:10686000858B048C4FF6FF7707EA012625F0F305A8
:1068700007EA031313432B43DA4A90420ED0DA4A55
:1068800090420BD0B0F1804F08D0D84A904205D04A
:10689000D74A904202D0D74A904205D124F40071E1
:1068A000314341F4807104E024F420620A4342F44D
:1068B000807183830184F0BD028B22F440620283E5
:1068C000028B4FF6FF7303EA01210A4302837047EC
:1068D000F0B5048C24F010040484068B048C4FF66D
:1068E000FF7505EA011726F4734605EA03333343BF
:1068F00005EA02221A43BB4B98420ED0BA4B98428B
:106900000BD0B0F1804F08D0B84B984205D0B84BAF
:10691000984202D0B74B984205D124F02001394368
:1069200041F0100104E024F0A0030B4343F01001F8
:1069300002830184F0BD028B22F00C020283028BE1
:106940000A430283704770B5048C24F00104048468
:10695000058B048C25F0F3054FF6FF7606EA03134A
:1069600013432B439F4A90420ED09F4A90420BD034
:10697000B0F1804F08D09D4A904205D09C4A904289
:1069800002D09C4A904205D124F002020A4342F010
:10699000010104E024F00A020A4342F001010383EA
:1069A000018470BD70B505460C468E48854209D0FD
:1069B0008D48854206D0B5F1804F03D08B48854283
:1069C00000D08B4820886188A288238958B1042888
:1069D00011D0082817D02846FFF702FFE188284683
:1069E000BDE87040F0E62846FFF7ADFFE188284695
:1069F000BDE870409FE72846FFF76AFFE188284618
:106A0000BDE8704058E72846FFF725FFE188284693
:106A1000BDE8704017E72DE9F04107460C46002518
:106A200001266188002900D10225A288012A00D10F
:106A300002262088238988B13846FFF749FFE1887C
:106A40003846FFF739FF2389324629463846FFF793
:106A50007AFFE1883846BDE8F0416CE73846FFF739
:106A600072FFE1883846FFF766FF238932462946E0
:106A70003846FFF72DFFE1883846BDE8F0411BE7B7
:106A800010B50A884B88CC881A438B8823431A4355
:106A90000B891A434B8989891A430A43A0F8442079
:106AA00010BD4FF6FF71818000210180C1804180BF
:106AB000017270470021018041808180C180018185
:106AC00041818181C1817047002101804180012283
:106AD0008280C180018170470021018041808180D6
:106AE000C1800181418181817047002904D00188E2
:106AF00041F0010101807047018821F0010101800E
:106B00007047002905D030F8441F41F4004101804E
:106B1000704730F8441FC1F30E0101807047002A0E
:106B200003D082890A438281704782898A438281A5
:106B30007047818270471143A0F848107047002ABF
:106B400003D082890A438281704782898A43828185
:106B50007047018921F0070101817047028922F005
:106B600070020A430281704700B503461846FFF7DA
:106B7000F5FF188940F00700188100BD70B50D467B
:106B800004461146602D0CD001222046FFF7DBFEA3
:106B900029462046FFF7E2FF208940F007002081C8
:106BA00070BD01222046FFF793FEF1E730B504895E
:106BB000E4B24FF6FF7505EA032313430B43234367
:106BC000038130BD10B504462046FFF7EFFF208952
:106BD00020F0070040F0070020F0700040F0700047
:106BE000208110BD002C0140003401400004004011
:106BF00000080040000C004010B504462046FFF796
:106C0000D5FF208940F480402081EAE70185828217
:106C10007047028822F070020A430280704770B504
:106C20000589048B068C25F007050D434FF6FC41C2
:106C30000C4040F201110C4326F022064FF6FF7182
:106C400001EA03111143314305810483018470BDBE
:106C5000028B22F070020A4302837047028B22F4F7
:106C6000E0424FF6FF7303EA0121114301837047AD
:106C7000828B22F070020A4382837047828B22F457
:106C8000E0424FF6FF7303EA01211143818370470D
:106C9000002904D0018841F08001018070470188FB
:106CA00021F0800101807047002904D0818841F0E3
:106CB000040181807047818821F004018180704740
:106CC000002904D0818841F00801818070478188C3
:106CD00021F0080181807047002904D0818841F0AB
:106CE000010181807047818821F001018180704716
:106CF000028B22F008020A4302837047028B22F4BF
:106D000000624FF6FF7303EA0121114301837047CC
:106D1000828B22F008020A4382837047828B22F41E
:106D200000624FF6FF7303EA01211143818370472C
:106D3000028B22F004020A4302837047028B22F482
:106D400080624FF6FF7303EA01211143018370470C
:106D5000828B22F004020A4382837047828B22F4E2
:106D600080624FF6FF7303EA01211143818370476C
:106D7000028B22F080020A4302837047028BC2F327
:106D80000E024FF6FF7303EA01211143018370479E
:106D9000828B22F080020A4382837047828BC2F387
:106DA0000E024FF6FF7303EA0121114381837047FE
:106DB000028C22F002020A4302847047028C22F005
:106DC00008020A4302847047028C22F020024FF628
:106DD000FF7303EA0111114301847047028C22F012
:106DE00080024FF6FF7303EA0111114301847047DB
:106DF000028C22F400724FF6FF7303EA0121114363
:106E000001847047028C22F400624FF6FF7303EA9C
:106E10000121114301847047028C22F400524FF685
:106E2000FF7303EA013111430184704710B5012358
:106E30008B40048C9C430484038C8A40134303845A
:106E4000CFE610B504238B40048C9C430484038C50
:106E50008A4013430384C4E630B500F118030124CB
:106E60008C40058CA5430584002911D008290FD03A
:106E7000091FC1F34E001844016821F4E04101608C
:106E800001684FF6FF7303EA02221143016030BD2F
:106E900003EB5100016821F07001016001681143AA
:106EA000016030BD002904D0018841F00201018059
:106EB0007047018821F0020101807047002904D049
:106EC000018841F0040101807047018821F004012C
:106ED00001807047002904D0818841F080018180C1
:106EE0007047818821F0800181807047028822F0FC
:106EF0000802028002880A4302807047828822F0DA
:106F00007002828082880A4382807047028922F060
:106F10000702028102890A4302817047028922F036
:106F20008002028102890A4302817047818470478E
:106F300081857047818670470187704781877047D8
:106F4000A0F840107047028822F440720280028844
:106F50000A4302807047808E7047008F7047808F91
:106F60007047B0F840007047808C7047008D7047C4
:106F700002460020128A0A4200D001207047C9430D
:106F80000182704702460020138A0B4092890A4012
:106F9000002B02D0002A00D001207047C943018293
:106FA00070470000FE4A116801F03801014311608A
:106FB0007047FB490A6822F008020A600A68024327
:106FC0000A607047F6490A6822F010020A600A68EF
:106FD00002430A607047F248F2494160F249416059
:106FE0007047EF48EF494160EF4941607047EC4816
:106FF000016941F0800101617047E948016941F090
:107000008001016170470420E549CA68D20701D0B8
:1070100001207047CA68520701D502207047C9682D
:10702000C906FBD50320704700B50346FFF7EBFF09
:1070300002E0FFF7E8FF5B1E012801D1002BF8D129
:10704000002B00D1052000BD70B505464FF4302659
:107050003046FFF7E9FF042811D1D14C206940F0F8
:10706000020020616561206940F0400020613046E7
:10707000FFF7DAFF216941F6FD721140216170BD11
:1070800030B54FF430252846FFF7CEFF042810D145
:10709000C34C206940F004002061206940F04000AA
:1070A00020612846FFF7C0FF216941F6FB721140BD
:1070B000216130BD00B50346FFF7A5FF02E0FFF7F1
:1070C000A2FF5B1E012801D1002BF8D1002B00D1BB
:1070D000052000BD30B54FF430252846FFF7EAFF04
:1070E000042810D1AE4C206940F0040020612069D2
:1070F00040F0400020612846FFF7DCFF216941F69F
:10710000FB721140216130BD0020A549C969890782
:1071100000D50120704770B5A525FFF7F5FF00B138
:1071200000254FF430263046FFF77EFF042818D1A3
:107130009B4C9C48A0609C48A060206940F02000C7
:107140002061206940F0400020613046FFF76CFF6D
:1071500041F6EF76042805D0052802D02169314098
:10716000216170BD206941F6DF710840206120690E
:1071700040F0100020618D4805804FF40050FFF76B
:1071800053FF0528EDD021693140216170BD2DE903
:10719000F84105460E46002000904FF4005738464F
:1071A000FFF742FF04280FD17D4C206940F0010019
:1071B00020612E80B8464046FFF736FFBF1E0428E8
:1071C00004D0216939402161BDE8F881AD1C0095EA
:1071D0000099300C08804046FFF726FF21693940AE
:1071E0002161F1E700887047F0B506460D464FF47F
:1071F00000573846FFF718FF04280CD1684C206967
:1072000040F00100206135803846FFF70DFF21690D
:10721000BA1E11402161F0BDF0B505460E464FF48F
:1072200000573846FFF700FF042813D15C4C5D4837
:10723000A0605D48A060206940F0100020612E80B1
:107240003846FFF7F1FE052804D0216941F6EF72B8
:1072500011402161F0BD2DE9F043C043C4B2C0F339
:107260000725C0F30746070E4FF400594846FFF7BD
:10727000DBFE04283CD1DFF828814A49C8F8081011
:107280004949C8F80810D8F8101041F01001C8F8A2
:107290001010FF2C05D04548083004804846FFF701
:1072A000C3FE042807D1FF2D05D040480A300580D1
:1072B0004846FFF7B9FE042807D1FF2E05D03B480A
:1072C0000C3006804846FFF7AFFE042807D1FF2F99
:1072D00005D036480E3007804846FFF7A5FE052842
:1072E00006D0D8F8101041F6EF721140C8F810100F
:1072F000BDE8F08370B505464FF430263046FFF701
:1073000093FE042818D1264C2648A0602648A06089
:10731000206940F020002061206940F04000206199
:107320003046FFF781FE41F6DF71042805D00528BD
:1073300002D022690A40226170BD206908402061A4
:10734000206940F010002061184815B1002101802B
:1073500001E0A52101803046FFF766FE0528EBD04D
:10736000216941F6EF721140216170BD2DE9F041B4
:1073700006460D4617460A4C0A48A0600A48A06017
:107380004FF400584046FFF74FFE04281DD12069F6
:1073900040F0100020613D43354345F0F80007E020
:1073A0000020024023016745AB89EFCD00F8FF1FA5
:1073B0002549891C08804046FFF736FE052804D081
:1073C000216941F6EF7211402161BDE8F0811F484B
:1073D000C069800870471D48006A704700201B493B
:1073E0000968890600D501207047184A002903D092
:1073F000116901431161704711698143116170473F
:1074000001460020114A012904D0D2680A4200D066
:1074100001207047D169C907FBD0012070470B4993
:10742000C860704704200949CA68D20701D001200A
:107430007047CA68520701D502207047C968C9065B
:10744000FBD503207047000000F8FF1F002002401A
:1074500001684FF6FE721140016000210160416039
:107460008160C1607249724A0839904204D148680B
:1074700040F00F00486070476D4A1432904204D1CA
:10748000486840F0F00048607047694A28329042EE
:1074900004D1486840F4706048607047644A3C32E8
:1074A000904204D1486840F4704048607047604A98
:1074B0005032904204D1486840F4702048607047D0
:1074C0005B4A6432904204D1486840F470004860DE
:1074D0007047574A7832904204D1486840F0706053
:1074E00048607047534A111F904204D1086840F029
:1074F0000F00086070474F4A1432904204D1086868
:1075000040F0F000086070474A4A2832904204D1A7
:10751000086840F4706008607047464A3C32904208
:1075200004D1086840F4704008607047414A503206
:107530009042FAD1086840F470200860704730B576
:10754000026847F6F0739A430C6A8B682343D1E9CB
:1075500004452C4323438C692343CC6923434C6A61
:1075600023438C6A234313430360CA6842600A685A
:1075700082604968C16030BD002101604160816066
:10758000C160016141618161C161016241628162E9
:107590007047002904D0016841F001010160704783
:1075A00001684FF6FE72114001607047002A03D057
:1075B00002680A430260704702688A4302607047AB
:1075C00041607047406880B2704702460020D10099
:1075D00003D518490839096802E0154908390968CE
:1075E000114200D001207047C10003D51149091F85
:1075F000086070470E49083948607047024600200D
:10760000D10003D50B490839096802E00849083957
:107610000968114200D001207047C10003D5054917
:10762000091F086070470249083948607047000028
:1076300008000240080402407047162205A10FA06E
:1076400003F0C6F811A003F0C3F8FEE7FEE7FEE77B
:10765000FEE770472E2E5C53544D3332463130785E
:107660005F46574C69625C7372635C73746D33324E
:10767000663130785F69742E630000004C6F674597
:1076800072723A2025732C256400000048617264F0
:107690004661756C745F48616E646C6572210000B0
:1076A00071B65A4801685A4A01F4E0611143016019
:1076B000BFF34F8FFEE70CB50022019200925548B0
:1076C000016841F4803101604FF4A063016801F466
:1076D000003100910199491C0191009911B901995A
:1076E0009942F3D10168890302D50121009100E09C
:1076F00000920099012930D147490A6842F01002EE
:107700000A600A6822F003020A600A6842F0020274
:107710000A604168416041684160416841F48061AC
:107720004160416821F47C114160416841F4E811F5
:107730004160016841F08071016001688901FCD5F8
:10774000416821F003014160416841F0020141605C
:107750004168C1F381010229FAD10CBDABE710B534
:107760002C48016841F00101016041682B4A114039
:10777000416001682A4A11400160016821F48021BA
:107780000160416821F4FE0141604FF41F018160F6
:10779000FFF7E4FF1D494FF00060091F086010BDAE
:1077A00010B51C4A506800F00C011E4B1E48002901
:1077B0000ED004290ED008290ED0036051681A4A51
:1077C000C1F30311121D515C0268CA40026010BD72
:1077D0000360F3E70360F1E7516801F47011536847
:1077E00003F48033022404EB914133B153689B03CB
:1077F00007D50E4B59430160E0E70C4B594301603C
:10780000DCE7084B59430160D8E700000CED00E0CD
:107810000400FA0500100240002002400000FFF8BA
:10782000FFFFF6FE00127A005406002000093D001A
:1078300010B5A94988420AD1841401212046FEF7D7
:1078400018F82046BDE810400021FEF712B8A34901
:1078500088420AD1041401212046FEF715F820467B
:10786000BDE810400021FEF70FB89D4988420AD1BB
:10787000C41301212046FEF707F82046BDE810405A
:107880000021FEF701B810BD30B5028802F4415363
:107890000A884C88CD8822438C882C4322430C894B
:1078A00022434C8922438C892243CC8922431A43A8
:1078B0000280828B22F400628283098A018230BDB9
:1078C000F0B585B005460C46022000210126AA8BA2
:1078D0004FF240031A40AA8302222A84AF8BA26887
:1078E000022A21D0A08800B102266846FDF753FF86
:1078F0000098E188B1F5007F2CD07101B0FBF1F068
:1079000000EB8000A1684000B0FBF1F0401D80B2A8
:107910000A21B0FBF1F000F00101401AC0F34F0062
:107920004FF6FF7202EA0121821EFE2A01D30220D5
:107930000021E288084302432A8420886188A289C2
:107940000843A18811430843384340F40060A883EA
:1079500005B0F0BD000A00EB8000A1684000B0FB5C
:10796000F1F0401D80B2D3E7002101804180818089
:10797000C180018141818181C181072101827047DC
:107980000021018041808180C1800222826081814A
:107990007047002904D0018841F040010180704700
:1079A000018821F0400101807047002904D0818BBB
:1079B00041F4806181837047818B21F480618183F0
:1079C0007047090901238B4099B2002A03D08288AD
:1079D0000A438280704782888A4382807047002AE7
:1079E00003D082880A438280704782888A438280DB
:1079F00070478181704780897047A1F57E42FF3AC8
:107A000004D0018841F4807101807047018821F41D
:107A1000807101807047002904D0818841F0040101
:107A200081807047818821F004018180704702883D
:107A300022F40062028002880A43028070470188B3
:107A400041F4805101807047002904D0018841F43D
:107A5000005101807047018821F400510180704776
:107A6000012901D0008B7047808A7047008A7047D7
:107A7000B1F5804F04D0018821F480410180704726
:107A8000018841F48041018070470246002012893C
:107A90000A4200D001207047C9430181704730B5C8
:107AA0000246002001F00F03012505FA03F4A3B2FA
:107AB000090905FA01F4A4B29188214012891A42F9
:107AC00002D0002900D0012030BD01F00F020121B9
:107AD0009140C943018170470030014000380040A7
:107AE000003C004030B5744900E011460A6882420B
:107AF000FBD34B685C18844203D14068184448604B
:107B000008460D6844682318AB420DD16A4B103B00
:107B10001B689A4206D05268224442600A68126882
:107B2000026002E0036000E00260814200D0086071
:107B300030BD4FF4B0416148420706D0C01D20F06F
:107B400007005E49411AC1F5B0415B4A106000234D
:107B500053600144083921F00701103A11604B606D
:107B60000B600B1A436001604068906050604FF0FA
:107B70000040D06070472DE9F0410546002601F035
:107B8000A4FB4D4F103F386808B9FFF7D2FFF868E3
:107B900005424AD175B1083568070BD005F00700DA
:107BA000C0F108000544680704D0C02244A14EA0DB
:107BB00002F00EFE002D38D07868854235D83E4957
:107BC0000846046801E0214604466068A84202D2E3
:107BD00020680028F7D13868844226D00E6808361D
:107BE000206808606068401B102811D904EB050864
:107BF0005FEA487004D0ED2231A13BA002F0E8FD1D
:107C00006068401BC8F8040065604046FFF76AFFE3
:107C100061687868401A7860BA68904200D2B860AB
:107C2000F868014361600020206001F0A2FA70074B
:107C300005D040F22D1222A12BA002F0C9FD304642
:107C4000BDE8F08170B500282BD0083804461A4DE5
:107C50006068103DE968084205D14FF4A27218A18E
:107C600021A002F0B5FD206828B140F2451214A110
:107C70001DA002F0ADFD6068E968084211D02268DD
:107C8000002A0ED18843606001F01FFB60686968BC
:107C9000084468602046FFF725FFBDE8704001F00A
:107CA00068BA70BD04481038406870470248103800
:107CB000806870477047000078060020305C002024
:107CC0002E2E5C4672656552544F535C706F727411
:107CD00061626C655C4D656D4D616E675C68656188
:107CE000705F342E630000004572726F723A257324
:107CF0002C25640D0A00000066484068401C04D032
:107D0000F52265A16FA002F063FD502080F3118879
:107D1000BFF34F8FBFF36F8FFEE720384FF08073B4
:107D2000C36121F0010181616A49416140F8202964
:107D30007047694864210068B0FBF1F14FF0E02022
:107D4000491E41610721016170471CB563490878EC
:107D50000190FF200870087800909DF800004D4ABF
:107D600000F0500010700720906006E09068401E00
:107D700090609DF80000400000909DF80000000613
:107D8000F4D4107A000200F4E0609060019808706A
:107D90005348016841F470010160016841F070418D
:107DA0000160FFF7C6FF00205060F4F797FA00204B
:107DB0001CBD38484068B0F57A7F05D04FF4B872E2
:107DC00035A140A002F004BD7047502080F3118817
:107DD000BFF34F8FBFF36F8F2E494868401C486038
:107DE00001280BD13E481C38006810F0FF0F05D069
:107DF0004FF4C07228A133A002F0EABC704710B55E
:107E0000244C6068002805D140F2871222A12DA0E1
:107E100002F0DEFC6068401E6060002801D180F343
:107E2000118810BD10B5502080F31188BFF34F8F1B
:107E3000BFF36F8F01F03DF920B129494FF0805019
:107E40001C390860002080F3118810BD10B5F4F7CC
:107E50007BFA104C10280CD300F1E02090F8F003CE
:107E60002178884205D240F2AE220BA115A002F083
:107E7000AFFC1B4814380068A16800F4E060884239
:107E800007D9BDE8104040F2BE2203A10DA002F0C8
:107E90009FBC10BD800600202E2E5C467265655288
:107EA000544F535C706F727461626C655C525644DF
:107EB000535C41524D5F434D335C706F72742E635F
:107EC000000000004572726F723A25732C25640D14
:107ED0000A000000F97C04085406002000E400E0D9
:107EE00020ED00E010B51C20FFF745FE044624B14C
:107EF00000202060201D00F0A5F9204610BD2DE9CE
:107F0000F041884600250446002805D140F21D2294
:107F1000C0A1C7A002F05CFC5FEA186005D040F287
:107F20001E22BCA1C2A002F053FC261D06F10807C8
:107F300001F0CBF9F068216841EA0801216020E0F6
:107F400046680168002201F07F4321F07F415FEA2B
:107F5000431C06D4D4F800C01CEA010F07D001224C
:107F600005E0D4F800C031EA0C0C00D101223AB18E
:107F7000DA0100D50D43216841F0007101F0D8FD10
:107F80003046B842DCD12068A843206001F0F1F807
:107F90002068BDE8F0812DE9F04104468846154689
:107FA0001F46280E04D0D7229AA1A1A002F010FCEF
:107FB00025B9D82297A19EA002F00AFC01F04EFE3E
:107FC00028B927B1DB2293A199A002F001FC01F0AE
:107FD0007CF9266841462046FFF791FF46EA0806ED
:107FE00035EA060008D067B145F0A0613A46201D89
:107FF00001F012FD002605E02068A843206000275C
:1080000000E0266801F0B5F8D7B138B98C494FF0D7
:1080100080500860BFF34F8FBFF36F8F01F017FFE1
:108020000646B0010AD4FFF7D0FE266835EA0600FE
:1080300002D126EA05002060FFF7E1FE26F07F4628
:108040003046A6E703460020002A03D0994300D11A
:10805000012070470B42FCD0012070472DE9F0470A
:108060000D46089F9046994604460026002805D1F3
:1080700040F24D1267A16EA002F0AAFB280E05D0B7
:108080004FF4A77263A16AA002F0A2FB2DB940F2DF
:108090004F1260A166A002F09BFB01F0DFFD30B93A
:1080A0002FB14FF4A9725BA161A002F091FB01F026
:1080B0000CF9D4F800A04A4629465046FFF7C2FF03
:1080C00040B156460027B8F1000F15D02068A843EC
:1080D000206011E0AFB1B8F1000F01D04FF0807611
:1080E000B9F1000F01D046F0806645EA06013A4634
:1080F000201D01F091FC002601F03BF81FB310B1E8
:1081000009E05646F8E74E494FF080500860BFF34B
:108110004F8FBFF36F8F01F09AFE0646B00110D467
:10812000FFF753FE26684A4629463046FFF78AFF86
:1081300028B1B8F1000F02D02068A8432060FFF7F3
:108140005EFE26F07F463046BDE8F08770B50E46ED
:108150000446002805D140F2DF122EA134A002F01F
:1081600037FB300E05D04FF4F0722AA130A002F098
:108170002FFBFFF72AFE256825EA06002060FFF79F
:108180003EFE284670BDE1E70A4600230146AFF2F5
:10819000090002F0C1BA5022EFF3118182F3118875
:1081A000BFF34F8FBFF36F8F006881F31188704763
:1081B0002DE9F0410646341D01F087F804F1080569
:1081C00040F27D274FF000780BE0E068A84204D130
:1081D0003A4610A116A002F0FBFA4146E06801F011
:1081E000A7FC20680028F0D13046FFF72BFDBDE842
:1081F000F04100F0BEBF82E613460A460146AFF2E8
:10820000090002F089BA002801D080697047002077
:10821000704700002E2E5C4672656552544F535CC9
:108220006576656E745F67726F7570732E6300009C
:108230004572726F723A25732C25640D0A00000096
:1082400004ED00E000F1080141604FF0FF32826070
:10825000C160016100210160704700210161704728
:1082600042684A6093688B609368596091600861C6
:108270000168491C0160704730B50C68621C02D06F
:1082800000F1080202E0026904E01A4653681D6822
:10829000A542FAD953684B6099608A6051600861C1
:1082A0000168491C016030BD0169D0E901329A6062
:1082B000D0E901235A604A68824201D182684A604B
:1082C000002202610868401E0860704770B50446CD
:1082D0000D46002C05D140F21B12F3A1F7A002F0CD
:1082E00077FAFFF772FDD4E90F20216802FB001135
:1082F00061600021A1632168A160E06B2268216CAC
:10830000401E00FB0121E1604FF0FF3084F8440083
:1083100084F8450004F110004DB1FFF793FF04F11C
:108320002400FFF78FFFFFF76AFD012070BD216970
:108330000029F8D001F0C5FB0028F4D0E3494FF044
:1083400080500860BFF34F8FBFF36F8FEBE770B5BE
:108350001D46049C00290BD02260E06321640121AA
:108360002046FFF7B3FF84F850500020A06470BD92
:108370002460F2E7F8B505460E461746002D05D1F4
:108380004FF4C472C8A1CDA002F022FA86B105FB59
:1083900006F05430FFF7EFFB04463CB104F1540201
:1083A0003B46314628460094FFF7D1FF2046F8BDF2
:1083B0000020EEE72DE9F041044617460026A56BA4
:1083C000226C002A10D0C7B1E06802F08FFDE1688E
:1083D000206C091AE1602268914202D26168081A91
:1083E000E060022F16D017E02068A8B9606801F09D
:1083F00080FC0646002060600EE0A06802F076FD7A
:10840000216CA0680844A0606168884204D3206899
:10841000A06001E005B16D1E6D1CA5633046BDE88E
:10842000F0812DE9F3410F460098846C0026002C62
:1084300005D140F6CE129CA1A0A002F0C9F9A06B14
:10844000E16B884205D340F6CF1297A19BA002F0C2
:10845000BFF9A06BE16B88420CD294F945503A46C3
:1084600069462046FFF7A6FF0646681C05D06D1C2E
:1084700084F845503046BDE8FC81606A0028F9D098
:1084800004F1240001F01DFB0028F3D00126F1E7E0
:108490002DE9F0410446FFF798FC94F9455004F1AA
:1084A000240613E0A06C38B100212046FFF7B9FF85
:1084B00050B101F0C2FB07E0606A48B1304601F0FC
:1084C00000FB08B101F0B9FB6D1E6DB2002DE9DCB7
:1084D0004FF0FF3684F84560FFF791FCFFF775FC1D
:1084E00094F9445004F1100709E0206948B1384676
:1084F00001F0E7FA08B101F0A0FB6D1E6DB2002D8E
:10850000F3DC84F84460BDE8F041FFF778BC10B5B7
:108510000446FFF75AFCA06BE16B884201D10124AD
:1085200000E00024FFF76BFC204610BD2DE9FF475B
:1085300082B004468A4698460025002C05D140F2B8
:10854000D92259A15DA002F043F9BAF1000F07D179
:10855000206C28B140F2DA2253A158A002F038F979
:10856000B8F1020F08D1E06B012805D040F2DB2200
:108570004DA152A002F02CF901F070FB38B904981B
:1085800028B140F2DE2248A14CA002F021F94FF0C0
:1085900000094FF080564D4FFFF717FCA06BE16BC1
:1085A000884206D3B8F1020F03D0049860B37DB3BC
:1085B00033E0424651462046FFF7FCFEA16C51B124
:1085C00041462046FFF72DFFC0B13E60BFF34F8FFD
:1085D000BFF36F8F12E0616A51B104F1240001F022
:1085E00070FA58B13E60BFF34F8FBFF36F8F05E055
:1085F00020B13E60BFF34F8FBFF36F8FFFF7FFFBDC
:10860000012006B0BDE8F087FFF7F9FB0020F8E78E
:10861000FFE7684601F0C7FA0125FFF7F0FB00F01D
:1086200054FEFFF7D2FB94F94400401C01D184F8BA
:10863000449094F94500401C01D184F84590FFF71F
:10864000DEFB04A9684601F0C0FA30B12046FFF70E
:108650001FFF00F08EFD0020D3E72046FFF757FFF5
:1086600088B104F11000049901F0BEF92046FFF72B
:108670000FFF00F07EFD00288ED13E60BFF34F8FCC
:10868000BFF36F8F88E72046FFF702FF00F071FD10
:1086900082E700281CD0002141600160C1600023F6
:1086A0001A46194642E700002E2E5C467265655256
:1086B000544F535C71756575652E63004572726F1A
:1086C000723A25732C25640D0A00000004ED00E0C9
:1086D000704710B5024600210120FFF74BFE04460B
:1086E0002046FFF7D6FF204610BD10B50446002CEB
:1086F00007D140F24122AFF25001AFF2400002F048
:1087000067F801F0A8FA616888420BD1E068401E62
:10871000E06028B900231A4619462046FFF706FFF5
:10872000012010BD002010BD10B50446FFF74DFB21
:10873000A06B20B10024FFF762FB204610BD01248E
:10874000F9E730B40B46026C002A0CD0C168114422
:10875000C1604468A14201D30168C160C16830BCF6
:10876000184602F0C3BB30BC70472DE9FF4F83B001
:1087700004468A469B460026002C07D140F2DC4284
:10878000AFF2DC01AFF2CC0002F022F8BAF1000F38
:1087900009D1206C38B140F2DD42AFF2F401AFF202
:1087A000E40002F015F801F059FA48B9059838B11B
:1087B0004FF49C62AFF21011AFF2001002F008F813
:1087C0004FF000094FF08057DFF85486FFF7FDFAAD
:1087D000A56B95B3E66851462046FFF7B2FFBBF1A3
:1087E000000F13D0E660606A50B104F1240001F07C
:1087F00068F928B1C8F80070BFF34F8FBFF36F8FCF
:10880000FFF7FDFA012007B0BDE8F08F6D1EA563EC
:10881000206810B901F025FB606020690028EFD0C6
:1088200004F1100001F04DF90028E9D0C8F80070FB
:10883000BFF34F8FBFF36F8FE2E7FFE7059808B1F3
:1088400026B107E0FFF7DBFA0020DCE701A801F022
:10885000AAF90126FFF7D3FA00F037FDFFF7B5FAC2
:1088600094F94400401C01D184F8449094F94500E7
:10887000401C01D184F84590FFF7C1FA05A901A871
:1088800001F0A3F958B12046FFF702FE00F071FC99
:108890002046FFF749FF002898D00020B3E7204684
:1088A000FFF742FFE0B1206830B9FFF78EFA606849
:1088B00001F0E0F9FFF7A3FA04F12400059901F0B3
:1088C00093F82046FFF7E4FD00F053FC00287FF406
:1088D0007DAFC8F80070BFF34F8FBFF36F8F75E7A0
:1088E0002046FFF7D5FD00F044FC6FE770B5044665
:1088F0000D46002C07D14FF41E72AFF25421AFF297
:10890000442001F065FF01F0A6F96368984204D1A4
:10891000E068401CE060012070BD00232A46194633
:108920002046FFF722FF0028F6D0E168491CE160ED
:1089300070BD70B505460C46002D07D140F2BD2232
:10894000AFF29C21AFF28C2001F042FFAC4207D97C
:1089500040F2BE22AFF2B021AFF2A02001F038FF0A
:10896000022200212846FFF705FD002800D084637D
:1089700070BD2DE9F0470446894615469846002CFF
:1089800007D140F29F32AFF2E021AFF2D02001F0E8
:108990001FFFB9F1000F09D1206C38B14FF4687294
:1089A000AFF2FC21AFF2EC2001F012FFB8F1020FA0
:1089B0000AD1E06B012807D040F2A132AFF21831A2
:1089C000AFF2083001F004FFFFF740FA5020EFF358
:1089D000118780F31188BFF34F8FBFF36F8FA06BA8
:1089E000E16B884206D3B8F1020F03D0002087F371
:1089F000118807E694F94560424649462046FFF74C
:108A0000D9FC701C04D0761C84F845600120EEE788
:108A1000A06C012648B141462046FFF702FD002820
:108A2000F4D0002DF2D02E60F0E7606A0028EDD07F
:108A300004F1240001F045F80028E7D0002DE5D02E
:108A40002E60E3E72DE9F04104460D46002C07D1E6
:108A500040F23C42AFF2B031AFF2A03001F0B8FECC
:108A6000206C38B14FF48862AFF2C431AFF2B43049
:108A700001F0AEFE206848B9606838B140F2454266
:108A8000AFF2DC31AFF2CC3001F0A2FEFFF7DEF93D
:108A90005020EFF3118680F31188BFF34F8FBFF39F
:108AA0006F8FA16BE06B884224D994F94500491C73
:108AB000A163411C04D0401C84F8450001201AE049
:108AC000A06C012748B100212046FFF7AAFC00282E
:108AD000F4D0002DF2D02F60F0E7606A0028EDD0CE
:108AE00004F1240000F0EDFF0028E7D0002DE5D0D0
:108AF0002F60E3E7002086F3118890E42DE9F0472A
:108B0000044689469046002C07D14FF4B462AFF278
:108B10006841AFF2584001F05BFEB9F1000F09D196
:108B2000206C38B140F2A152AFF28441AFF27440F0
:108B300001F04EFEFFF78AF95020EFF3118780F322
:108B40001188BFF34F8FBFF36F8FA66BF6B194F907
:108B5000445049462046FFF7F4FD761EA663681C84
:108B600004D06D1C84F84450012010E020690028D6
:108B7000FAD004F1100000F0A4FF0028F4D0B8F1FE
:108B8000000FF1D00120C8F80000EDE7002087F3C6
:108B9000118837E52DE9F04104460F46002C07D136
:108BA00040F2FC52AFF20051AFF2F04001F010FE83
:108BB0004FB9206C38B140F2FD52AFF21451AFF210
:108BC000045001F005FE206C38B940F2FE52AFF2BD
:108BD0002851AFF2185001F0FBFDFFF737F9502094
:108BE000EFF3118580F31188BFF34F8FBFF36F8FC1
:108BF000A06B38B1E66839462046FFF7A2FDE66073
:108C0000012000E0002085F3118808E410B5044637
:108C1000002C07D140F22F62AFF27451AFF26450D2
:108C200001F0D6FDFFF7D1F8A46BFFF7E8F8204676
:108C300010BD10B50446002C07D140F24162AFF2DE
:108C40009851AFF2885001F0C3FDFFF7BEF8D4E9A8
:108C50000E10441AFFF7D3F8204610BD10B5044695
:108C6000002C07D140F25162AFF2C451AFF2B450C0
:108C700001F0AEFDA06B10BD00216A4A02EBC103FA
:108C80005B68834206D1002042F8310002EBC1014B
:108C900048607047491C0829F0D3704710B5044656
:108CA000002C07D140F25D62AFF20461AFF2F450E4
:108CB00001F08EFD2046FFF7DFFF2046BDE81040A3
:108CC000FEF7C0BFC06C7047C164704790F8500099
:108CD000704710B50446002C07D140F29372AFF2F2
:108CE0003861AFF2286001F073FDA06B08B100207D
:108CF00010BD012010BD10B50446002C07D140F274
:108D0000BA72AFF25C61AFF24C6001F061FDA06B32
:108D1000E16B884201D1012010BD002010BD10B5CB
:108D20000022404B53F832401CB1521C082AF9D3A0
:108D300010BD43F8321003EBC201486010BD10B5FE
:108D400000240021374A02EBC1035B68834202D151
:108D500052F8314002E0491C0829F4D3204610BDE6
:108D600070B504460D461646FFF72FF894F94430C7
:108D70004FF000005B1C01D184F8440094F94510C9
:108D8000491C01D184F84500FFF739F8A06B28B9D8
:108D90003246294604F1240000F076FE2046BDE864
:108DA0007040FFF775BB00220421FFF7E3BA70B5EE
:108DB00004460D46FFF709F8A06C08B1002405E051
:108DC000A06B08B1002401E0A5640124FFF717F8A7
:108DD000204670BD10B50446A06C884201D000202A
:108DE00010BDA06B08B1002010BDFEF7EEFF002003
:108DF000A064FFF704F8012010BD08B5002300931C
:108E00000A466946FFF7B1FC009808BD08B5002185
:108E1000009100226946FFF771FE009808BD00002E
:108E200004ED00E030B4002070B50024FE4D04EBEA
:108E3000840005EB8000FFF705FA641C202CF6D3B4
:108E4000FA48FFF7FFF9F9481430FFF7FBF9F74844
:108E50002830FFF7F7F9F5483C30FFF7F3F9F3480E
:108E60005030FFF7EFF9F248F04941631431816364
:108E700070BD70B50446FEF7A8FFED4DA868401C14
:108E8000A860286810B1686938B10CE02C60A86847
:108E9000012808D1FFF7C8FF05E02868E16AC06A29
:108EA000884200D82C60686A401C68626064E06A8E
:108EB00001212A69814011432961DB4900EB8000CF
:108EC00001EB8000211DFFF7CBF9FEF798FF6869E1
:108ED00000280CD02868E16AC06A884207D2D549C8
:108EE0004FF080500860BFF34F8FBFF36F8F70BD9E
:108EF0002DE9F0478146DDE908580A9C0E461746E1
:108F00009A46B900A522206B02F067F8206B7F1EFD
:108F100000EB870020F00707780705D040F22E32DB
:108F2000C5A1CAA001F054FC00202218315C82F8CF
:108F30003410315C11B1401C1028F6D3002684F89F
:108F40004360202D00D31F25E562E5642665201DC2
:108F5000FFF783F904F11800FFF77FF92461C5F1E9
:108F60002000A0616462666584F8586052464946F4
:108F70003846FEF7D2FE2060B8F1000F01D0C8F8E5
:108F80000040BDE8F0872DE9FF5F8146DDE90E78FE
:108F90008A4616469B46B000FEF7EDFD05462800C2
:108FA0000AD05C20FEF7E7FD04460CB1256304E01F
:108FB0002846FEF747FE00E000248CB10020CDE9F2
:108FC0000240CDE900785B46324651464846FFF7FD
:108FD0008FFF2046FFF74DFF012004B0BDE8F09F52
:108FE0004FF0FF30F9E79248416B0968002905D03E
:108FF000416BC968C9684968816270474FF0FF31A9
:109000008162704710B50446206BFEF71BFE2046B8
:10901000BDE81040FEF716BE70B50446FEF7D5FE5B
:10902000834D04B92C68201DFFF73EF958B9E06A5A
:109030007D4A00EB800152F8211021B901218140C5
:10904000286988432861A06A18B104F11800FFF765
:109050002BF9686A401C68622868844208D173480A
:10906000211D3C30FFF7FCF86868401C686007E091
:10907000A868401EA8602046FFF7C4FFFFF7B3FFB3
:10908000FEF7BDFE6869002812D0286884420FD11F
:10909000286B28B14FF48D6267A16CA001F098FB9A
:1090A00064494FF080500860BFF34F8FBFF36F8F5C
:1090B00070BD2DE9F04100265D4F386B002808D0C7
:1090C000B869401CB861F86900B101263046BDE8B6
:1090D000F081FD686D1CFD608DB9786B006828B16A
:1090E00040F6DE1254A159A001F072FB786BB96B07
:1090F0007963B863386A401C3862FFF774FFB86A56
:10910000DFF8248185420DD3786B006838B1786B25
:10911000C068C468606885420ED2B86202E04FF051
:10912000FF30B8623868C06A00EB800058F8200051
:109130000128C8D90126C6E7201DFFF7B5F8A06AA7
:1091400018B104F11800FFF7AFF8E06A01213A699D
:1091500081401143396100EB800008EB8000211D44
:10916000FFF77EF8E06A3968C96A8842CCD30126E5
:10917000CAE72DE9F041002400272D4D286B002877
:1091800005D140F2EC722CA130A001F021FBFEF7DA
:109190001CFE286B401E2863286BE8BBA868D8B368
:1091A000DFF88880012608F128081DE0D8F80C00B7
:1091B000C46804F11800FFF777F8201DFFF774F872
:1091C000E06A2A6906FA00F111432961164900EBA9
:1091D000800001EB8000211DFFF742F8E06A29685A
:1091E000C96A884200D3EE61D8F800000028DDD1BA
:1091F0000CB1FFF7F8FEAC6944B1FFF75AFF00B1BC
:10920000EE61641E002CF8D10020A861E86918B155
:1092100001273807074900E004E00860BFF34F8FDB
:10922000BFF36F8F1AE0000070B40020F0B600208A
:109230008C06002004ED00E02E2E5C46726565521F
:10924000544F535C7461736B732E63004572726F7D
:10925000723A25732C25640D0A000000FEF7CFFD3D
:10926000384634E72DE9F04104460F46FE4EF568D6
:109270003068001DFFF718F838B9306890F82C10E6
:1092800001208840316981433161601C07D137B1C9
:109290003168BDE8F041091DF448FEF7E1BF2C44F8
:1092A00030684460AC4206D23168B06B091DBDE83D
:1092B000F041FEF7E1BF3168706B091DFEF7DCFF7E
:1092C000B06A844200D2B46201E7E748016B491CEE
:1092D000016370472DE9F04105460E460024002D3C
:1092E00007D140F27C42AFF2B001AFF2A00001F032
:1092F0006FFA3EB940F27D42AFF2C401AFF2B40062
:1093000001F066FAD84F386B38B140F27E42AFF2C6
:10931000D801AFF2C80001F05BFAFFF7D6FFFA6898
:109320002B689919934205D98B4208D9914206D9E5
:10933000012404E08B4201D8914200D90124296024
:109340001CB1881A0021FFF78DFFFFF712FF0028DC
:1093500007D1C7494FF080500860BFF34F8FBFF36C
:109360006F8FB4E610B504460020002C12D0BE4822
:10937000006B38B140F2D242AFF24411AFF2341078
:1093800001F026FAFFF7A1FF00212046FFF76AFF50
:10939000FFF7EFFE002807D1B5494FF08050086075
:1093A000BFF34F8FBFF36F8F10BD70B50546002D13
:1093B00007D140F2FE42AFF28011AFF2701001F01F
:1093C00007FAA94E3068854201D1002070BDFEF732
:1093D000FCFC6C69FEF713FD706B844202D0B06B2D
:1093E000844201D1022070BDA048844205D1A86A00
:1093F00008B1022070BD032070BD9C48143884421F
:1094000002D00CB1012070BD042070BD10B504461F
:10941000FEF7DBFC0CB994480468E46AFEF7EFFC45
:10942000204610BD10B50446FEF710FD5020EFF3A6
:10943000118180F31188BFF34F8FBFF36F8F0CB989
:1094400089480468E06A81F3118810BD2DE9F04174
:1094500004460D460026202D07D340F28352AFF27A
:109460002821AFF2182001F0B3F9202D00D31F25D9
:10947000FEF7ABFC7C4F04B93C68E06CA84241D0DD
:10948000854208D939688C4209D03968C96AA9422D
:1094900005D8012603E039688C4200D10126D4F8B2
:1094A0002C80404500D1E562E564A069002802DB1C
:1094B000C5F12000A0616F4D08EB8801606905EBE4
:1094C0008101884215D1201DFEF7EEFE012120B951
:1094D0003A6901FA08F082433A61E06A3A698140E8
:1094E0001143396100EB800005EB8000211DFEF780
:1094F000B7FE3EB15E494FF080500860BFF34F8F1A
:10950000BFF36F8FBDE8F041FEF779BC70B5564DE3
:10951000286B002802D00120E86170BD0020E861BE
:109520002869B0FA80F0C0F11F00524E00EB8004B1
:1095300056F8240038B940F6FF22AFF20431AFF2FA
:10954000F42001F045F906EB840041684968416068
:1095500000F10802914201D1496841604068C06849
:10956000286070BD70B50446FEF72FFC3E4D04B96F
:109570002C68201DFEF798FE58B9E06A3D4A00EBC2
:10958000800152F8211021B90121814028698843C6
:109590002861A06A18B104F11800FEF785FE211DAC
:1095A0003248FEF75DFEFEF72AFC686928B1FEF737
:1095B0000CFCFFF718FDFEF722FC2868844213D14B
:1095C000686990B1286B38B140F25B62AFF29831B4
:1095D000AFF2883001F0FCF825494FF08050086068
:1095E000BFF34F8FBFF36F8F70BD2048A96800682D
:1095F000884202D10020286070BDBDE8704085E738
:1096000070B500250446002807D140F28562AFF20C
:10961000D831AFF2C83001F0DBF8144960698842F4
:1096200005D1A06A2839884201D000B90125284611
:1096300070BD70B50446002807D140F2AF62AFF2AA
:109640000841AFF2F83001F0C3F8002C35D0064DD8
:109650002868844231D0FEF7B8FB2046FFF7D0FFE0
:1096600038B3201D08E000008C06002040B7002021
:1096700004ED00E070B40020FEF716FEE06A012160
:109680002A69814011432961F84900EB800001EB10
:109690008000211DFEF7E4FDE06A2968C96A88425E
:1096A00007D3F3494FF080500860BFF34F8FBFF3EB
:1096B0006F8FBDE87040FEF7A2BB70BD2DE9F04191
:1096C00000260446002807D140F2E662AFF2984136
:1096D000AFF2884001F07CF8FEF7B8FB5020EFF3C2
:1096E000118580F31188BFF34F8FBFF36F8F204632
:1096F000FFF786FF38B1DF4F386B40B104F1180136
:10970000DD48FEF7ADFD85F311883046DFE4E06A01
:109710003968C96A884200D30126201DFEF7C4FDBE
:10972000E06A01213A69814011433961CF4900EB78
:10973000800001EB8000211DFEF792FDE3E770B58C
:10974000CD4ECC4D14361CE0FFF7BFFD306820B184
:109750000024FFF70EFDA4B901E00124F9E7FEF7AC
:1097600034FBF068C468201DFEF79EFDA868401E0B
:10977000A8606868401E6860FEF741FB2046FFF75E
:1097800041FC68680028DFD170BDB84E4FF08054AE
:10979000B74DFFF7D4FF30680128FAD92C60BFF32A
:1097A0004F8FBFF36F8FF4E71CB5B24800242C3005
:1097B000CDE9004023468222B0A1B248FFF7E3FB87
:1097C000012801D100F0B9FE01280CD0401C1CD1A9
:1097D0004FF4F162AFF2A051AFF2905002B0BDE889
:1097E000104000F0F5BF502080F31188BFF34F8F79
:1097F000BFF36F8F9F484FF0FF31816201214161BC
:10980000C460BDE81C40FEF7A0BA1CBD502080F328
:109810001188BFF34F8FBFF36F8F964900204861C7
:10982000FEF7C7BA9348C068704710B5FEF70EFB45
:109830009048C06810BD8F488068704710B50028F8
:1098400002D004461CB10AE08A480468FAE74FF4E3
:109850000962AFF21C61AFF20C6000F0B9FF04F1D5
:10986000340010BD002101E0401C491C0278A52AEB
:10987000FAD0880880B270472DE9F04707460C46B9
:1098800090461E46002F0ED03D46256005F134005F
:109890006060E86A2061286BE061686CA060207BF2
:1098A000032803D00AE073480568EEE7FFF70DFDD3
:1098B000A86A08B102202073FFF75BFCE86C6061C6
:1098C0004FF00009C4F81890052E01D0267303E06C
:1098D0003846FFF76AFD2073B8F1000F05D0286BFA
:1098E000FFF7C0FF2084BDE8F087A4F82090FAE7D6
:1098F0002DE9F04780460C46914600262068002856
:1099000021D0214648684068486001F10807B84204
:1099100001D1406848604868D0F80CA0606845688C
:109920006560BD4201D1696861606068C56806EB29
:10993000C60008EB80014B4601222846FFF79CFF3A
:10994000761C5545EAD13046CDE72DE9F04706466D
:109950000B46174600242025FFF7B7FCDFF81481DB
:10996000D8F8080083423BD3DFF800916D1E05EB69
:10997000850009EB800104EBC40006EB80000122A6
:10998000FFF7B6FF0444002DF0D104EBC40006EB52
:1099900080000222D8F83410FFF7AAFF044404EB39
:1099A000C40006EB80000222D8F83810FFF7A0FFB1
:1099B0000444314904EBC40006EB80000422143156
:1099C000FFF796FF04442C4904EBC40006EB80002B
:1099D00003222831FFF78CFF04440FB100203860C8
:1099E000FFF7C7FB20467EE770B504460D46002C06
:1099F00007D140F60F32AFF2C071AFF2B07000F095
:109A0000E7FE1C48016820461831FEF735FC284661
:109A1000BDE87040012125E42DE9F04105460E46E0
:109A20001746002D07D14FF43262AFF2F471AFF256
:109A3000E47000F0CDFE0F4C206B38B940F62432B4
:109A4000AFF60C01AFF2FC7000F0C2FE216846F0E8
:109A500000408861216828461831FEF701FC38462D
:109A6000BDE8F0410121FFF7FDBB000070B400200C
:109A700004ED00E08C06002018B7002049444C4556
:109A8000000000008B97040870B506460D4614468A
:109A9000002E07D140F63A32AFF66401AFF654001B
:109AA00000F096FEFE48016830461831FEF7D8FBFC
:109AB0000CB14FF0FF3521462846BDE87040FFF756
:109AC000D1BB2DE9F041C068C468002C07D140F635
:109AD0006A32AFF69C01AFF68C0000F079FE04F11B
:109AE00018000746FEF7E0FBED4D2A6B01265AB140
:109AF0003946EC48FEF7B4FBE06A2968C96A884237
:109B000014D90120EE612CE4201DFEF7CDFBE06AA4
:109B10002A6906FA00F111432961E34900EB80004C
:109B200001EB8000211DFEF79BFBE5E7002018E418
:109B300070B506460C46DA4D286B002807D140F672
:109B4000A232AFF60C11AFF6FC0000F041FE44F07B
:109B500000403060F4683CB940F6AA32AFF62811F4
:109B6000AFF6181000F034FE3046FEF79DFB201DC6
:109B7000FEF79AFBE06A01262A6906FA00F1114312
:109B80002961C94900EB800001EB8000211DFEF72F
:109B900067FBE06A2968C96A884202D90120EE6140
:109BA00070BD002070BD10B50446002C07D140F6F2
:109BB000CA32AFF67C11AFF66C1000F009FEB8485F
:109BC000016A2160C068606010BD70B504460D4632
:109BD000002C07D140F6D432AFF6A411AFF69410A2
:109BE00000F0F6FD3DB940F6D532AFF6B411AFF650
:109BF000A41000F0EDFDFEF7E8F8A94AD068296846
:109C00004B1C08D02368126A934206D062688242D5
:109C100003D801240DE000240BE06268801A88421A
:109C200006D2081A28602046FFF7BDFF002400E096
:109C30000124FEF7E4F8204670BD99490120C8616F
:109C40007047002801D0806C7047002070470028C2
:109C500000D081647047924800687047904841691D
:109C6000002903D0006B18B1002070470120704715
:109C70000220704770B50446002839D0884DE06A4C
:109C80002968C96A884233D2A069002804DB2868A1
:109C9000C06AC0F12000A061E06A834E00EB800042
:109CA000616906EB800081421FD1201DFEF7FCFA9E
:109CB000012150B9E06A00EB800256F8222022B957
:109CC0002A6901FA00F082432A612868C06AE062CA
:109CD0002A6981401143296100EB800006EB800076
:109CE000211DBDE87040FEF7BBBA2868C06AE0627B
:109CF00070BD70B504460026002840D0684D286825
:109D0000844207D04FF46D62AFF6D421AFF6C42081
:109D100000F05EFD206D38B940F6D262AFF6E82162
:109D2000AFF6D82000F054FD206D401E2065E26C97
:109D3000E16A914223D010BB201DFEF7B5FA5A4AC2
:109D4000012150B9E06A00EB800352F8233023B9B7
:109D50002B6901FA00F083432B61E06CE062C0F1F3
:109D60002000A061E06A2B6981401943296100EB62
:109D7000800002EB8000211DFEF772FA01263046BA
:109D800070BD10B50446204601F00BF8204601F0E6
:109D900037F8202101E02154401C0F28FBD300217B
:109DA0002154204410BD7FB50646002434703C4841
:109DB00081680391806800EBC0008000FDF7DBFE46
:109DC0000546280042D000220399FFF7BEFD03900C
:109DD000029429E0029800EBC00005EB8000017BB3
:109DE00001292BD002292BD003292BD004292BD0D9
:109DF000002441683046FFF7C4FF0646029800EB96
:109E0000C00005EB80008168028CCDE90021036968
:109E1000224626A1304600F0E7FC304600F0F0FF75
:109E200006440298401C0290DDE902018842D1D329
:109E300004B02846BDE87040FDF704BF5224D8E7BF
:109E40004224D6E75324D4E74424D2E77FBD144903
:109E5000086880690A680968D26AC2F120028A61CA
:109E600070470F490868002803D00868026D521C2B
:109E700002650868704770B506460C46FDF7A5FFF9
:109E8000074D2868406DF8B92A68012082F858000B
:109E9000D4B101212046FFF7E5F94FF080500DE0E5
:109EA0008C06002018B7002070B400200925630933
:109EB00025750925750925750D0A0000D249086028
:109EC000BFF34F8FBFF36F8FFDF799FFFDF77DFF56
:109ED0002868446D002034B116B12968486502E055
:109EE0002A68611E5165296881F85800FDF787FFCF
:109EF000204670BD2DE9F04781460F46164698462C
:109F0000FDF763FFC14D286890F85800022817D06C
:109F10002C68606D20EA090060652968012081F8DD
:109F20005800B8F1000F0BD001214046FFF79AF915
:109F3000B5494FF080500860BFF34F8FBFF36F8F6C
:109F4000FDF75DFFFDF741FF16B12868406D3060F9
:109F5000286890F8580001280CD02868416DB94352
:109F6000416501242968002081F85800FDF747FF6A
:109F70002046B8E40024F5E72DE9F04104460D46FB
:109F800090461F460126002C07D141F20612AFF67B
:109F90005851AFF6485000F01BFCFDF716FF0FB10B
:109FA000606D386094F85800022184F85810B8F1B8
:109FB000050F13D2DFE808F01203070B0D00616DE7
:109FC000294361650AE0616D491C616506E06565CC
:109FD00004E0022801D0656500E00026012828D1B0
:109FE000201DFEF761F9894DE06A01212A6981404F
:109FF00011432961864900EB800001EB8000211D9F
:10A00000FEF72EF9A06A38B141F23E12AFF6D851F0
:10A01000AFF6C85000F0DCFBE06A2968C96A8842E4
:10A0200007D979494FF080500860BFF34F8FBFF3D5
:10A030006F8FFDF7E4FE304665E52DE9F0470446F5
:10A04000DDF820800D4691469A460127002C07D165
:10A0500041F27212AFF62061AFF6106000F0B8FB6B
:10A06000FDF7F4FE5020EFF3118680F31188BFF363
:10A070004F8FBFF36F8FBAF1000F02D0606DCAF837
:10A08000000094F85800022184F85810B9F1050F27
:10A0900013D2DFE809F01203070B0D00616D2943AD
:10A0A00061650AE0616D491C616506E0656504E073
:10A0B000022801D0656500E00027012832D1A06A9E
:10A0C00038B141F2B912AFF69061AFF6806000F09E
:10A0D0007FFB4E4D286B4FF0010978B104F1180158
:10A0E0004C48FEF7BDF8E06A2968C96A884219D968
:10A0F000B8F1000F14D0C8F8009013E0201DFEF74F
:10A10000D3F8E06A2A6909FA00F11143296100EBEA
:10A1100080013F4800EB8100211DFEF7A1F8E2E736
:10A12000C5F81C9086F3118838460DE42DE9F041FE
:10A1300004468846002C07D141F2ED12AFF60871B3
:10A14000AFF6F86000F044FBFDF780FE5020EFF31F
:10A15000118780F31188BFF34F8FBFF36F8F94F88F
:10A160005800022184F85810616D491C616501286E
:10A1700030D1A06A38B141F21322AFF64471AFF684
:10A18000347000F025FB214D286B012678B104F1D5
:10A1900018012048FEF764F8E06A2968C96A884215
:10A1A00018D9B8F1000F14D0C8F8006012E0201DD3
:10A1B000FEF77AF8E06A2A6906FA00F1114329618C
:10A1C000134900EB800001EB8000211DFEF748F8E9
:10A1D000E2E7EE6187F3118895E410B500280BD013
:10A1E0000446FDF7F2FD94F85800022807D0002439
:10A1F000FDF705FE204610BD04480468F1E7002085
:10A2000084F858000124F3E704ED00E08C060020F8
:10A2100070B4002018B7002070B5002441600061C0
:10A22000F74D91420AD8D11A8269914201D3012493
:10A230000EE0011D2869FEF71FF809E09A4203D2DB
:10A24000994201D3012403E0011DE868FEF714F8E8
:10A25000204670BD2DE9FF470546DDF830A00E46CB
:10A26000904699460027002D05D14FF4D372E5A101
:10A27000EAA000F0ADFAE24C2068F8B10096CDF803
:10A2800004800295062E13DAFFF7E8FC022807D0B7
:10A2900000231A4669462068FEF748F907460DE094
:10A2A0000023524669462068FEF740F9074605E05C
:10A2B00000234A466946FEF75CFB074604B0384671
:10A2C000BDE8F087F8B5CE4E25E0C0680568C468E3
:10A2D000201DFDF7E9FF616A20468847E0690128F3
:10A2E00019D1A0692844A84206D960602461211DC3
:10A2F000F068FDF7C1FF0EE0002003460146009024
:10A300002A462046FFF7A6FF28B940F29232BDA1A7
:10A31000C2A000F05DFAF06801680029D5D1F068AC
:10A320003169F1603061F8BD70B50546FFF77AFA22
:10A330000446B34EB068844204D2FFF7C3FF012045
:10A34000286001E000202860B460204670BD70B530
:10A3500086B0AB4E53E00298002803DADDE9032013
:10A36000059990470298002849DB049C606910B168
:10A37000201DFDF799FF01A8FFF7D6FF05460298BB
:10A380000A283CD2DFE800F00505053B2738050523
:10A390003B270398A169034601442A462046FFF75C
:10A3A0003BFF00282BD0616A20468847E0690128DE
:10A3B00025D1002000900398A16900234218194676
:10A3C0002046FFF747FFD0B940F221328DA193A07C
:10A3D00000F0FEF913E00398A06128B94FF44E7223
:10A3E00088A18EA000F0F4F9A0692B4641192A46F5
:10A3F0002046FFF711FF02E02046FDF723FC002373
:10A400001A4602A93068FEF7B0F90028A3D106B0B9
:10A4100070BDF8B505460E467948C068C068C46886
:10A42000201DFDF741FFE069012816D1A0692B46E8
:10A43000411932462046FFF7EFFE70B10020034677
:10A44000014600902A462046FFF704FF28B94FF442
:10A4500002726CA171A000F0BBF9616A01B02046E4
:10A46000BDE8F0400847F8B506460D46FEF72DFF5B
:10A470006846FFF759FF0446009810B1FEF779FED1
:10A48000F8BD45B9A64206D8FEF773FE2146304610
:10A49000FFF7BFFFF8BD5A481DB10169096891B1C6
:10A4A0000025311B2A460068FEF75AFCFEF761FEC4
:10A4B0000028EFD15D494FF080500860BFF34F8F07
:10A4C000BFF36F8FF8BD0125EBE74D49CA681168EE
:10A4D000002904D00021016019B10020704701213A
:10A4E000F9E7D0680068704708B56846FFF7EDFFE8
:10A4F0000099FFF7B8FFFFF72AFFF6E710B5FDF761
:10A5000064FC3F4C2068A0B94948FDF79BFE4848D1
:10A510001430FDF797FE4648E060143020610022B9
:10A5200010210520FDF726FF206010B141A1FEF7A4
:10A53000F6FBBDE81040FDF762BC1CB50024FFF738
:10A54000DDFF2F48006860B12D481F21001DCDE9B7
:10A55000001000234FF4827238A13A48FEF713FD31
:10A5600004462CB940F2331226A12CA000F030F999
:10A5700020461CBD2DE9F0470646DDE908940D464E
:10A5800017469846002D05D14FF4C6721DA123A091
:10A5900000F01EF9002C0DD0FFF7B0FF2660A5617A
:10A5A000E761C4F82080C4F82490201DBDE8F0477E
:10A5B000FDF753BE84E62DE9FC4706460A9D0F468B
:10A5C000904699462C20FDF7D6FA04463CB1CDE9D9
:10A5D00000544B46424639463046FFF7CBFF2046F3
:10A5E000BDE8FC8710B5064C6068002805D14FF423
:10A5F000E87204A109A000F0EBF8606810BD00004B
:10A60000C80600202E2E5C4672656552544F535C7E
:10A6100074696D6572732E63000000004572726F7D
:10A62000723A25732C25640D0A00000004ED00E049
:10A6300054B70020546D725100000000546D722018
:10A6400053766300E9A4040810B50446002807D136
:10A6500040F2D912AFF25401AFF2400000F0B8F866
:10A66000A069CBE710B50446002807D140F2E312F9
:10A67000AFF27001AFF25C0000F0AAF86068BDE7CD
:10A6800010B50446002807D140F2ED12AFF28C015C
:10A69000AFF2780000F09CF82068AFE710B50446F0
:10A6A000002807D140F2DA32AFF2A801AFF29400ED
:10A6B00000F08EF8FDF789FB606908B1012400E025
:10A6C0000024FDF79CFB204698E710B504460028BF
:10A6D00007D140F2EF32AFF2D401AFF2C00000F088
:10A6E00077F8FDF772FB246AFDF789FB204685E7C2
:10A6F00070B50D460446002807D140F2FF32AFF294
:10A70000FC01AFF2E80000F063F8FDF75EFB2562A4
:10A71000BDE87040FDF773BB7FB51D466FF00104C7
:10A720000094019002910392144800232A4669463E
:10A730000068FEF71EF904B070BD2DE9FF41044624
:10A740000D46164698460D4F3A68002A07D140F24A
:10A750002B42AFF25011AFF23C1000F039F84FF03D
:10A76000FF32009201940295039600234246694607
:10A770003868FDF7DBFE04B0BDE8F081C8060020B4
:10A78000704710B5044600F0A9FC0068005DC006E3
:10A7900002D504F1200010BD204610BD7CB51D4639
:10A7A00016460C00009001D02044401E074B7B440D
:10A7B0002A4669460190304600F015FF05461CB157
:10A7C0000020694600F022FF28467CBD650E00008F
:10A7D0000FB4044910B503AA029800F03BFF10BC67
:10A7E0005DF814FBC40500200FB41CB5084B06AA85
:10A7F0007B4469460090059800F0F5FE0446002071
:10A80000694600F003FF20461CBC5DF814FB000005
:10A81000190E00000FB47CB50C0009AA009001D0FD
:10A820002044401E084B7B4469460190089800F084
:10A83000DAFE05461CB10020694600F0E7FE284616
:10A840007CBC5DF814FB0000ED0D000070B5044603
:10A8500085690068C10601D5302600E02026C007C2
:10A8600007D070BDD4E9012130469047206A401CD2
:10A8700020626D1EF6D570BD70B5044685690078FE
:10A88000C00707D170BDD4E9012120209047206A7C
:10A89000401C20626D1EF6D570BD09684A0501D5C1
:10A8A00040B27047C905FCD500B2704709684A0537
:10A8B00001D5C0B27047C905FCD580B2704770B5EC
:10A8C0000C460546012A05D02878800600D5EA699D
:10A8D000002302E0012305E05B1C934202D2E05C0E
:10A8E0000028F9D1A869E618C01AA861286A184496
:10A8F00028622846FFF7AAFF04E0D5E9012114F8F1
:10A90000010B9047B442F8D32846FFF7B5FF70BD5E
:10A910002DE9F0410646002410687529314616A538
:10A9200010D0FFF7BAFF002802DA404213A507E073
:10A9300031688A0701D512A502E0490704D511A59F
:10A94000012401E0FFF7B2FF00210A2206F12407EB
:10A9500009E0B0FBF2FCB0FBF2F302FB1C0030306C
:10A9600078541846491C0028F3D123462A4630461D
:10A97000BDE8F04100F0C9BB000000002D00000060
:10A980002B0000002000000011680268006A5305D7
:10A9900001D508700AE0D30501D5088006E013064A
:10A9A00003D5C217C1E9000200E00860012070472A
:10A9B0002DE9FF5F15468A460446DFF8AC80F8446F
:10A9C0000027D8E900103E46CDE9001010E03AF823
:10A9D00016106A4602A800F0DBFE411C07D0217861
:10A9E000890603D5E269391891420DD80744761CCF
:10A9F0002078800602D5E069B84205DDAE42E6DB8C
:10AA00003AF816000028E2D1A069C01BA0612046D8
:10AA1000FFF71CFFD8E90010CDE90010002017E077
:10AA20003AF818106A4602A800F0B2FEB0F1FF3FF3
:10AA300081460BD000250DF1080B05E0D4E901217A
:10AA40001BF8050090476D1C4D45F7D308F1010038
:10AA5000B0428046E4DB206A384420622046FFF79B
:10AA60000BFFBDE8FF9F0000AE4D000030B4002199
:10AA700000F1240408E002F00705D208303542EA6C
:10AA80004372DB086554491C52EA0305F3D104689C
:10AA9000002310A2250707D5A40600D421B1C4695C
:10AAA00001230DA2641EC46130BC00F02EBB10B5A2
:10AAB000044621461068FFF7F9FE02462046BDE82D
:10AAC00010400023D2E7D21D22F00701D1E9002374
:10AAD000CCE700000000000030000000F0B40D469C
:10AAE0000188090502D5214C7C4402E01F4C7C44BE
:10AAF0000E34002100F1240608E002F00F071209CD
:10AB0000E75D42EA03721B097754491C52EA0307C6
:10AB1000F3D102780023120704D5702D06D009B1B5
:10AB2000022311342246F0BC00F0EFBA01231034A6
:10AB3000F8E770B504460D4621461068FFF7B6FEEB
:10AB4000024629462046BDE870400023C6E7D21DD4
:10AB500022F00703D3E90023C0E70368126843F03B
:10AB6000200303600823C3610023B7E78C4C000077
:10AB70002DE9F05F894604464FF0000ADFF874B112
:10AB8000FB44C0F820A02046E1688847002874D024
:10AB9000252806D0D4E901219047206A401C206274
:10ABA000F1E700265F462046E168884720280546F1
:10ABB00007DB312D05D2781910F8200C08B10643B7
:10ABC000F1E7B00701D526F00406C4F81CA0002761
:10ABD000C4F818A02A2D09D0284601F09BFD38B3EF
:10ABE00004EB8708303DC8F8185019E059F8041BE9
:10ABF000204604EB87029161E1688847012F0546F2
:10AC000018D1E069002820DA26F020061DE0D8F8E7
:10AC1000180000EB800005EB40003038C8F8180041
:10AC20002046E1688847054601F074FD0028EED112
:10AC3000012F0AD02E2D08D12046E16888477F1CBD
:10AC40000546022F46F02006C4DBA069002803DA7F
:10AC5000404246F00106A061F00701D026F0100640
:10AC60006C2D0BD0682D09D04C2D39D06A2D35D0E4
:10AC7000742D35D07A2D33D016E038E0E1682F46B8
:10AC800020468847B842054609D16C2F26D04FF49C
:10AC90008060E168064320468847054604E06C2F43
:10ACA0001AD04FF4807006430DB3A5F14100192866
:10ACB00002D8203546F400664A46294620462660DA
:10ACC0004E46F1F78FFA80B101280BD0F61D26F021
:10ACD000070000F1080956E74020E4E78020D8E7A4
:10ACE0000020D6E706F104094DE7284652E7206A1E
:10ACF000BDE8F09F1C4C000070B5064600F0F6F968
:10AD00000468054630460A22002100F009FD2C6047
:10AD100070BD401ECAB210F8011F8A4202D000293D
:10AD2000F9D10020704710B5431E13F8014F002CD5
:10AD3000FBD105E011F8014B002C03F8014B03D0C7
:10AD4000521EF7D20021197010BD40EA010310B560
:10AD50009B070FD1042A0DD310C808C9121F9C42AB
:10AD6000F8D020BA19BA884201D9012010BD4FF09D
:10AD7000FF3010BD1AB1D30703D0521C07E00020EA
:10AD800010BD10F8013B11F8014B1B1B07D110F847
:10AD9000013B11F8014B1B1B01D1921EF1D118464A
:10ADA00010BD40EA0103024630B59B0710D14FF0B9
:10ADB000013400E008C208C91D1B9D4315EAC41FE9
:10ADC000F8D013F0FF0102F8011B0DD01B0AF8E7C1
:10ADD00011F8013B002B02F8013B05D011F8013BB3
:10ADE000002B02F8013BF3D130BD0022CBB210F8AA
:10ADF000011B994200D1421E0029F8D1104670472C
:10AE000010B5431C02E010F8011B71B18107FAD1A3
:10AE10004FF0013202C88C1A8C4314EAC211F9D0E7
:10AE2000C01A0A0603D0C01E10BDC01A10BD0A0405
:10AE300001D0801E10BD0902FCD0401E10BD40EAAA
:10AE4000010370B59B072ED14FF00136042A2AD397
:10AE500008C810C99D1B9D43121F15EAC61517D0BF
:10AE6000D8B2E1B2401A50EA056110D198B2A1B24D
:10AE7000401A50EA05410AD123F07F4024F07F4177
:10AE8000401A50EA052102D1180EA0EB146070BDE3
:10AE9000A342DBD018BA21BA884201D9012070BD83
:10AEA0004FF0FF3070BD0AB9002070BD10F8013BB3
:10AEB00011F8014B63B1A3420AD1521E08D010F819
:10AEC000013B11F8014B1BB1A34201D1521EEDD140
:10AED000181B70BD421E12F8013F002BFBD111F868
:10AEE000013B002B02F8013BF9D17047032A40F2E5
:10AEF000308010F0030C00F0158011F8013BBCF11C
:10AF0000020F624498BF11F801CB00F8013B38BF33
:10AF100011F8013BA2F1040298BF00F801CB38BF41
:10AF200000F8013B11F0030300F02580083AC0F05F
:10AF3000088051F8043B083A51F804CBA0E8081007
:10AF4000F5E7121D5CBF51F8043B40F8043BAFF33A
:10AF50000080D20724BF11F8013B11F801CB48BF94
:10AF600011F8012B24BF00F8013B00F801CB48BFCA
:10AF700000F8012B704710B5203AC0F00B80B1E803
:10AF80001850203AA0E81850B1E81850A0E818501E
:10AF9000BFF4F5AF5FEA027C24BFB1E81850A0E827
:10AFA000185044BF18C918C0BDE810405FEA827C41
:10AFB00024BF51F8043B40F8043B08BF7047D20758
:10AFC00028BF31F8023B48BF11F8012B28BF20F8F9
:10AFD000023B48BF00F8012B704702F0FF0343EA31
:10AFE000032242EA024200F002B84FF000020429B4
:10AFF000C0F0128010F0030C00F01B80CCF1040CA8
:10B00000BCF1020F18BF00F8012BA8BF20F8022BDB
:10B01000A1EB0C0100F00DB85FEAC17C24BF00F881
:10B02000012B00F8012B48BF00F8012B70474FF0AF
:10B03000000200B5134694469646203922BFA0E888
:10B040000C50A0E80C50B1F12001BFF4F7AF090794
:10B0500028BFA0E80C5048BF0CC05DF804EB890085
:10B0600028BF40F8042B08BF704748BF20F8022BC8
:10B0700011F0804F18BF00F8012B704710B504463F
:10B0800010F0030F08BF11F0030F40F015804FF0D0
:10B09000013E121FC0F20E8051F8043BA3EB0E0CD0
:10B0A0002CEA030C1CEACE1C08BF40F8043BF0D08D
:10B0B000A1F1040102F10402521E08DB11F8013B68
:10B0C000002B00F8013BF7D11146FFF78EFF204619
:10B0D00010BD7047704770477047000010B500F012
:10B0E0007BFB001D10BD00BF992400000048704785
:10B0F0007CB7002010B5FFF7F9FF006810BD10B550
:10B100000446FFF7F3FF046010BD2DE9F0470D463C
:10B1100099469246044600F124080168880604D541
:10B12000E06921F01001216000E00120A84201DD6A
:10B13000471B00E00027A1697A1902EB0900081AF1
:10B14000A0612078C00602D42046FFF77FFB0026CE
:10B1500008E0D4E901211AF806009047206A401C53
:10B16000761C20624E45F4DB2078C0060AD52046C6
:10B17000FFF76CFB06E0D4E9012130209047206AFC
:10B18000401C2062381EA7F10107F4DC07E0D4E977
:10B19000012118F805009047206A401C2062281EF3
:10B1A000A5F10105F3DC2046FFF766FB20780006D9
:10B1B00002D50220BDE8F0870120FBE770472DE9AA
:10B1C000FF4F0C461E464FF0FF378BB0D2E900010F
:10B1D000DDF860800A908A46C1F30A5505B93D46FC
:10B1E000002108464FF00000BAF1000F00F44000C3
:10B1F00005DA00EB80004FF4400101EA50004FEA0D
:10B200009059B9F1010F00DDB9460A9850EA4A0099
:10B210000ED044F61050A5F2FF3545432F14B8F177
:10B22000000F1ED07542291E1EDDC9F100021CE070
:10B23000B8F1010F4FF0000001D0302103E0F243DC
:10B2400005E02154401CB042FBDB304600220021C7
:10B2500021540B99C1F80880C1E900200FB0BDE866
:10B26000F08FBD1B6D1CDEE74A4600DA694206A876
:10B2700000F00AFD06AB93E8070003AB83E8070084
:10B2800050460A9900F0F2FD8DE80700A0F5005045
:10B290001F3800900398002D0ADD42F21F014A4634
:10B2A0000844002303A90390684601F05BF809E015
:10B2B000A0F500504A461F38002303A903906846B2
:10B2C00001F065F88DE807000004000C03D04FF092
:10B2D000FF30410800E01046B8F1000F03D0002213
:10B2E000009215461EE0751E05D400F079FA303242
:10B2F00062556D1EF9D5B3460122084302D00022E3
:10B300007F1C04E02078302801D100227F1E002A13
:10B31000099784D01DE0112D07DA00F061FA303270
:10B3200062556D1C50EA0102F5D1084302D0009825
:10B33000C8B10EE00021681E05E0235C625C635426
:10B340002254401E491C8142F7DBAB46A81B401E1D
:10B350000990002004F80B000B98099AC0F80880A7
:10B36000C0E9002B7AE711264FF0000857E72DE9D6
:10B37000F04F88460446D21D22F0070191B0D1E972
:10B380000001CDE90A0101F039F902460B98C00F1E
:10B3900001D02D2007E02068810701D52B2002E095
:10B3A000202101EAC000032A099001D0072A05DB09
:10B3B00003464146204600F0D7FB0BE1207880068B
:10B3C00001D5E06900E00620B8F1650F814606D09E
:10B3D000B8F1660F18D0B8F1670F70D131E00020D6
:10B3E000B9F1110F009001DB112301E009F1010314
:10B3F0000AAA01A90CA8FFF7E2FEDDE90C700026FD
:10B4000009F10105834647E001204B4600904FF0CB
:10B4100000470AAA01A90CA8FFF7D1FEDDE90DB08B
:10B420000C995D46002610B909F101000D18B9EB21
:10B43000050003D4C0F1FF3609F10105A5EB0900B1
:10B440002BE0B9F1010F01DA4FF001090020B9F149
:10B45000110F0090484601DD112300E003460AAABF
:10B4600001A90CA8FFF7ABFEDDE90C704D460026E4
:10B470008346207800070AD4AB4500DA5D4601A870
:10B48000012D04DD411911F8011C302907D04F4569
:10B4900002DA17F1040F04DA012082460FE06D1E74
:10B4A000EEE7002F02DCED1B3E4403E0781CA842CF
:10B4B00000DD7D1CB81B00F1010A4FF00047207829
:10B4C000000703D4AA4501DB4FF0FF3A0021B7F192
:10B4D000004F0DF143088DF8431024D002202B2398
:10B4E000002F01DA7F422D230A21021EA0F1010064
:10B4F00000DC5FB197FBF1FC97FBF1F201FB1C7CD8
:10B5000017460CF1300C08F801CDEEE7A8F1010068
:10B5100003702188090501D5452100E06521A0F1CE
:10B52000010800F8011C09980FA9A1EB0807FF1DED
:10B5300000B10120411901EBEA70A1693844081AF1
:10B54000401EA0612078C00602D42046FFF77EF995
:10B55000099828B1D4E901219047206A401C206253
:10B560002078C00622D52046FFF770F91EE0002E95
:10B5700004DBB34502DD01A8805D00E03020D4E9A2
:10B5800001219047206A401C2062761CAAF101002C
:10B590005FEA000A0AD100F01FF9C0680168405C48
:10B5A000D4E901219047206A401C2062281EA5F1A1
:10B5B0000105DCDC07E0D4E9012118F8010B904714
:10B5C000206A401C2062381EA7F10107F3DC2046E8
:10B5D000FFF752F9032011B041E6000001694A1C4F
:10B5E00002610878704700B58FB0CDE901310021C4
:10B5F000059105497944CDE9031011466846FFF7E6
:10B60000B7FA0FB000BD0000E5FFFFFF0A6802F8BF
:10B61000010B0A607047D1E900239A4202D2531C01
:10B620000B601070704710B5436913B1AFF3008021
:10B6300001E0FFF744F9012010BD127800F1240168
:10B640000A7000224A700122EDE711684FF0FF32C4
:10B65000E9E70000074B70B50D467B44FFF7C3FFD9
:10B660000446284600F082FB10B14FF0FF3070BD59
:10B67000204670BD197AFFFF10B5436913B1AFF3CF
:10B68000008001E0FFF794F9012010BD128800F15D
:10B69000240182840022C2840122EDE711684FF068
:10B6A000FF32E9E72DE9F0418046D21D22F0070282
:10B6B0000025D2E90002F52915A614D0011E72F169
:10B6C000000106DA0023D0EB030063EB020211A6AF
:10B6D00008E0D8F800108B0701D50FA602E0490753
:10B6E00001D50EA601251146002408F1240704E027
:10B6F00000F076F830323A55641C50EA0102F7D176
:10B700002B46324621464046BDE8F041FFF7FDBCDE
:10B71000000000002D0000002B00000020000000B1
:10B720002DE9F04791460F4680460446002614F85E
:10B73000015B2DB1FFF7D2FC0068405DC007F6D178
:10B740002B2D02D02D2D18D0641E4A463946204696
:10B7500000F04AFA27B13968A14201D1C7F8008048
:10B760004FF0020471050BD54042002803DDFFF7BE
:10B77000BDFC0460A007BDE8F08746F48066E4E7FE
:10B780000028F8DAFFF7B2FC04606FF00040F2E73F
:10B7900070B516460C460546FFF7A0FC036893F803
:10B7A0000101012806D0FF2C0FD8185D68B10120D7
:10B7B0002C7070BDD3F807013246214603F20713FF
:10B7C00003442846BDE8704018474FF0FF3070BD75
:10B7D000004870477CB70020004870479CB70020A5
:10B7E00030B5B0F10A024FEA900E71F100034EEA53
:10B7F000817EB0EB0E0061EB91014FEA101E4EEA24
:10B80000017E10EB0E0041EB11114FEA102E4EEAB3
:10B81000016E10EB0E0041EB11214FEA104E4EEA83
:10B82000014E10EB0E0041EB1141401841F10001B7
:10B830004FEAD00040EA41704FEAD10110EB800599
:10B840004FEA810444EA907444EB01046D1944EB1F
:10B850000404521BA3414FF0000348BF0A3200D535
:10B8600030BD401C41F1000130BD00002DE9F04F1A
:10B8700004460D46D21D22F0070089B0D0E900979A
:10B880004846394600F0BAFE0246F80F01D02D2393
:10B8900007E02068810701D52B2302E0202101EA7F
:10B8A000C0038DF820300BB1012000E00020032AF6
:10B8B000824601D0072A04DB2946204600F054F9CD
:10B8C0003FE12078800601D40D2500E0E569C7F34B
:10B8D0000A560D2D49DA00214FEA175B08464FF052
:10B8E0000000002F00F4400007DA00EB80004FF466
:10B8F000400100EBD07001EA60008115012901DDF3
:10B900004FF0FF3100224FEA850CBCF1180F06D32F
:10B910001346ACF118004FF08052C24003E04FF4E0
:10B92000801323FA0CF30CF10C0CBCF1200F04D3A0
:10B93000ACF1200C09FA0CF001E007FA0CF0002938
:10B940004FF0004801DD18B90FE00ED140450CD38F
:10B9500019EB02095F4121B9404502D19F4329EA11
:10B960000209BBEB175F00D0761C2088000502D5CA
:10B970007B48784402E07A487844193808AA302392
:10B9800002F80A30037C0AF10101002E0AF1020AD2
:10B9900053546A4602DC4FF0300101E04FF03101B0
:10B9A0004FF001088DF8001002D0A6F2FF3603E038
:10B9B00059EA470100D06B4E002D02DC21780907BF
:10B9C00004D54FF002082E218DF80110C446002145
:10B9D0000BE0C7F303433F01C35C491C6D1E02F833
:10B9E0000830052908F1010801DA002DF1DC0021F9
:10B9F0000CE000EB1973491C1B786D1E082902F836
:10BA000008304FEA091908F1010801DA002DF0DCCD
:10BA100021688B0602D516E0A8F10108E04505DD96
:10BA200002EB080313F8013C302BF5D0B8F1000FFE
:10BA300009DD02EB080313F8013C2E2B03D10907A3
:10BA400001D4A8F10108002D05DD3E2102F80810FF
:10BA50006D1E08F10108407C002E02F8080008F174
:10BA6000010804DA2D20764202F8080002E02B20BB
:10BA700002F808000A214FF47A70864208F10108A2
:10BA80000BDB96FBF0F3303302F8083096FBF0F353
:10BA900008F1010800FB136601E0642E0CDB642052
:10BAA00096FBF0F3303302F8083096FBF0F308F120
:10BAB000010800FB136601E00A2E06DB96FBF1F09D
:10BAC000303002F8080008F1010896FBF1F001FBA4
:10BAD0001060303002F80800A16908F1010808EB95
:10BAE000050202EB0A00081AA0612078C00602D401
:10BAF0002046FEF7ABFE216A08AE01EB0A00206289
:10BB000004E0D4E9012116F8010B9047BAF1010ACB
:10BB1000F7D22078C00602D52046FEF797FE6E4683
:10BB200009E016F8010B3E280FD0D4E90121904717
:10BB3000206A401C2062B8F10108F2D22046FEF7CC
:10BB40009BFE09B00320BDE8F08F206A28442062E4
:10BB500003E0D4E90121302090476D1EEBD3F8E7D4
:10BB60001D3F000002FCFFFF2DE9F0411F46044687
:10BB700003260168072A01F4006004DB08B116A55A
:10BB800005E016A503E008B115A500E015A521F014
:10BB900010002060A069C01EA0610FB1401EA0610E
:10BBA0002046FEF753FE4FB1D4E9012138469047B5
:10BBB000206A401C2062C01C206206E0206AFAE76E
:10BBC000D4E9012115F8010B9047761EF8D22046E2
:10BBD000FEF752FEBDE8F0814E414E006E616E00F0
:10BBE000494E4600696E66002DE9F05F82461546B3
:10BBF0008B4600270AF10104B9460078302801D0AD
:10BC00009DB113E014F8010B0127782803D05828C0
:10BC100001D045B10AE00DB1102D07D1002714F86D
:10BC2000010B102502E0082500E00A250026B04699
:10BC30000EE005FB080005FB06F101271FFA80F85E
:10BC400001EB1046B6F5803F00D3B94614F8010B5E
:10BC5000294600F0B4F80028EBDABBF1000F05D05C
:10BC60000FB1641E00E05446CBF80040B9F1000F5C
:10BC700006D0FFF73BFA02210160C81EBDE8F09F25
:10BC800048EA0640FAE700002DE9F04781461646EB
:10BC90008AB0354878440DC88DE80D0032487844A4
:10BCA000801C03AC0DC884E80D0041F69B300844AD
:10BCB000372190FBF1F290FBF1F5A5F1800501FB36
:10BCC00012041B3C02D56442012000E00020DFF892
:10BCD00098A080460027FA44AAF1BE0A0EE0E007C9
:10BCE0000AD03246684607EB470101230AEB81017F
:10BCF00000F04DFB8DE8070064107F1C002CEED196
:10BD0000194F7F44AE3F19E0E80715D007EB041048
:10BD10000DF1180A90E80E008AE80E00C068F042A3
:10BD200001D1981908903246012306A903A800F012
:10BD30002EFB03AB83E807006D10641C002DE3D1DC
:10BD40004FF0010332466946B8F1000F03A802D054
:10BD500000F008FB01E000F01AFBC9E90001C9F896
:10BD600008200AB0BDE8F0878C3C0000007B00F0A2
:10BD7000800070477546FFF72BFDAE46050069460B
:10BD8000534620F00700854618B020B5F0F7EEFACC
:10BD9000BDE820404FF000064FF000074FF00008CC
:10BDA0004FF0000B21F00701AC46ACE8C009ACE84D
:10BDB000C009ACE8C009ACE8C0098D4670473A2814
:10BDC00000D2303820F02002412A01D3A2F13700FE
:10BDD000884201D34FF0FF30704710B50446AFF3EF
:10BDE00000802046BDE81040F0F75FBA4FF0013CFC
:10BDF00050F8042B51F8043B9A4221D1A2EB0C03DA
:10BE0000934313EACC1317D150F8042B51F8043B99
:10BE10009A4215D1A2EB0C03934313EACC130BD136
:10BE200050F8042B51F8043B9A4209D1A2EB0C03C1
:10BE3000934313EACC13DBD04FF00000704700BFF0
:10BE4000D01A01BAB1FA81F101F0180122FA01F019
:10BE5000CB40C1F12001DBB2C0B2C01A2CFA01F311
:10BE6000D11A914311EAC311E6D170475FEA400C41
:10BE700008BF91F0000F4FEA8C234FEAC12243EA3A
:10BE800051514FEA1C5018BF00F5F0404FEA300006
:10BE900018BF41F000415FEA6C5C00F02980BCF102
:10BEA000FF3F08BF40F080407047130C06BF1204EC
:10BEB0004FF0100C4FF0000C130E04BF12020CF1E7
:10BEC000080C130F04BF12010CF1040C930F04BFF4
:10BED00092000CF1020CD30F04BF52000CF1010CC4
:10BEE00011464FF00002A0F11F00A0EB0C007047BC
:10BEF00011F0004F08BF704731F000413FF4D5AF5B
:10BF00000B0C06BF09044FF0100C4FF0000C0B0E89
:10BF100004BF09020CF1080C0B0F04BF09010CF15E
:10BF2000040C8B0F04BF89000CF1020CCB0F04BF73
:10BF300049000CF1010CCCF12003A0EB0C0022FA1B
:10BF400003F302FA0CF241EA030100F10100704729
:10BF500020F07F4C80EA030023F07F47ACEB07031F
:10BF600003F57C5300F0004003F1FF032DE9804905
:10BF70004FEA154B09B44FEA144325EA0B4E24EA65
:10BF800003480FF2042606EB132749083E785FEAC0
:10BF9000320203FB0667C7F5000707FB06F64FEA08
:10BFA00054374FEAD64606F1020607FB066CCCF181
:10BFB000005C4FEA1C472CEA074C07FB06F40CFB1D
:10BFC00006F504EB15464FEA961634BF00204FF0F5
:10BFD00000404FEAD13706FB07FC4FEA1C4C0CFB34
:10BFE0000BF7D21B03FB0CF761EB07010CFB0EF701
:10BFF000B0EB074072EB17420CFB08F734BFA2EB23
:10C000000742B2EB074261EB17414FEA0C444FEA9B
:10C01000910706FB07FC4FEA1C4C0CFB0BF7B0EB3F
:10C02000C74072EB573203FB0CF734BFA2EBC74299
:10C03000B2EBC74261EB57310CFB0EF7B0EBC70018
:10C0400072EB57720CFB08F734BFA2EBC702B2EBDE
:10C05000C70261EB5771039F4FEA816141EA921178
:10C0600004EBCC044FEAD1374FEA826206FB07FCAF
:10C0700042EA90124FEA80604FEA1C4C0CFB0BF72F
:10C08000D21B03FB0CF761EB07010CFB0EF7B0EBC7
:10C09000074072EB17420CFB08F734BFA2EB0742D4
:10C0A000B2EB074261EB17414FEA8C554FEA91071B
:10C0B00004EB9C2406FB07FC4FEA1C4C0CFB0BF723
:10C0C000B0EBC74072EB573203FB0CF734BFA2EB67
:10C0D000C742B2EBC74261EB57310CFB0EF7B0EB36
:10C0E000C70072EB57720CFB08F734BFA2EBC70214
:10C0F000B2EBC70261EB577115EB4C254FEA81613A
:10C1000041EA92114FEA82624FEAD13742EA901235
:10C1100006FB07FC44F100044FEA80604FEA1C4C28
:10C120000CFB0BF7D21B03FB0CF761EB07010CFBBD
:10C130000EF7B0EB074072EB17420CFB08F734BF69
:10C14000A2EB0742B2EB074261EB174115EB1C155E
:10C150004FEA813141EA92414FEA823242EA90420B
:10C160004FEA80304FEA0C7644F1000448EA03437A
:10C170004EEA0B484FF0000EB2EB080C71EB0307D0
:10C1800024BF624639464EEB0E0E4FF0000B0018EE
:10C19000524149414BEB0B0BB2EB080C71EB03071F
:10C1A0007BF1000B24BF624639464EEB0E0E4FF07A
:10C1B000000B0018524149414BEB0B0BB2EB080C42
:10C1C00071EB03077BF1000B24BF624639464EEB4F
:10C1D0000E0E51EA020718BF46F0010616EB0E7666
:10C1E00055F1000254F1000103D5BDE88901BDE815
:10C1F0000088BDE88901BDE80048B619524141EB0D
:10C200000101A3F10103704780807F7E7D7C7B7AF2
:10C210007978777676757473727171706F6E6E6DF2
:10C220006C6C6B6A6A696868676666656464636398
:10C2300062616160605F5F5E5E5D5D5C5C5B5B5A1E
:10C240005A5959585857575656555555545453538B
:10C2500052525251515050504F4F4F4E4E4D4D4DE6
:10C260004C4C4C4B4B4B4A4A4A4949494848484731
:10C27000474747464646454545444444444343436F
:10C280004342424242414141002B9C4630D4770018
:10C290002BD01CB54FEA370703B44FF010004FF016
:10C2A0001001BAF1000F06D0BCF1000FDCBF40F066
:10C2B000080040F008014FF000000FBCBDE810403E
:10C2C0000BF1010BBBF1010F08BF5FEA170722BF9B
:10C2D00012F1010211F101014FF0004143F100039D
:10C2E00000F0004043EA00007047F9D35708D0E758
:10C2F00046EA064613F1400F4FEA16461FDD13F1DA
:10C30000200FDFBF16430A46002120335B42BED018
:10C31000C3F1200746EA064602FA07F74FEA164637
:10C3200046EA0706C3F1200722FA03F201FA07F7EB
:10C3300021FA03F14FF0000342EA0702A7E746EAB9
:10C34000020646EA06464FEA164646EA0106BCBF22
:10C3500046EA0646360C4FF000034FF000024FF05D
:10C36000000194E72DE9804C9A46934670B491E819
:10C37000380007C831EA400C48BF34EA430C03D503
:10C38000FFF7E6FDFFF780FFF0BCBDE8008C2DE96C
:10C39000804C9A46934670B491E8380007C810F074
:10C3A000804F08BF13F0804F03D100F005F8FFF76E
:10C3B0006BFFF0BCBDE8008C20F07F4780EA0300F3
:10C3C00023F07F4C07EB0C03A3F57C5300F00040F7
:10C3D000A3F1FE0392F0000F00F0B38095F0000F80
:10C3E00000F077802DE901494FEA11404FEA1446E9
:10C3F00021EA004800FB06FC24EA064708FB06F693
:10C4000007FB08F800FB07F718EB06484CEB164C47
:10C410004FEA124B18EB07484FEA15464CEB174012
:10C4200022EA0B4E0BFB06FC25EA06470EFB06F63E
:10C4300007FB0EFE0BFB07F71EEB064E4CEB164CF4
:10C440004FF000061EEB074E4CEB174B18EB0B089A
:10C4500040F1000018EB0E0B58EB000840F1000013
:10C460008F1A4FF000013CBFC943661B14BFB5EBE8
:10C47000040C00213CBFC943F61B4FEA17444EEAA7
:10C480008E0E27EA04454FEA1C4704FB07622CEA9C
:10C49000074C05FB07F70CFB05F604FB0CFC16EB41
:10C4A000074642EB174216EB0C4642EB1C421BEBD5
:10C4B000060658EB0202414146EA9E0601D5BDE858
:10C4C0000189B619524141EB0101A3F10103BDE815
:10C4D00001894FEA14454FEA114724EA054621EA4B
:10C4E000074C05FB07F406FB07F70CFB06F105FB01
:10C4F0000CFC11EB074144EB17444FEA124711EBD8
:10C500000C4144EB1C4422EA074C05FB07F206FBF6
:10C5100007F70CFB06F605FB0CFC16EB074642EB97
:10C52000174216EB0C4642EB1C456A1854F1000109
:10C5300048BF7047B619524141EB0101A3F1010315
:10C54000704795F0000F37D04FEA11424FEA144779
:10C5500021EA024624EA074C02FB07F106FB07F733
:10C560000CFB06F402FB0CFC14EB074441EB1741F7
:10C570004FEA154714EB0C4441EB1C4125EA074CEC
:10C5800002FB07F506FB07F70CFB06F602FB0CFCAB
:10C5900016EB074645EB174516EB0C4645EB1C42E0
:10C5A000121951F1000148BF7047B619524141EBD1
:10C5B0000101A3F1010370474FEA14454FEA114707
:10C5C00024EA054621EA074C05FB07F106FB07F7BD
:10C5D0000CFB06F24FF0000605FB0CFC12EB0742C9
:10C5E00041EB174112EB0C4251EB1C4148BF704725
:10C5F000921841EB0101A3F101037047490050EA91
:10C60000C12018BF04204A0D18BF40F0010040F2BD
:10C61000FF72B2EB515F08BF40F00200012808BF73
:10C62000052070472DE9F0414F1E00EBC70104467D
:10C63000D1E9000115461E4637F006020DD02A4604
:10C64000334601F0DDFA7F1E04EBC703D3E9002374
:10C6500000F0C2FF37F00602F1D1022F25D0042FDF
:10C6600013D0062F18BFBDE8F0812A46334601F0EB
:10C67000C7FAD4E90A2300F0AFFF2A46334601F097
:10C68000BFFAD4E9082300F0A7FF2A46334601F099
:10C69000B7FAD4E9062300F09FFF2A46334601F09B
:10C6A000AFFAD4E9042300F097FF2A46334601F09D
:10C6B000A7FAD4E9022300F08FFF2A46334601F09F
:10C6C0009FFAD4E90023BDE8F04100F085BF0000E7
:10C6D000002213461046014901F03AB80000F03F2D
:10C6E000012201F058BE00F077BF00221346104629
:10C6F000114601F02DB840F2013200204FF0E04128
:10C7000001F049BE024A0020110701F044BE0000BA
:10C7100001FDFFFF30380A2801D2012070470020B8
:10C72000704700002DE9F041C1F30A52A2F2FF3632
:10C730002F4A304B0D460446142E2FDA002E12DA03
:10C7400000F04AFF0022134601F058FB4CD2002DA6
:10C75000A4BF0024254647DA25F00040204318BF37
:10C76000254D41D018E0DFF894C02CFA06F705EA11
:10C77000070C5CEA040C08BFBDE8F08100F02CFF58
:10C780000022134601F03AFB2ED2002D03DA4FF4BB
:10C790008010F0400544BD43002425E0332EC8BF7F
:10C7A000BDE8F081A6F1140C4FF0FF3727FA0CF723
:10C7B0003C4208BFBDE8F08101F056FB0022134661
:10C7C00001F01CFB10D2002D0DDA142E08BF6D1CD9
:10C7D00009D0C6F13400012101FA00F02044A04242
:10C7E00038BF6D1C0446BC4329462046BDE8F08195
:10C7F0009C7500883CE4377E0000F0BFFFFF0F000F
:10C800002DE9F04DC84A002490B0914205DA21F09C
:10C810000043934201D805D120B110B0BDE8F04DDE
:10C82000FFF75EBFB1F5801F1BDA53EA000209D0A3
:10C83000002911DA0120FEF762FC10B0BDE8F04DCE
:10C84000FFF753BF0220FEF75AFCFFF741FF10B07D
:10C8500081F00041BDE8F08D6FF03504362201F023
:10C860009AFD04EB2152C1F31308B049A2F2FF3341
:10C87000414401F4801282F07F6103EB225281F087
:10C880004051009241EA08010022A94B01F0DEFB71
:10C89000044608F10200A74EC0F313000D467E4483
:10C8A000032867D2D6E90023204601F0A9F81ED15B
:10C8B0000098002802BFD6E9000110B0BDE8F08D55
:10C8C00001F037F907460C469B4A9C4B01F098F95A
:10C8D00006460D469A4A9B4B3846214601F090F990
:10C8E00010B032462B46BDE8F04D00F075BE4FF05B
:10C8F0005532954B2046294601F082F90022934B90
:10C9000001F0B2FA06460F4622462B46104619465B
:10C9100001F076F932463B4601F072F9064600987E
:10C920000F46F0B101F005F980468A46824A834BF2
:10C9300001F066F932463B4601F096FA22462B4654
:10C9400001F084FB05460C467D4A7E4B404651462D
:10C9500001F056F910B02A462346BDE8F04D01F02B
:10C9600075BB0B4610B0324620462946BDE8F04D57
:10C9700001F06CBB00224FF08043204600F02CFEFB
:10C9800002460B462046294600F0E2FE06460F46C8
:10C99000009801F0CEF8CDE9040132463B4610463E
:10C9A000394601F02DF90C9069480C9A40440190E9
:10C9B00009910B46104601F023F98246024665486C
:10C9C0008B46C8F151080B4608F5D7280321784457
:10C9D000FFF728FE52465B4601F012F90A905E48C6
:10C9E0000D9152465B4604217844FFF71BFE099BDC
:10C9F0000C9A01F005F9844601980D9B40EA08085D
:10CA000060460A9A00F0E8FD83460891B8F1000FED
:10CA10004EDD4FF0FF322046294601F0BCFC224695
:10CA20002B4601F0EDF8804600988A4660B3DDE9B8
:10CA30000401414A414B01F0E3F8099100905A4644
:10CA400040465146089B00F0C7FD32463B4601F088
:10CA5000D7F8099B009A00F0BFFD4246534601F00B
:10CA600003FA22462B4601F0F1FA04460D46DDE9B1
:10CA70000401334A334B01F0C3F810B022462B4671
:10CA8000BDE8F04D01F0E2BA5A464046089B00F07E
:10CA9000A3FD32463B4601F0B3F84246534601F04F
:10CAA000E3F910B022462B46BDE8F04D01F0DCB9A9
:10CAB000009840B3DDE904011F4A204B01F0A0F8C3
:10CAC00080468A465A4620462946089B01F0BEFA0F
:10CAD00032463B4601F094F84246534601F0B6FA1E
:10CAE00022462B4601F0B2FA04460D46DDE9040168
:10CAF000134A144B01F084F810B022462B46BDE8CF
:10CB0000F04D01F0A3BA0B465A462046294601F0E3
:10CB10009DFA32463B4601F073F810B022462B4690
:10CB2000BDE8F04D01F0A0B90000F07F645F09009E
:10CB30000000F03FD62F0000763C7935EF39EA3D12
:10CB40000000E0FE422EE63F5555D53F0000E03F95
:10CB500086EBF9FFE62D0000E42D00002DE9F04DF5
:10CB60001D460C4698B0174621F0004123F00043C3
:10CB7000002814BF4FF0010C4FF0000C0CEB440CDC
:10CB8000FE4A0CEB02064FEA620C66452BD33E00D0
:10CB900018BF012606EB45061644F94A964222D3F1
:10CBA000F84A53EA070C02D0944205D148B918B0AC
:10CBB00000201146BDE8F08D002808BF4FF0000CA2
:10CBC00001D04FF0010C0CEB440212F5001F0AD803
:10CBD000002F14BF4FF0010C4FF0000C0CEB45027E
:10CBE00012F5001F07D918B03A462B462146BDE87A
:10CBF000F04DFFF778BD0022DFF88CA3002CB8BF02
:10CC0000534526DADFF884C36345A8BF022220DA41
:10CC1000DFF870C39C451CDCDFF874C30CEB235CAD
:10CC2000BCF1140F08DDCCF1340627FA06FC0CFA2F
:10CC300006F6BE420DD108E05FB9CCF1140623FA26
:10CC400006FC0CFA06F69E4203D10CF00102C2F17A
:10CC5000020251EA000C19D1002D17DA002C18BF7E
:10CC6000022A01D0012A07D00220FEF748FA18B0A4
:10CC7000BDE8F04DFFF72CBD0220FEF740FAFFF7AC
:10CC800027FD18B081F00041BDE8F08DB7F1000C30
:10CC90006CD1534525D104F1804212F5801201BFB9
:10CCA00000280020B74918B008BFBDE8F08DB5488E
:10CCB000884207DC002DA1BF6046294618B0BDE8B8
:10CCC000F08D07E0281E05DA80F0004118B06046BC
:10CCD000BDE8F08DAF497944D1E9000118B0BDE855
:10CCE000F08DDFF8A0C2634525D1002D1FDA19B100
:10CCF000514512D1D8B909E0002840F0EC82A24A8F
:10CD0000214618B062F31E01BDE8F08D00202146D7
:10CD100018B060F31E01BDE8F08D08DA18B02346A4
:10CD2000BDE8F04D02460020614600F011BD18B08C
:10CD30002146BDE8F08D514518DAB5F1804F0DD090
:10CD4000A5F1005CBCF1FF5C10D1B4F1000C0DDB6F
:10CD500018B06146BDE8F04D00F0ECBB234618B0BA
:10CD60000246BDE8F04D194600F04ABF060024F027
:10CD7000004C3BD1D9B1514533D1002C06DD002DFB
:10CD8000A1BF0020514618B0BDE8F08D002C01DD98
:10CD9000002D1BDB002C13DA002D11DB012A4FF0D4
:10CDA000000014BF78497C4918B0BDE8F08D022A14
:10CDB00018BF002C0AD0012A08D1002C06DA0AE09C
:10CDC000002CB8BF002D11DA012A04D0002018B0C1
:10CDD0000146BDE8F08D18B000204FF00041BDE8DD
:10CDE000F08DA1F14050B0F17F601AD0012000EB2E
:10CDF000E47050EA020421D0624C521E4FF0000B46
:10CE0000104304BF4FF0000B644C654883427CDD47
:10CE1000644A654893421FDD884217DB002D25DBFD
:10CE200037E0002C00DA4AB1022A0CBF01204FF093
:10CE3000FF3018B0BDE8F04D00F07BBE0120FEF7DA
:10CE40005EF918B0BDE8F04DFFF74FBC4D4A8A427D
:10CE500002DC002D0ADC1CE0814202DA002D18DA27
:10CE600004E0484B994220DD002D12DD0220FEF740
:10CE700046F9FFF740FC05460E4600225346584649
:10CE8000214600F0BDFE18B066F31E012846BDE83D
:10CE9000F08D0220FEF733F9FFF734FC0A462146F5
:10CEA00018B062F31E01BDE8F08D002230466146E5
:10CEB00001F0CCF880460E466FF0010201F06BFAEB
:10CEC0004FF05532394B00F0CFFF4246334600F069
:10CED00097FE0022364B00F0C7FF8246424633469B
:10CEE00004911046194600F08BFE5246049B00F058
:10CEF00087FE8A4600904FF0C0422E4B4046314696
:10CF000000F07EFE2C4A2B4B00E027E0CDE9060125
:10CF10005146009800F074FE82460191274A284B42
:10CF20004046314600F06CFE5246019B01F08EF8FF
:10CF300082460B4602460591DDE9060100F04CFBF6
:10CF4000DDE9062300268846304601F07FF8524688
:10CF5000059B00F089FF024600F07EB90020B1F584
:10CF6000801F07DA35223046614601F014FA064682
:10CF70006FF0340000EB215024E00000FFFF1F00A1
:10CF8000FFFF0F000000F03F0000F07F0000404373
:10CF900001FCFFFF9E2B00000000F0FF0000F0BF2F
:10CFA0000000E0410000F043FFFFEF3F5555D53F43
:10CFB0000000E03F4715F73FFE822B6544DF5DF838
:10CFC0000BAE543EA0F2FF300190C1F3130040F0CD
:10CFD0007F6141F040510291FE498842D8BF002054
:10CFE00004DDFD498142C8BF012001DD0D9008E04C
:10CFF00000200D900198401C01900298A0F580102F
:10D0000002900299F54878440B910D9900EBC1000C
:10D01000D0E900230F9330460A920B9901F016F8DD
:10D02000CDE90601DDE90A2130460F9B00F0D4FA74
:10D0300002460B460020EA4900F08AFB05910246B1
:10D040000B460090DDE9060100F0DAFD1490E5489A
:10D050008A464FF0000878440299006812904FF019
:10D06000005040EA61010D980F9B01EB804000F5F4
:10D07000002109910A9A129800F0E8FF32460B9BB2
:10D0800000F0F2FE4246534600F0BAFD0646029119
:10D0900040465146099B129A00F0B2FDDDE9062395
:10D0A00000F0E2FE3246029B00F0D0FF059B009AA2
:10D0B00000F0A6FD0091149A0490534610461946BC
:10D0C00000F09EFD06460246C7480B460291062127
:10D0D0007844FFF7A7FACDE90510029B32461046C7
:10D0E000194600F08DFDDDE9053200F089FD05915E
:10D0F0000646534640461946149A00F06DFA009BC6
:10D10000049A00F07DFD3246059B00F065FACDE9FA
:10D110000510424653461046194600F071FD0022A4
:10D12000B24B02910A9000F057FADDE9053200F0A7
:10D1300053FA0E464246AD4B404600F087FF029B35
:10D140000A9A00F083FFDDE9053200F08DFE4246C9
:10D1500002910A9033461046514600F051FDCDE948
:10D1600006015346149A02990A9800F049FD8A462E
:10D170000290334642460099049800F041FD534620
:10D18000029A00F029FA82460B4602460591DDE933
:10D19000060100F021FADDE9062300208846064654
:10D1A00000F054FF5246059B00F05EFE8246099156
:10D1B0004FF060428E4B3046414600F021FD049016
:10D1C00006918C4A8A4B5046099900F019FD824617
:10D1D0000291894A894B3046414600F011FD524682
:10D1E000029B00F0F9F9864B7B440D9A03EBC203D6
:10D1F000D3E9002300F0F0F90E900791019800F0B8
:10D2000098FC0591DDE9061382460E9A049800F019
:10D21000E3F97C4A7A440D9B02EBC303D3E9002374
:10D220000093029200F0D8F95246059B00F0D4F921
:10D230000026884652463046059B00F007FF009BBB
:10D24000029A00F003FF069B049A00F0FFFE079B82
:10D250000E9A00F009FE024600200B460290384666
:10D26000294600F0CDFC824601912B4638461946EE
:10D27000029A00F0EBFE3246434600F0C1FC5246F3
:10D28000019B00F0A9F907468A46324643462946E3
:10D29000029800F0B5FC05460E463A46534600F0AB
:10D2A0009BF9594A8846914221DBA8EB020353EAD5
:10D2B000000210D12A46334600F0C8FECDE9040131
:10D2C000524A534B3846514600F086F9DDE90423B3
:10D2D00000F094FD21D20220FDF711FFFFF70BFAB9
:10D2E0000A46214618B062F31E01BDE8F08D494B95
:10D2F00028F000429A4210D3474A08EB020353EA4F
:10D3000000027FF4C6AD2A46334600F09FFE3A463F
:10D31000534600F073FD7FF6BCAD0022019228F069
:10D3200000403E493E4A01EB2051824223DA481C2C
:10D330004FF4801121FA00F040443A4AC0F30A51F8
:10D340007A44394BA1F2FF31CB4020EA0303C0F30A
:10D35000130040F48010C1F11401C840126801901C
:10D36000B8F1000FBCBF404201902846314600F0A2
:10D370006DFE05460E462A4633463846514600F0B5
:10D380002BF94FF000084246284B4046059100F02B
:10D3900037FCCDE90601264A264B4046059900F0A8
:10D3A0002FFC009102902A4633464046059900F032
:10D3B0004DFE3A46534600F057FD1F4A1F4B00F002
:10D3C0001FFC009B029A00F007F9074688460246B8
:10D3D0000B4635E08E9803007AB60B00E627000076
:10D3E0000000F03F1E2800004C270000000008400D
:10D3F00009C7EE3FFD033ADCF5015B14E02F3EBEAA
:10D4000024260000E825000000009040FE822B65E5
:10D410004715973C00CC904000346F3F01FCFFFF64
:10D420000000E03F34250000FFFF0F00432EE63FE1
:10D43000396CA80C615C20BEEF39FAFE422EE63F43
:10D44000DDE9060100F0C8F8DDE9062305460E46D1
:10D4500000F0FCFD3A46434600F006FD0F462A4622
:10D46000334600901046194600F0CAFB8246024639
:10D470002E4888460B4605217844FFF7D3F85246DC
:10D48000434600F0BDFB2A46334600F0EDFC8046E3
:10D490008A463B4628463146009A00F0B1FB3B469F
:10D4A000009A00F099F80691009000224FF0804316
:10D4B0004046514600F0CAFD0F460C904246534686
:10D4C0002846314600F09CFB3B460C9A00F040F9A0
:10D4D000069B009A00F0BAFD2A46334600F0B6FDDE
:10D4E0000022134B00F0C0FC054601980E4601EBEC
:10D4F00000510815002810DC28463146019A00F03A
:10D500004AFFFFF77BF8042808BFFFF7FBF828461F
:10D510003146019A00F03FFF05460B4618B02A46F7
:10D5200058462146BDE8F04D00F06ABBD423000008
:10D530000000F03F2DE9F04106460F4600F0A0FC48
:10D54000041E0D4618BF0120284320F00040C0F102
:10D550007F6000F1E040C00F0ED0301C18BF0120EA
:10D56000384320F00040C0F17F6000F1E040C00F80
:10D5700004BF0120FDF7C3FD20462946BDE8F08128
:10D5800010B500290AD00878002807D0054878444B
:10D59000FEF72CFC002801D0002010BD0248784482
:10D5A00010BD0000CE280000C628000010B50029DC
:10D5B0000AD00878002807D005487844FEF716FC02
:10D5C000002801D0002010BD0248784410BD0000A2
:10D5D000B2290000AA29000010B591EA030F48BF44
:10D5E00083F0004300F13A85841A71EB030C05D2F5
:10D5F000121943EB0C03001B61EB0C01DFF824E173
:10D600004FEA1154A4EB135C1EEA430F18BF9EEAC5
:10D61000445F73D023EA0E03DCF1200E21EA0451AB
:10D6200043F4801332D322FA0CFE10EB0E0023FADF
:10D630000CFE41EB0E01CCF1200E03FA0EFE10EBB6
:10D640000E0051F10001B1F5801FCCF1200E32D255
:10D6500001EB045112FA0EF2BDE8104058BF7047BA
:10D66000401C38BF5FEA420218BF7047002814BF51
:10D6700020F0010041F100014FEA410313F5001FC2
:10D6800038BF7047A1F1C04100F0B2BB012A43EBA3
:10D690000302ACF1200CDCF11F0E32BF4FF0000E84
:10D6A00023FA0CF310EB030041EB0451B4EB115FD0
:10D6B000D0D0A1EB045101F5801149085FEA300098
:10D6C00001EB04510ED350F1000038BF12FA0EFEE8
:10D6D00008D1BDE81040C9E7401C38BF5FEA4202EC
:10D6E000CAD1C3E7BDE810404FEA410313F5001F5C
:10D6F00038BF7047A1F1C04100F07ABB9EEA445F99
:10D7000008D011EA5E0FBDE8104004BF01F00041EF
:10D7100000207047BDE8104070B500F01BFB00BF53
:10D7200064FBBE3E0000E0FF02494FF0000000F045
:10D7300000BE00BF0000F87F491058BFC1F1404152
:10D740005B1058BFC3F140438B42EFF3008070473A
:10D750002DE9C04130B4DFF8A0C23CEA111418BF73
:10D760003CEA131400F0EC8081EA03051CEA111472
:10D7700044EAD57418BF1CEA131500F0C780A4EB67
:10D7800005044FF0004545EAC12145EAC32341EABB
:10D79000505143EA525304F17F74994204F5003426
:10D7A0004FEAC0204FEAC22208BF904200F09C809E
:10D7B0004FEA13650FF24016765D4FEA134506FBFC
:10D7C00005F7C7F1807706FB07F74FEAD737A7FBC6
:10D7D00003687642C8F58038A7FB06CE38BFA8F1AB
:10D7E000010807FB08E64FF0000EA6FB028CE6FBE3
:10D7F00003CEDCF1000CCEF1004E38BFAEF1010ECD
:10D80000A6FB0C584FF000074FF00005E6FB0E8713
:10D81000A1FB08C6A0FB07CE16EB0E0645F10005DE
:10D82000E1FB076515F1E04E7EBFA4F580345FEAA9
:10D8300046066D4116F1800745F100054FEA1727AE
:10D840004FEA066647EA0567A6F1DE46B6F1805F55
:10D850004FEA15251FD9384624F0010C05EBC47199
:10D86000BCF1FE6F01EB0C1102D8F0BCBDE80081E9
:10D8700024425CBF01F5801E9EEAC47F02D4F0BC46
:10D88000BDE80081244238D4F0BCA1F1C041BDE81C
:10D89000004100F0ADBA4FEAD22242EA43524FEAC9
:10D8A000D323A7FB02864FEAD02040EA415007FB72
:10D8B00003661EEA0E0F4FEAD12105FB026658BF30
:10D8C000A6EB0056B6EB00564FEA520E4EEAC37E68
:10D8D00018EB0E0E56EB530EBDD518EB02085E4149
:10D8E0007F1C55F10005B6E74FF480154FF0000797
:10D8F0004FF000064FF00008ADE7F0BC4FF000001D
:10D9000001F1C04101F00041BDE8008111EA0C1FA6
:10D910000CEA131500D00CE013EA0C1F00F0258070
:10D920004FF00000F0BC81EA030101F00041BDE8C6
:10D930000081F0BCBDE8004181EA030100F058BA63
:10D94000F0BCBDE8004170B500F004FA097EFC3E71
:10D9500000F007B881EA03014FF0000001F0004138
:10D96000704781EA030100F043BAF0BCBDE8004112
:10D970004FF0000021497047FFFDFBF9F7F5F4F285
:10D98000F0EEEDEBE9E8E6E4E3E1E0DEDDDBDAD85A
:10D99000D7D5D4D3D1D0CFCDCCCBCAC8C7C6C5C4B8
:10D9A000C2C1C0BFBEBDBCBBBAB9B8B7B6B5B4B3CF
:10D9B000B2B1B0AFAEADACABAAA9A8A8A7A6A5A4BA
:10D9C000A3A3A2A1A09F9F9E9D9C9C9B9A9999987E
:10D9D0009797969595949393929191908F8F8E8E21
:10D9E0008D8C8C8B8B8A89898888878786858584AE
:10D9F00084838382828181800000FF070000F87F9A
:10DA000051EA030C17D41CF5801F58BFBCF5801FCA
:10DA100000F10680994218BF704708BF90427047D6
:10DA200007D711F5801F58BF13F5801F19D49942ED
:10DA30007047894270471CF5801F08D5BCF5801FD0
:10DA4000F7D58B4218BF704708BF824270474FF42A
:10DA5000001C1CEB410F38BF1CEB430F01D28B4263
:10DA6000704770B500F076F9922449004FF00051EC
:10DA70004FF08053FFF760BE4FEA41034FEA535324
:10DA8000A3F58063D3F11E03C8BFD3F1210C0CDDD5
:10DA90004FF0004242EAC12242EA505232FA03FCFD
:10DAA0008CEAE17CACEBE1707047102BC4BF002026
:10DAB000704703F5787CBCF1FF3F04D06FF0004263
:10DAC00082EA2100704770B500F044F94992248041
:10DAD00000207047F2E700004FEA1153A3F580637E
:10DAE000D3F11E03A8BFD3F1200C08DB4FF0004296
:10DAF00042EAC12252EA505232FA03F07047094218
:10DB00000BD4102BC4BF0020704703F5787CBCF108
:10DB1000FF3F05D04FF0FF3070474FF000007047D7
:10DB200070B500F017F900BF4992248000207047BB
:10DB3000F0E710F0004248BF4042B0FA80F310FA1C
:10DB400003F10AD0C3F11D0303F580634FEA41508E
:10DB500002EB035202EBD12170474FF000007047F7
:10DB6000B0FA80F310FA03F10AD0C3F11D0303F5F4
:10DB700080634FEA41504FEA035202EBD1217047D4
:10DB80004FF000007047000051EA030C17D41CF559
:10DB9000801F58BFBCF5801F00F10680994218BF56
:10DBA000704708BF9042704707D711F5801F58BFD4
:10DBB00013F5801F19D499427047894270471CF5AC
:10DBC000801F08D5BCF5801FF7D58B4218BF704762
:10DBD00008BF824270474FF4001C1CEB410F38BF56
:10DBE0001CEB430F01D28B42704770B500F0B2F8C6
:10DBF000922449004FF000514FF08053FFF79CBD35
